:100000000C9423280C9454280C9454280C945428B1
:100010000C9454280C9454280C9454280C94542870
:100020000C9454280C9454280C9454280C94542860
:100030000C9454280C94534E0C9454280C9454282B
:100040000C9454280C94AC5D0C9454280C945428B3
:100050000C9454280C9454280C946FCB0C94B350EB
:100060000C9454280C94D08F0C9454280C9454283D
:100070000C9454280C9454280C9454280C94542810
:100080000C9454280C9454280C9454280C94542800
:100090000C9454280C9454280C9454280C945428F0
:1000A0000C9454280C9454280C9454280C945428E0
:1000B0000C9454280C9454280C9454280C945428D0
:1000C0000C9454280C9454280C9454280C945428C0
:1000D0000C9454280C9454280C9454280C945428B0
:1000E0000C945428314F344F234F274F2D4F6B4FD3
:1000F000384F3C4F424F464F4A4F504F544F584F46
:100100006B4F5E4F624F664FCF4FD44FD94FE34F87
:10011000ED4F6650F74FFF4F075011501B502550C1
:1001200034503E506650485052505C50084AD73BBD
:100130003BCE016E84BCBFFDC12F3D6C74319ABDB6
:1001400056833DDA3D00C77F11BED9E4BB4C3E91DA
:100150006BAAAABE000000803F05A84CCDB2D44EC9
:10016000B93836A9020C50B9918688083CA6AAAACB
:100170002ABE000000803F004E414E494E4954596E
:10018000494E46CDCCCC3D0AD7233C17B7D1387762
:10019000CC2B329595E6241FB14F0A000020410078
:1001A00000C84200401C4620BCBE4CCA1B0E5AAEC2
:1001B000C59D74434F4D4D554E49434154494F4E93
:1001C0000044525952554E004552524F5253004925
:1001D0004E464F004543484F0047322F4733206279
:1001E000616420706172616D65746572730A005399
:1001F0006C6565702E2E2E00205A3A200020593A48
:10020000200042656420583A2000436865617033DD
:100210004420563330302072656164792E00526577
:1002200073756D696E67207072696E7400436C69D6
:10023000636B20746F20726573756D652E2E2E00B2
:10024000456E642066696C65206C6973740A0042AF
:100250006567696E2066696C65206C6973740A0055
:100260005344207072696E74696E67206279746598
:1002700020004E6F74205344207072696E74696E52
:10028000670A0046696C652064656C657465643A4C
:100290000044656C6574696F6E206661696C6564A5
:1002A0002C2046696C653A20006F70656E2066618F
:1002B000696C65642C2046696C653A200025697379
:1002C0000025696D20256973002569682025696D01
:1002D0002025697300256964202569682025696DDA
:1002E00020256973002569792025696420256968BE
:1002F0002025696D20256973005072696E74207421
:10030000696D653A200050726F746563746564208E
:1003100050696E0A004525692025730043686561B0
:1003200070334420563330302072656164792E007A
:10033000D401CF01C801C101B3016F666600444515
:100340004255473A004B494C4C45442E20004D3114
:1003500031332053006F6B0048656174696E67200C
:10036000646F6E652E003F0A0020573A00452569EC
:100370002025730043686561703344205633303064
:100380002072656164792E0042656420646F6E6539
:100390002E003F0A0020573A0042656420486561FC
:1003A00074696E672E00436865617033442056336C
:1003B0003030204F66662E0056333030204C3120CE
:1003C000423A312054303A312054313A30204649B3
:1003D000524D574152455F4E414D453A4D61726C09
:1003E000696E20312E312E3020284769746875627D
:1003F0002920534F555243455F434F44455F555263
:100400004C3A68747470733A2F2F67697468756218
:100410002E636F6D2F4D61726C696E4669726D77D8
:100420006172652F4D61726C696E2050524F544F4E
:10043000434F4C5F56455253494F4E3A312E302070
:100440004D414348494E455F545950453A436865CC
:10045000617033442056333030204558545255444F
:1004600045525F434F554E543A3120555549443A11
:1004700063656465326132662D343161322D343703
:1004800034382D396231322D633535633632663377
:10049000363766660A0053657474696E6720547255
:1004A0006176656C20416363656C65726174696F28
:1004B0006E3A200053657474696E672052657472D9
:1004C00061637420416363656C65726174696F6E0A
:1004D0003A200053657474696E67205072696E74B7
:1004E00020416363656C65726174696F6E3A2000C8
:1004F00053657474696E67205072696E7420616E02
:10050000642054726176656C20416363656C65722A
:100510006174696F6E3A2000205A0020590058001B
:1005200020204D61783A2000205A002059005800C0
:1005300020204D696E3A20004F6E20004F66660005
:10054000536F667420656E6473746F70733A200025
:1005500020643A0020693A0020703A0043290A00DA
:1005600061626C656420286D696E2074656D702011
:1005700000436F6C642065787472756465732061E4
:100580007265200023646566696E652020444546D7
:1005900041554C545F4B64200023646566696E6569
:1005A000202044454641554C545F4B69200023644C
:1005B0006566696E65202044454641554C545F4B45
:1005C000702000504944204175746F74756E652029
:1005D00066696E697368656421205075742074685B
:1005E00065206C617374204B702C204B6920616E08
:1005F00064204B6420636F6E7374616E7473206645
:10060000726F6D2062656C6F7720696E746F204326
:100610006F6E66696775726174696F6E2E680A0025
:10062000504944204175746F74756E652066616928
:100630006C6564212074696D656F75740A0050499A
:1006400044204175746F74756E65206661696C65D0
:1006500064212054656D70657261747572652074D3
:100660006F6F20686967680A00204B643A20002099
:100670004B693A2000204B703A20000A20436C61FD
:100680007373696320504944200A002054753A204E
:1006900000204B753A2000206D61783A2000206DD3
:1006A000696E3A200020643A200020626961733A42
:1006B00020004F666673657473206170706C6965A5
:1006C00064004572723A20546F6F20666172210097
:1006D000546F6F206661722066726F6D207265665E
:1006E0006572656E636520706F696E740A004545BA
:1006F00050524F4D2064697361626C65640A003A20
:1007000020007A5F6D696E3A20202D3230207A5FAA
:100710006D61783A20203230005A204F666673654A
:100720007420004E6F2063617365206C6967687484
:100730000A00416374697665204578747275646552
:10074000723A2000556E6B6E6F776E20636F6D6D21
:10075000616E643A20220025753A253032750025F5
:100760003032753A253032750025756420253032D7
:10077000753A25303275005A00590058000920009A
:100780000000000000000000000000007FFFE0000B
:1007900000000000000000000000007000E0000009
:1007A0000000000000000000000061F86000000090
:1007B00000000000000000000041F82000000000E0
:1007C000000000000000000040F0200000000000D9
:1007D0000000000000000040602000000000000059
:1007E0000000000000005801A07F80000000000011
:1007F00000004104005C63A0FFC000000000000096
:10080000002082005EF7A0FFC00000000000000092
:100810002082005EF7A0FFC0000000000000004141
:1008200004005C63A07F80000000000000008208DC
:10083000005801A07F8000000000000001041000AB
:10084000406020FFC00000000000000104100040D4
:10085000F020FFC00000000000000082080041F806
:1008600020FFC00000000000000041040061F860AB
:100870003F00000000000000000000007000E01ECB
:100880000000000000000001FFFF807FFFE00C007F
:1008900000000000000001FFFF80000000000000D9
:1008A0000000000000000000007FFFE000000000EA
:1008B00000000000000000007000E00000000000E8
:1008C00000000000000000630C6000000000000059
:1008D000000000000000470E2000000000000000A3
:1008E00000000000004F0F2000000000000000008A
:1008F000000000005F0FA0000000000000000000EA
:100900000000005E07A07F800000000000000041A2
:100910000400406020FFC0000000000000002082B2
:100920000040F020FFC00000000000000020820016
:1009300040F020FFC0000000000000004104004023
:1009400060207F80000000000000008208005E0739
:10095000A07F80000000000000010410005F0FA0D5
:10096000FFC0000000000000010410004F0F20FF36
:10097000C000000000000000820800470E20FFC0F9
:1009800000000000000000410400630C603F000014
:100990000000000000000000007000E01E000000E9
:1009A0000000000001FFFF807FFFE00C000000005E
:1009B00000000001FFFF800000005072696E74208B
:1009C00061626F72746564004E6F205344206361EE
:1009D0007264005072696E742066726F6D205344A9
:1009E0000053746F70207072696E74005265737575
:1009F0006D65207072696E7400506175736520704A
:100A000072696E7400436F6E74726F6C0050726521
:100A1000706172650054756E6500496E666F207373
:100A2000637265656E0000060900FE0000000000AC
:100A300001090008FE000005080806000040F0C893
:100A40008888987810050808060000C0F88888880B
:100A50008888F80505050600012030F830200508D3
:100A6000080600002070F820202020E00509090673
:100A700000FF2070A8A8B888887020050909060022
:100A8000FFE080C0B0A8283028280509090600FF2B
:100A9000F8A88888888888A8F8050A0A0600FE2031
:100AA0005050505088A8A8887003030306000340E4
:100AB000A04000002200250028002B002E0031005D
:100AC000340002010000050108010B0100002000B4
:100AD0002300260029002C002F0032000001000016
:100AE00003010601090105050505070508080808B1
:100AF000020202020A0A08080404040401010101B6
:100B000001010101030303030303030304070707B0
:100B10000C0C0C0C0C0C0C0C020202020606060655
:100B2000060606060B0B0B0B0B0B0B0B0102102022
:100B30002008081020401020408002010201080413
:100B400002010102040810204080804020100804A7
:100B50000201800402018040201008040201080400
:100B60000201010204081020408001020408102044
:100B7000408000000A0B02090C0D0E080703040157
:100B80000000000000000000000000000000000065
:100B90000000000000000000000000000000121132
:100BA0001000000000000000000000000000000035
:100BB00000000000000000004B494C4C45442E2032
:100BC00000202D20496E76616C696420657874720E
:100BD00075646572206E756D62657220210A002051
:100BE00020506C616E6E6572427566666572427900
:100BF0007465733A20002046726565204D656D6FFF
:100C000072793A2000436F6D70696C65643A204DCB
:100C1000617920323320323031370A00207C204184
:100C20007574686F723A20286E6F6E652C2064654B
:100C30006661756C7420636F6E666967290A00329D
:100C40003031372D30352D30342031323A303000CC
:100C5000204C61737420557064617465643A20009F
:100C6000312E312E300A004D61726C696E002053B6
:100C70006F6674776172652052657365740A00202F
:100C80005761746368646F672052657365740A0006
:100C90002042726F776E206F757420526573657491
:100CA0000A002045787465726E616C205265736528
:100CB000740A00506F77657255700A007374617220
:100CC000740A006572726F722077726974696E6758
:100CD00020746F2066696C650A00456E6473746FDA
:100CE0007073202563202563202563202563002061
:100CF0005A3A0020593A0020583A00656E647374DD
:100D00006F7073206869743A2000446F6E652073B9
:100D10006176696E672066696C652E0A004D32390E
:100D20000002436172642072656D6F7665640043F2
:100D300061726420696E73657274656400000021DD
:100D400000240027002A002D00300033000101009C
:100D500000040107010A0100060900FE07019203D1
:100D60002120FFFF08FF07FF000000060000010729
:100D70000706020080808080800080030202060156
:100D800005A0A00507070600005050F850F8505085
:100D90000507070600002078A07028F02005070747
:100DA000060000C0C810204098180507070600007C
:100DB0006090A040A89068020303060104C0408030
:100DC00003070706010020408080804020030707BA
:100DD0000601008040202020408005050506000116
:100DE00020A870A8200505050600012020F8202075
:100DF0000203030602FFC04080050101060003F85C
:100E0000020202060200C0C0050505060001081026
:100E10002040800507070600007088888888887051
:100E200003070706010040C040404040E0050707B7
:100E3000060000708808708080F80507070600002B
:100E4000F81020100808F0050707060000103050C1
:100E500090F81010050707060000F880F0080888D1
:100E600070050707060000708080F088887005070D
:100E700007060000F80810202020200507070600BC
:100E800000708888708888700507070600007088E1
:100E90008878080870020505060200C0C000C0C0BE
:100EA0000206060602FFC0C000C040800407070615
:100EB000000010204080402010050303060002F8C7
:100EC00000F804070706010080402010204080053C
:100ED0000707060000708808102000200507070695
:100EE000000070880868A8A8700507070600007051
:100EF0008888F8888888050707060000F08888F049
:100F00008888F00507070600007088808080887058
:100F1000050707060000F08888888888F00507071D
:100F2000060000F88080F08080F8050707060000C2
:100F3000F88080F0808080050707060000708880B8
:100F4000B8888870050707060000888888F88888B0
:100F50008801070706020080808080808080050766
:100F600007060000381010101090600507070600F3
:100F7000008890A0C0A09088050707060000808028
:100F800080808080F805070706000088D8A8888838
:100F900088880507070600008888C8A898888805FB
:100FA000070706000070888888888870050707068C
:100FB0000000F08888F08080800507070600007038
:100FC000888888A89068050707060000F08888F0E0
:100FD000A09088050707060000788080700808F058
:100FE000050707060000F82020202020200507071D
:100FF0000600008888888888887005070706000032
:101000008888888888502005070706000088888817
:101010008888A85005070706000088885020508857
:1010200088050707060000888888502020200507CB
:1010300007060000F80810204080F80307070601A3
:1010400000E08080808080E005050506000180408A
:10105000201008030707060100E02020202020E0E0
:10106000050303060004205088050101060000F86E
:101070000202020602058040050505060000700810
:101080007888780507070600008080B0C88888F057
:1010900005050506000070808088700507070600BA
:1010A000000808689888887805050506000070889B
:1010B000F880700507070600003048E040404040D7
:1010C0000506060600FF7088887808700507070681
:1010D00000008080B0C88888880107070602008069
:1010E0000080808080800308080601FF2000202007
:1010F0002020A040040707060000808090A0C0A028
:1011000090030707060100C04040404040E005054D
:1011100005060000D0A8A8A8A8050505060000B08F
:10112000C8888888050505060000708888887005CD
:1011300006060600FFF08888F08080050606060097
:10114000FF788888780808050505060000B0C88083
:10115000808005050506000070807008F004070710
:101160000600004040E04040403005050506000014
:1011700088888898680505050600008888885020BA
:101180000505050600008888A8A850050505060085
:101190000088502050880506060600FF8888887859
:1011A0000870050505060000F8102040F803070741
:1011B0000601002040408040402001070706020051
:1011C0008080808080808003070706010080404087
:1011D00020404080050202060002689000000006E0
:1011E00000000000000600000000000600000000F3
:1011F00000060000000000060000000000060000DD
:1012000000000006000000000006000000000006CC
:1012100000000000000600000000000600000000C2
:1012200000060000000000060000000000060000AC
:10123000000000060000000000060000000000069C
:101240000000000000060000000000060000000092
:10125000000600000000000600000000000600007C
:10126000000000060000000000060000000000066C
:101270000000000000060000000000060000000062
:10128000000600000000000600000000000600004C
:10129000000000060000000000060000000000063C
:1012A00000000000000600000107070602008000A1
:1012B00080808080800507070600002070A8A0A815
:1012C0007020050707060000304040E04050A805A8
:1012D00005050600008870507088050707060000A5
:1012E000885020F820F8200107070602008080803F
:1012F00000808080050808060000304820505020FB
:101300009060030101060107A0050707060000F829
:1013100088B8B8B888F8050707060001700878880B
:101320007800F80505050600012850A0502805039F
:1013300003060001F80808020202060206408005C2
:101340000707060000F888A88898A8F80501010694
:101350000006F80404040600036090906005070787
:101360000600002020F8202000F8040505060003F0
:1013700060902040F0030505060003E020E020E037
:1013800002020206020640800508080600FF88885F
:10139000888898E880800507070600007898987884
:1013A000181818020202060202C0C0020202060257
:1013B000FF408003050506000340C04040E00507EC
:1013C00007060001708888887000F805050506008A
:1013D00001A0502850A00507070600008890A858D3
:1013E000B808080507070600008890B84898203814
:1013F000050808060000C040C048D838080805079E
:1014000007060000200020408088700508080600BC
:10141000004020007088F888880508080600001041
:1014200020007088F8888805080806000020500011
:101430007088F888880508080600006890007088A1
:10144000F888880508080600005000708888F88829
:10145000880508080600002050207088F888880554
:1014600007070600003860A0B8E0A0B80508080625
:1014700000FF7088808088702060050808060000E2
:10148000402000F880F080F80508080600000810E9
:1014900000F880F080F8050808060000205000F8E9
:1014A00080F080F80507070600005000F880F08003
:1014B000F8030808060100804000E0404040E003D7
:1014C0000808060100204000E0404040E003080812
:1014D00006010040A000E0404040E003070706018D
:1014E00000A000E0404040E005070706000070480B
:1014F00048E848487005080806000068900088C859
:10150000A898880508080600004020708888888808
:10151000700508080600001020708888888870050B
:1015200008080600002050007088888870050808A8
:10153000060000689000708888887005080806001A
:1015400000500070888888887005050506000188AD
:10155000502050880508080600FF1070A8A8A8A809
:101560007040050808060000402088888888887038
:1015700005080806000010208888888888700508FB
:101580000806000020500088888888700508080632
:1015900000005000888888888870050808060000C8
:1015A00010208850202020200509090600FFC04097
:1015B000704848704040E00408080601FF609090C1
:1015C000A09090E080050808060000402000700808
:1015D00078887805080806000010200070087888D0
:1015E0007805080806000020500070087888780503
:1015F00008080600006890007008788878050707DA
:101600000600005000700878887805080806000079
:101610002050207008788878050606060000D0283B
:1016200078A0A8500506060600FF7080887020602C
:101630000508080600004020007088F88070050842
:10164000080600001020007088F880700508080661
:1016500000002050007088F8807005070706000021
:1016600050007088F8807003080806010080400070
:1016700040C04040E003080806010020400040C090
:101680004040E003080806010040A00040C0404080
:10169000E0030707060100A00040C04040E0050746
:1016A00007060000A040A010788870050808060012
:1016B00000689000B0C888888805080806000040C7
:1016C0002000708888887005080806000010200037
:1016D000708888887005080806000020500070880F
:1016E000888870050808060000689000708888885F
:1016F000700507070600005000708888887005058F
:10170000050600012000F800200507070600FF106D
:1017100070A8A8A8704005080806000040200088AE
:1017200088889868050808060000102000888888C6
:101730009868050808060000205000888888986886
:101740000507070600005000888888986805090981
:101750000600FF102000888888F808700407070634
:1017600001FFC04060506040E00508080600FF50DF
:101770000088888878087024F4D43050C38E20C242
:10178000A24017828B7011127A910D816CD90AA830
:1017900061E108C7586607615143061E4B5D05C1EC
:1017A00045A7041A411104093D98037139310340DA
:1017B00036DB0265339102D4305402802E1D026361
:1017C0002CEE01752AC501B028A001102781018FD8
:1017D0002564012B244B01E0223401AC211F018D33
:1017E000200D01801FFC00841EED00971DDF00B856
:1017F0001CD200E61BC600201BBC00641AB200B25B
:1018000019A8000A19A0006A189900D11791004080
:10181000178B00B516840031167E00B31579003A97
:10182000157300C7146F0058146A00EE1366008821
:1018300013630025135E00C7125B006C125700157E
:10184000125400C111510070114F0021114B00D6EC
:101850001049008D1047004610440002104200C09D
:101860000F4000800F3E00420F3C00060F3B00CBB4
:101870000E3800930E37005C0E3500270E3400F34F
:101880000D3200C10D3100900D3000600D2E003280
:101890000D2D00050D2C00D90C2B00AE0C29008558
:1018A0000C29005C0C2700350C27000E0C2600E8E4
:1018B0000B2400C40B2400A00B23007D0B23005A33
:1018C0000B2100390B2100180B2000F80A1F00D94A
:1018D0000A1E00BB0A1E009D0A1D00800A1D00632F
:1018E0000A1C00470A1B002C0A1B00110A1A00F7E9
:1018F000091A00DD091900C4091900AB0919009281
:101900000917007B091800630917004C09160036F7
:10191000091600200916000A091500F5081500E04F
:10192000081400CC081400B8081400A4081400908F
:101930000813007D0812006B0813005808120046B7
:1019400008120034081100230811001208110001C8
:10195000081100F0071000E0071000D0071000C0C9
:10196000071000B0070F00A107100091070E0083B9
:10197000070F0074070F0065070E0057070E004998
:10198000070E003B070D002E070E0020070D001369
:10199000070D0006070D00F9060C00ED060D00E02E
:1019A000060C00D4060C00C8060C00BC060C00B0E7
:1019B000060C00A4060B0099060C008D060B008295
:1019C000060B0077060B006C060B0061060A005739
:1019D000060B004C060A0042060A0038060A002ED2
:1019E000060A0024060A001A060A00100609000763
:1019F000060A00FD050900F4050900EB050900E2EF
:101A0000050900D9050900D0050900C7050900BE70
:101A1000050900B5050800AD050800A50509009CED
:101A2000050800940508008C050800840508007C62
:101A3000050800740508006C050700650508005DD1
:101A4000050700560508004E05070047050700403A
:101A500005080038050700310507002A050700239F
:101A60000507001C050600160507000F05070008FE
:101A700005060002050700FB040600F5040700EE5A
:101A8000040600E8040600E2040700DB040600D5B3
:101A9000040600CF040600C9040600C3040600BD06
:101AA000040600B7040600B1040500AC040600A655
:101AB000040600A00405009B0406009504050090A0
:101AC0000406008A04050085040500800406007AE7
:101AD00004050075040500700405006B040500662C
:101AE000040500610405005C04050057040500526C
:101AF0000405004D04050048040500430405003EAC
:101B00000404003A04050035040500300404002CE8
:101B100004050027040400230405001E0404001A21
:101B200004040016040500110404000D0404000957
:101B30000405000404040000040400FC030400F88D
:101B4000030400F4030400F0030400EC030400E8C1
:101B5000030400E4030400E0030400DC030400D8F1
:101B6000030400D4030400D0030400CC030400C821
:101B7000030300C503030024F404D9201BC40C5C38
:101B80000E9804C4095F0265077101F405F900FBB2
:101B900004B30048048700C10369005803550003DB
:101BA000034500BE023A008402310053022A002994
:101BB00002250004022000E4011C00C8011900AF46
:101BC00001170098011400840113007101100061D5
:101BD00001100051010E0043010D0036010B002BD6
:101BE000010B0020010B00150109000C0109000385
:101BF000010800FB000800F3000800EB000700E408
:101C0000000600DE000600D8000600D2000600CC68
:101C1000000500C7000500C2000500BD000400B9B2
:101C2000000400B5000400B1000400AD000400A9E8
:101C3000000400A5000300A20003009F0004009B15
:101C40000003009800030095000200930003009039
:101C50000003008D0002008B000300880002008654
:101C600000020084000300810002007F0002007D6A
:101C70000002007B0002007900020077000100767C
:101C80000002007400020072000100710002006F87
:101C90000002006D0001006C0002006A0001006992
:101CA0000002006700010066000100650001006499
:101CB0000002006200010061000100600001005F9D
:101CC0000002005D0001005C0001005B0001005AA1
:101CD00000010059000100580001005700010056A2
:101CE00000010055000100540001005300000053A2
:101CF0000001005200010051000100500001004F9E
:101D00000001004E0000004E0001004D0001004C9B
:101D10000001004B0000004B0001004A0001004997
:101D20000001004800000048000100470001004693
:101D3000000000460001004500000045000100448D
:101D40000001004300000043000100420000004287
:101D50000001004100000041000100400001003F7F
:101D60000000003F0001003E0000003E0001003D79
:101D70000000003D0001003C0000003C0000003C71
:101D80000001003B0000003B0001003A0000003A67
:101D9000000100390000003900010038000000385F
:101DA0000000003800010037000000370001003655
:101DB000000000360000003600010035000000354C
:101DC0000000003500010034000000340000003441
:101DD0000001003300000033000000330001003236
:101DE000000000320000003200010031000000312C
:101DF0000000003100010030000000300000003021
:101E00000001002F0000002F0000002F0000002F15
:101E10000001002E0000002E0000002E0001002D09
:101E20000000002D0000002D0000002D0001002CFE
:101E30000000002C0000002C0000002C0001002BF2
:101E40000000002B0000002B0000002B0001002AE6
:101E50000000002A0000002A0000002A00010029DA
:101E600000000029000000290000002900000029CE
:101E700000010028000000280000002800000028C1
:101E800000000028000100270000002700000027B4
:101E900000000027000000270001002600000026A7
:101EA000000000260000002600000026000100259A
:101EB000000000250000002500000025000000258E
:101EC0000000002500010024000000240000002480
:101ED0000000002400000024000100230000002373
:101EE0000000002300000023000000230000002366
:101EF0000000002300010022000000220000002258
:101F00000000002200000022000000220001002149
:101F1000000000210000002100000021000000213D
:101F2000000000210000002100010020000000202E
:101F30000000002000000020000000200000002021
:101F400000000020000000200001001F0000001F12
:101F50000000001F0000001F0000001F0000001F05
:101F60000000001F0001001E0000001E0000001EF7
:101F70000000001E0000004D383420582059205A1F
:101F80002045006265640A002C2073797374656DC6
:101F90002073746F70706564212048656174657288
:101FA0005F49443A200048656174696E6720666144
:101FB000696C65640048656174696E672066616973
:101FC0006C65640048656174696E67206661696C60
:101FD00065640048656174696E67206661696C6557
:101FE0006400466C6F7700466C6F770046616E2028
:101FF00073706565640046616E207370656564008A
:1020000042656400426564004E6F7A7A6C65004EEA
:102010006F7A7A6C6500537065656400537065650E
:1020200064004D61696E005072656865617420508E
:102030004C412042656400507265686561742050AF
:102040004C4120456E640050726568656174205093
:102050004C41005072657061726500507265686530
:102060006174204142532042656400507265686586
:1020700061742041425320456E640050726568656A
:102080006174204142530050726570617265004D69
:1020900034323800507265686561742041425300E3
:1020A0005072656865617420504C4100436F6F6CDD
:1020B000646F776E004D38340044697361626C65FB
:1020C0002073746570706572730053657420686F57
:1020D0006D65206F66667365747300473238004122
:1020E00075746F20686F6D65004D6F76652061783F
:1020F0006973004D61696E004D6F76652058004D23
:102100006F76652059004D6F7665205A00457874CA
:102110007275646572004D6F766520302E316D6D7D
:10212000004D6F766520316D6D004D6F7665203105
:10213000306D6D004D6F766520617869730045786C
:10214000747275646572004D6F7665205A004D6F2C
:1021500076652059004D6F766520580020204D3857
:102160003531205A005A2D50726F6265204F6666D5
:1021700073657420286D6D293A0A002044002049B7
:102180000020204D333031205000504944207365E9
:102190007474696E67733A0A00204600204200207A
:1021A000480020204D3134352053004D6174657254
:1021B00069616C2068656174757020706172616D11
:1021C00065746572733A0A00205A00205900202075
:1021D0004D323036205800486F6D65206F6666734B
:1021E00065743A0A00204500205A00205900205802
:1021F0000020420020540020204D32303520530072
:10220000416476616E6365643A20533C6D696E5F2C
:1022100066656564726174653E20543C6D696E5FED
:1022200074726176656C5F66656564726174653E43
:1022300020423C6D696E5F7365676D656E745F7497
:10224000696D655F6D733E20583C6D61785F78798C
:102250005F6A65726B3E205A3C6D61785F7A5F6A97
:1022600065726B3E20453C6D61785F655F6A6572A3
:102270006B3E0A0020540020520020204D323034A2
:10228000205000416363656C65726174696F6E20F4
:1022900028756E6974732F7332293A20503C70721E
:1022A000696E745F616363656C3E20523C72657455
:1022B000726163745F616363656C3E20543C747249
:1022C0006176656C5F616363656C3E0A0020450062
:1022D000205A0020590020204D3230312058004D26
:1022E0006178696D756D20416363656C65726174B9
:1022F000696F6E2028756E6974732F7332293A0ADC
:1023000000204500205A0020590020204D32303353
:102310002058004D6178696D756D20666565647241
:10232000617465732028756E6974732F73293A0A76
:1023300000204500205A0020590020204D3932202D
:10234000580053746570732070657220756E6974DF
:102350003A0A0020204D3230302044300A0020203C
:102360004D3230302044002044697361626C6564F2
:102370000A0046696C616D656E74207365747469DA
:102380006E67733A002020473231203B20556E693A
:10239000747320696E206D6D0A0A007A5F6D696E34
:1023A0003A2000795F6D696E3A2000785F6D696E42
:1023B0003A20005265706F7274696E6720656E64B2
:1023C00073746F70207374617475730A007C3C3E83
:1023D0005E2B3D3F2F5B5D3B2C2A225C00457874D1
:1023E0007275646572004D6F7665205A004D6F7688
:1023F000652059004D6F76652058005072657061F8
:10240000726500526573746F7265206661696C73E2
:102410006166650046696C616D656E74004D6F7430
:10242000696F6E0054656D706572617475726500D8
:102430004D61696E00507265686561742041425358
:1024400020636F6E66005072656865617420504C41
:102450004120636F6E66005049442D44005049444A
:102460002D44005049442D49005049442D49005005
:1024700049442D50005049442D5000200820466109
:1024800063740020082046616374002008204D61B9
:1024900078002008204D6178002008204D617800E8
:1024A0002008204D696E002008204D696E0020082C
:1024B000204D696E004F6666004F6E2000417574B6
:1024C0006F74656D700046616E20737065656400A1
:1024D00046616E2073706565640042656400426504
:1024E00064004E6F7A7A6C65004E6F7A7A6C650084
:1024F000436F6E74726F6C004265640042656400E5
:102500004E6F7A7A6C65004E6F7A7A6C6500466120
:102510006E2073706565640046616E20737065653A
:10252000640054656D706572617475726500534422
:102530002063617264206F6B0A006F70656E526F6A
:102540006F74206661696C65640A00766F6C756DE6
:10255000652E696E6974206661696C65640A005352
:102560004420696E6974206661696C0A0061757443
:102570006F25692E67004D3234004D3233202573AC
:102580000057726974696E6720746F2066696C65A4
:102590003A20006F70656E206661696C65642C205E
:1025A00046696C653A20006F70656E206661696CE3
:1025B00065642C2046696C653A200046696C65208C
:1025C00073656C65637465640A002053697A653AC3
:1025D000200046696C65206F70656E65643A200066
:1025E0006F70656E206661696C65642C2046696C4D
:1025F000653A20002066696C653A20004E6F7720AE
:10260000002220706F73002220706172656E743A30
:102610002200535542524F5554494E452043414C98
:102620004C207461726765743A22004B494C4C45EA
:10263000442E2000747279696E6720746F20636184
:102640006C6C207375622D67636F64652066696CBE
:102650006573207769746820746F6F206D616E797F
:10266000206C6576656C732E204D4158206C657624
:10267000656C2069733A004572726F723A006F6B35
:1026800000627573793A2070617573656420666FB6
:102690007220696E7075740A00627573793A2070E1
:1026A000617573656420666F7220757365720A00C8
:1026B000627573793A2070726F63657373696E67C0
:1026C0000A004B494C4C45442E20004B494C4C20B1
:1026D000636175736564206279204B494C4C2062BC
:1026E0007574746F6E2F70696E0A004B494C4C45BF
:1026F000442E20004B494C4C206361757365642067
:10270000627920746F6F206D75636820696E6163F4
:10271000746976652074696D65202D206375727209
:10272000656E7420636F6D6D616E643A2000506C4D
:1027300065617365207265736574005052494E542B
:1027400045522048414C544544005072696E7465AE
:10275000722068616C7465642E206B696C6C28292A
:102760002063616C6C6564210A00656E7175657526
:1027700065696E6720220000000000000000000074
:102780000000005761726E696E673A20486F6D698C
:102790006E672042756D702044697669736F722090
:1027A0003C20310A000000A0400000A040000000D2
:1027B00040000096430000964300009643FFFFFF51
:1027C0004E6F204C696E65204E756D626572207784
:1027D00069746820636865636B73756D2C204C6148
:1027E0007374204C696E653A20004B494C4C45444B
:1027F0002E200053544F505045442E2000507269F3
:102800006E7465722073746F707065642064756592
:1028100020746F206572726F72732E204669782063
:10282000746865206572726F7220616E64207573C2
:1028300065204D39393920746F2072657374617267
:10284000742E202854656D706572617475726520F0
:1028500069732072657365742E20536574206974E2
:102860002061667465722072657374617274696E3A
:1028700067290A004E6F20436865636B73756D208E
:1028800077697468206C696E65206E756D6265721B
:102890002C204C617374204C696E653A200063688B
:1028A00065636B73756D206D69736D617463682CFE
:1028B000204C617374204C696E653A20004C696E3F
:1028C00065204E756D626572206973206E6F74208D
:1028D0004C617374204C696E65204E756D62657233
:1028E0002B312C204C617374204C696E653A2000AA
:1028F0004D313130004D3331004D3834205820599E
:10290000205A20450053442072656164206572722C
:102910006F720A00446F6E65207072696E74696E22
:10292000672066696C650A0020496E76616C69648F
:10293000206578747275646572200000009643000B
:1029400000964300009643000000000000000000D5
:10295000000000205A3A200020593A2000426564C5
:1029600020583A200020746F6F206C6F6E672065CE
:102970007874727573696F6E2070726576656E74A7
:1029800065640A0020636F6C6420657874727573E7
:10299000696F6E2070726576656E7465640A0020DA
:1029A000706F736974696F6E206F7574206F662025
:1029B00072616E67652E0A003F50726F626520007B
:1029C0004E6F206D6F76652E00486F6D6520257304
:1029D00025732573206669727374002066697273AB
:1029E000740A005A0059005800486F6D6520005362
:1029F00074616E6461726420446576696174696FA4
:102A00006E3A20002052616E67653A2000204D61C9
:102A1000783A2000204D696E3A20004D65616E3A8B
:102A2000200046696E697368656421002072616EDA
:102A300067653A2000206D61783A2000206D696E4C
:102A40003A2000207369676D613A2000206D65614E
:102A50006E3A20003A207A3A2000206F662000204B
:102A60005A00205900205800476F696E6720746F24
:102A70003A00436C6F636B776973650A00436F7547
:102A80006E7465722D0020446972656374696F6E9F
:102A90003A2000202020616E676C653A2000537454
:102AA000617274696E67207261646975733A20009F
:102AB000506F736974696F6E696E67207468652002
:102AC00070726F62652E2E2E0A003F4E756D626524
:102AD00072206F66206C65677320696E206D6F765B
:102AE000656D656E74206E6F7420706C61757369AE
:102AF000626C652028302D3135292E0A0059005886
:102B0000003F53616D706C652073697A65206E6F4C
:102B10007420706C61757369626C652028342D3582
:102B200030292E0A004D3438205A2D50726F6265BC
:102B3000205265706561746162696C6974792054B2
:102B40006573740A003F566572626F7365204C6549
:102B500076656C206E6F7420706C61757369626C41
:102B6000652028302D34292E0A0043616E6E6F7463
:102B7000206F70656E2073756264697220006563F2
:102B8000686F3A0046696C2E204469612E004669E0
:102B90006C2E204469612E004F6666004F6E200047
:102BA0004520696E206D6D3300436F6E74726F6CDB
:102BB0000043616E6E6F7420656E7465722073756C
:102BC000626469723A2000022E2E004D61696E0027
:102BD00048617264636F6465642044656661756C06
:102BE000742053657474696E6773204C6F616465FB
:102BF000640A004573746570732F6D6D00457374BE
:102C00006570732F6D6D005A73746570732F6D6DE1
:102C1000005A73746570732F6D6D0059737465700D
:102C2000732F6D6D005973746570732F6D6D00583F
:102C300073746570732F6D6D005873746570732FA6
:102C40006D6D00412D74726176656C00412D74725A
:102C50006176656C00412D72657472616374004128
:102C60002D7265747261637400416D617820450056
:102C7000416D6178204500416D6178205A00416DB9
:102C80006178205A00416D6178205900416D61786A
:102C9000205900416D6178205800416D61782058BD
:102CA000005654726176206D696E005654726176DA
:102CB000206D696E005654726176206D696E005603
:102CC0006D696E00566D696E00566D696E00566DC9
:102CD0006178204500566D6178204500566D617819
:102CE000204500566D6178205A00566D6178205A53
:102CF00000566D6178205A00566D61782059005653
:102D00006D6178205900566D6178205900566D61CB
:102D100078205800566D6178205800566D617820F3
:102D2000580056652D6A65726B0056652D6A65728E
:102D30006B0056652D6A65726B00567A2D6A657256
:102D40006B00567A2D6A65726B0056792D6A657232
:102D50006B0056792D6A65726B0056792D6A657223
:102D60006B0056782D6A65726B0056782D6A657215
:102D70006B0056782D6A65726B00416363656C0069
:102D8000416363656C005A204F6666736574005A30
:102D9000204F666673657400436F6E74726F6C00CB
:102DA00020746F6F206C6F6E672065787472757316
:102DB000696F6E2070726576656E7465640A0020B6
:102DC000636F6C6420657874727573696F6E2070C0
:102DD000726576656E7465640A0070012C0190015D
:102DE0002701B0012201C0011D01F00118011002EC
:102DF000130130020E016002090190020401C002B9
:102E0000FF000003FA004003F5008003F000D00348
:102E1000EB002004E6007004E100E004DC00400563
:102E2000D700C005D2004006CD00D006C8008007FC
:102E3000C3003008BE00F008B900C009B400B00AF1
:102E4000AF00B00BAA00D00CA500000EA000500FE0
:102E50009B00C01096005012910000148C00C01509
:102E60008700B0178200B0197D00D01B7800001ECB
:102E7000730040206E0090226900F0246400402717
:102E80005F0090295A00E02B5500102E5000203092
:102E90004B0010324600E033410090353C001037C3
:102EA000370070383200A0392D00B03A2800A03B1E
:102EB0002300603C1E00103D1900903D1400103EA0
:102EC0000F00703E0A00C03E0500003F0000403F7A
:102ED000FBFF803FF6FFC03FF1FF544845524D4194
:102EE0004C2052554E4157415900546865726D61EE
:102EF0006C2052756E61776179004572723A204D8F
:102F0000494E54454D5020424544004572723A2086
:102F10004D494E54454D50004D494E54454D50205D
:102F2000747269676765726564004572723A204D14
:102F3000415854454D5020424544004572723A2054
:102F40004D415854454D50004D415854454D502029
:102F5000747269676765726564001FFFFFFFFFFF9A
:102F6000FF600000000001FF400000000000FF8043
:102F700000000000007F83CF00000C303F87FF80FF
:102F8000000C301F867980000C000F8C30C7838CBA
:102F900030E78C30CFC7CC31F38C30DCECEC33B97C
:102FA0008C30D86C6C33198C30D06C0C33198C305D
:102FB000D86C0C33198C30DC6C0E3B198C30CF7C08
:102FC000079F198C30C77C038F1940000000000058
:102FD00002600000000000061FFFFFFFFFFFF80077
:102FE000600000000000600000E00000E000000160
:102FF000F80000000001F80003F80003F8000007E3
:10300000FE0000000007FE000FFE000F1E00001F64
:103010000F81C000381F0F803F0F803E0F80007C63
:1030200003E1C000387C03E0FC03E0F803E000F0BB
:1030300000F1C00038F000F1F000F1E000F000C055
:103040000071C00038C00071C00071C0007000C0C5
:103050000001C00038C003E1C00031C0003000C032
:103060000001C00038C00F81C00031C0003000C076
:103070000001FFFFF8C07E01FFFC31C0003000C03E
:103080000001FFFFF8C1F001FFFC31C0003000C0BB
:103090000001FFFFF8C7C001FFFC31C0003000C0D5
:1030A0000001C00038FF0001C00031C0003000C086
:1030B0000001C00038FC0001C00031C0003000C079
:1030C0000031C00038E00031C00031C0003000E005
:1030D00000F1C00038E000F1C00031C00070007C99
:1030E00003E1C000387C03E1C00031F001E0001FC3
:1030F0000F81C000381F0F81C00031FC07C00007DE
:10310000FE0000000007FE00000001CF0F000001DC
:10311000F80000000001F800000001C3FC000000FE
:103120006000000000006000000001C0F00000002E
:10313000000000000000000000000000600000002F
:10314000000000000000000000000000000000007F
:10315000000000000000000000000000000000006F
:10316000000000000000000000000E00001F03002F
:10317000000000000000000000003F80007FC3004E
:1031800000000000000000000000FFE001FBF30071
:1031900000000000000000000003E0F807E0FF006E
:1031A0000000000000000000000F803E1F8E3F0066
:1031B0000000000000000000000E001F9E3F8F0076
:1031C00000000000000000000000001F98FFE30066
:1031D00000000000000000000000007E19FFF30066
:1031E0000000000000000000000001F819FFF300DB
:1031F000000000000000000000000FE019FFF300D5
:10320000000000000000000000001F8019FFF30014
:103210000000000000000000000007E019FFF300BC
:103220000000000000000000000001FC19FFF30096
:1032300000000000000000000000003F19FFF30044
:103240000000000000000000000C000F9C7FC70081
:103250000000000000000000000F001F9F1F1F0063
:103260000000000000000000000FC07E0FC07E00C4
:1032700000000000000000000003F1F803F1F80076
:1032800000000000000000000000FFE000FFE00080
:10329000000000000000000000003F80003F8000B0
:1032A000000000000000000000000E00000E000002
:1032B000000000000000000000000000000000000E
:1032C00000000000000000000000000000000000FE
:1032D00000000000000000000000000000000000EE
:1032E00000000000000000000000000000000000DE
:104FD00000000000000000000000000000000020B1
:104FE00042403A0020403A00202F0020423A002060
:104FF0002F0020543A004D31343520533C696E6403
:1050000065783E206F7574206F662072616E6765EB
:105010002028302D31290A00205A3A0020593A0020
:1050200020436F756E7420583A0020453A00205A8C
:105030003A0020593A00583A00526573656E643A56
:1050400020005DDE26DE11241FBECFEFD1E2DEBFE1
:10505000CDBF00E00CBF14E0A0E0B2E0E8E4FBED5F
:1050600001E00BBF02C007900D92A235B107D9F73E
:1050700024E1A2E5B4E001C01D92AB36B207E1F72E
:1050800018E2C2E2D8E200E006C021970109802FB1
:10509000FE010E940DEDC132D10780E00807A9F79B
:1050A0000E94C4D90C9493ED0C9400002F923F926F
:1050B0004F925F926F927F928F929F92AF92BF9228
:1050C000CF92DF92EF92FF920F931F93CF93DF93D4
:1050D000CDB7DEB7CF58D1090FB6F894DEBF0FBEFB
:1050E000CDBF80916D0620E6829FC00111248351BF
:1050F0009B4F9093620C8093610C80911B1380FFF7
:105100001BC0EEE7FBE284918F010F5F1F4F8823E6
:1051100021F00E94C08EF801F6CF0091610C109131
:10512000620CD8018D918D01882319F00E94C08EE8
:10513000F8CF8AE00E94C08EE091610CF091620C81
:105140008081803231F43196F093620CE093610CEF
:10515000F3CF8E3469F01091610C0091620C6AE219
:1051600070E0812F902F0E945BED009721F52AC0FF
:10517000818190ED980F9A3010F08D3261F7329660
:10518000F093620CE093610CE091610CF091620C81
:10519000808180538A3010F43196F2CFE091610C17
:1051A000F091620C80818032B1F63196F093620CFE
:1051B000E093610CF3CFFC0131968291803231F0A3
:1051C0008A3221F0A12FB02F9D9102C01082F5CF1D
:1051D000FD01808111968032D9F380538A3020F00E
:1051E000EEE7FBE20C946141E12CF12C2AE02E9DCC
:1051F000B0012F9D700D11247B01B0E3EB1AF10873
:105200008191E80EF11C87FDFA94808180538A30E9
:1052100070F38F013196D8018C918032D1F31093C5
:105220005D0400935C0421E030E03093600C209337
:105230005F0C9D3409F4DAC7943511F40C94F740EF
:10524000973411F00C940F41B4E0EB16F10409F41B
:1052500087C540F4F2E0EF16F10410F50E94B2A306
:105260000C9458412AE5E216F10409F4FDC660F4F5
:105270004CE1E416F10409F4B1C55EE1E516F10470
:1052800009F42DC60C9458418BE5E816F10409F495
:10529000EFC69CE5E916F10409F4EFC60C945841F9
:1052A00080911602882311F40C94584111E0A2E079
:1052B000EA16F10409F010E00E94519A82E50E947A
:1052C0006699882309F452C10E94289A6B017C01D7
:1052D0004090BC045090BD046090BE047090BF0428
:1052E0002091C0043091C1044091C2045091C30484
:1052F0002BAF3CAF4DAF5EAF8091830C9091840C8F
:10530000A091850CB091860C23968CAF9DAFAEAF6B
:10531000BFAF23972091870C3091880C4091890C66
:1053200050918A0C2B962CAF3DAF4EAF5FAF2B97B1
:1053300020E030E0A901C701B6010E94FFE5882303
:1053400009F4F4C4A301920123966CAD7DAD8EAD3A
:105350009FAD23970E94FFE581110FC02BAD3CAD9F
:105360004DAD5EAD2B966CAD7DAD8EAD9FAD2B97EB
:105370000E94FFE5882309F4D9C420E030E0A901A8
:10538000C701B6010E94FFE5881F8827881F1813F0
:105390000BC080E090E0A0E8BFE367968CAF9DAFC4
:1053A000AEAFBFAF67970AC020E030E040E85FEBE8
:1053B00067962CAF3DAF4EAF5FAF6797A3019201E9
:1053C00023966CAD7DAD8EAD9FAD23970E9421EAF3
:1053D0002F966CAF7DAF8EAF9FAF2F972BAD3CADAF
:1053E0004DAD5EAD2B966CAD7DAD8EAD9FAD2B976B
:1053F0000E9421EA63966CAF7DAF8EAF9FAF63973B
:105400002F962CAD3DAD4EAD5FAD2F97CA01B901C2
:105410000E9464E64B015C0163962CAD3DAD4EAD40
:105420005FAD6397CA01B9010E9464E69B01AC01BC
:10543000C501B4010E9422EA0E948DEC27966CAF50
:105440007DAF8EAF9FAF279720E030E040E05FE375
:105450000E9464E64B015C01A7019601C701B601F9
:105460000E9464E66B017C01A5019401C501B401B1
:105470000E9464E69B01AC01C701B6010E9421EACB
:105480000E948DEC9B01AC0167966CAD7DAD8EAD3D
:105490009FAD67970E9464E64B015C0123962CAD9B
:1054A0003DAD4EAD5FAD2397C301B2010E9422EA2C
:1054B00020E030E040E05FE30E9464E66B017C01A5
:1054C00063966CAD7DAD8EAD9FAD6397905827967A
:1054D0002CAD3DAD4EAD5FAD27970E94FEEA9B011E
:1054E000AC01C501B4010E9464E69B01AC01C70197
:1054F000B6010E9422EAA30192010E9421EA6B01F7
:105500007C012B962CAD3DAD4EAD5FAD2B976BADB9
:105510007CAD8DAD9EAD0E9422EA20E030E040E0FF
:105520005FE30E9464E62B013C0127962CAD3DAD64
:105530004EAD5FAD27972F966CAD7DAD8EAD9FAD17
:105540002F970E94FEEA9B01AC01C501B4010E94A5
:1055500064E69B01AC01C301B2010E9422EA2BADBB
:105560003CAD4DAD5EAD0E9421EA14C089E40E94BD
:105570006699882329F00E94289A6B017C0103C058
:10558000C12CD12C76018AE40E9466998823F9F017
:105590000E94289A2B966CAF7DAF8EAF9FAF2B9752
:1055A00020E030E0A901C701B6010E94FFE58111AA
:1055B0001EC020E030E0A9012B966CAD7DAD8EAD14
:1055C0009FAD2B970E94FFE5811111C0AFC320E072
:1055D00030E0A901C701B6010E94FFE5882309F464
:1055E000A5C32B961CAE1DAE1EAE1FAE2B97D701CA
:1055F000C601B0588BAF9CAFADAFBEAF2B962CADF4
:105600003DAD4EAD5FAD2B97505823962CAF3DAFBF
:105610004EAF5FAF23979C01AD01BC01CD010E944D
:1056200064E64B015C0123962CAD3DAD4EAD5FAD04
:105630002397CA01B9010E9464E69B01AC01C50130
:10564000B4010E9422EA0E948DECA7966CAF7DAF58
:105650008EAF9FAFA7978091BC049091BD04A0919D
:10566000BE04B091BF0427968CAF9DAFAEAFBFAF65
:105670002797A7019601BC01CD010E9422EA6796F7
:105680006CAF7DAF8EAF9FAF67972091C004309114
:10569000C1044091C2045091C3042F962CAF3DAF7A
:1056A0004EAF5FAF2F972B962CAD3DAD4EAD5FAD9E
:1056B0002B972F966CAD7DAD8EAD9FAD2F970E9431
:1056C00022EA6B966CAF7DAF8EAF9FAF6B978091E8
:1056D000830C9091840CA091850CB091860C6F96F0
:1056E0008CAF9DAFAEAFBFAF6F9767962CAD3DADA2
:1056F0004EAD5FAD6797BC01CD010E9421EA6B0101
:105700007C012091870C3091880C4091890C50913C
:105710008A0CA3962CAF3DAF4EAF5FAFA3976B96AD
:105720002CAD3DAD4EAD5FAD6B97A3966CAD7DAD31
:105730008EAD9FADA3970E9421EA4B015C01809141
:10574000C4049091C504A091C604B091C704AF965B
:105750008CAF9DAFAEAFBFAFAF979C01AD01609175
:105760008B0C70918C0C80918D0C90918E0C0E9402
:1057700021EA63966CAF7DAF8EAF9FAF63972091A8
:105780008F0C3091900C4091910C5091920CAB96F3
:105790002CAF3DAF4EAF5FAFAB978091C8049091F7
:1057A000C904A091CA04B091CB04E3968CAF9DAF1D
:1057B000AEAFBFAFE397A70196016BAD7CAD8DADEA
:1057C0009EAD0E9464E62B013C01A5019401239645
:1057D0006CAD7DAD8EAD9FAD23970E9464E69B01BD
:1057E000AC01C301B2010E9422EA2B013C01A501D8
:1057F00094016BAD7CAD8DAD9EAD0E9464E64B0116
:105800005C01A701960123966CAD7DAD8EAD9FAD79
:1058100023970E9464E69B01AC01C501B4010E947C
:1058200021EAA30192010E9495EA6B017C0120E02C
:1058300030E0A9010E94FFE587FF0AC02BED3FE0A1
:1058400049EC50E4C701B6010E9422EA6B017C01D9
:10585000112351F02BED3FE049EC50E4C701B601B4
:105860000E9421EA6B017C0120E030E0A901C70120
:10587000B6010E94FFE581112AC06F962CAD3DADA7
:105880004EAD5FAD6F9727966CAD7DAD8EAD9FAD84
:1058900027970E94FFE581111AC0A3962CAD3DAD5C
:1058A0004EAD5FADA3972F966CAD7DAD8EAD9FAD28
:1058B0002F970E94FFE581110AC02BED3FE049ECD4
:1058C00050E4C701B6010E9422EA6B017C01A79651
:1058D0002CAD3DAD4EAD5FADA797C701B6010E949F
:1058E00064E69B01AC010E9464E64B015C01639697
:1058F0002CAD3DAD4EAD5FAD6397CA01B9010E94BD
:1059000064E69B01AC01C501B4010E9422EA0E9439
:105910008DEC4B015C012FE632E143E85AE30E9433
:10592000FFE587FDFFC1C501B4010E9497EB0E940E
:105930006BEB2D967FAF6EAF2D97DB01AB2B31F468
:10594000E1E0F0E02D96FFAFEEAF2D972D962EAD56
:105950003FAD2D97B90180E090E00E9403E64B0136
:105960005C019B01AC01C701B6010E94FEEA2796CB
:105970006CAF7DAF8EAF9FAF2797A5019401639663
:105980006CAD7DAD8EAD9FAD63970E94FEEAA7968C
:105990006CAF7DAF8EAF9FAFA797E3962CAD3DADBB
:1059A0004EAD5FADE397AB966CAD7DAD8EAD9FAD6B
:1059B000AB970E9421EAA50194010E94FEEAAB96F2
:1059C0006CAF7DAF8EAF9FAFAB9727962CAD3DAD43
:1059D0004EAD5FAD2797CA01B9010E9464E620E091
:1059E00030E040E05FE30E9464E69B01AC0160E0D0
:1059F00070E080E89FE30E9421EA63966CAF7DAF80
:105A00008EAF9FAF6397AF968CAD9DADAEADBFAD82
:105A1000AF9789879A87AB87BC87E3962CAD3DAD5E
:105A20004EAD5FADE3972D873E874F87588B6091D2
:105A3000190270911A02072E000C880B990B0E9414
:105A400005E620910002309101024091020250913E
:105A500003020E9464E62AE037ED43E25CE30E9421
:105A600064E66F966CAF7DAF8EAF9FAF6F970E946D
:105A7000A7509B01AC0128533F4F4F4F5F4FA39658
:105A80002CAF3DAF4EAF5FAFA3974BAC5CAC6DACF2
:105A90007EAC22242394312CD12C2D968EAD9FAD3B
:105AA0002D972816390609F429C10E94C65B0E9469
:105AB000A750DC01CB01A3962CAD3DAD4EAD5FAD43
:105AC000A397821B930BA40BB50BB7FD10C00E94CC
:105AD000A7509B01AC0128533F4F4F4F5F4FA396F8
:105AE0002CAF3DAF4EAF5FAFA3970E947D92D39492
:105AF00038E13D150CF44BC063962CAD3DAD4EAD79
:105B00005FAD639723966CAD7DAD8EAD9FAD239752
:105B10000E9464E64B015C0127962CAD3DAD4EAD75
:105B20005FAD2797B201C3010E9464E6A50194010D
:105B30000E9422EA7B018C0163962CAD3DAD4EADF7
:105B40005FAD6397B201C3010E9464E64B015C0143
:105B500027962CAD3DAD4EAD5FAD279723966CAD2E
:105B60007DAD8EAD9FAD23970E9464E69B01AC0195
:105B7000C501B4010E9421EA2B013C01C701D801F3
:105B800023968CAF9DAFAEAFBFAF239756C0B10188
:105B900080E090E00E9403E627962CAD3DAD4EAD2F
:105BA0005FAD27970E9464E64B015C010E94FBEA0F
:105BB0006B017C01C501B4010E9483EC4B015C01C7
:105BC000A70196016BAD7CAD8DAD9EAD0E9464E6E4
:105BD0002B013C01A50194012B966CAD7DAD8EADE2
:105BE0009FAD2B970E9464E69B01AC01C301B201FB
:105BF0000E9422EA2B013C01A50194016BAD7CAD12
:105C00008DAD9EAD0E9464E64B015C01A70196013B
:105C10002B966CAD7DAD8EAD9FAD2B970E9464E64B
:105C20009B01AC01C501B4010E9421EA23966CAF2F
:105C30007DAF8EAF9FAF2397D12C9201A3016796C2
:105C40006CAD7DAD8EAD9FAD67970E9422EA6983F2
:105C50007A838B839C8323962CAD3DAD4EAD5FAD97
:105C600023976B966CAD7DAD8EAD9FAD6B970E940B
:105C700022EA6D837E838F839887A7962CAD3DADF6
:105C80004EAD5FADA79769857A858B859C850E940F
:105C900022EA69877A878B879C87AB962CAD3DADCE
:105CA0004EAD5FADAB976D857E858F8598890E94DF
:105CB00022EA6D877E878F87988B809127028823C1
:105CC00021F0CE0101960E94FE8FC09056046F967F
:105CD000ECACFDAC0EAD1FAD6F979E01235F3F4F47
:105CE000AE01475F5F4FBE016B5F7F4FCE010196F4
:105CF0000E94FBBC4FEF241A340ACFCEC09056044A
:105D00006F96ECACFDAC0EAD1FAD6F972FE83CE08D
:105D10004BE85CE067E87CE083E89CE00E94FBBC29
:105D20000E94EF980E946B710C945841E7E7F6E2ED
:105D300084918F010F5F1F4F882321F00E94C08E36
:105D4000F801F6CFE9EDF1E084918F010F5F1F4F6D
:105D5000882311F40C9458410E94C08EF801F4CFAE
:105D600080E50E946699882329F00E941D9A6B01A4
:105D70007C0103C0C12CD12C760183E50E94669979
:105D8000882321F00E94C09A6B017C010E945B5D18
:105D90000E946B718091630C9091640CA091650CD2
:105DA000B091660CC80ED91EEA1EFB1E80914602F9
:105DB000811105C060E08FEE91E00E9448560E947C
:105DC000A750DC01CB018C199D09AE09BF09B7FDB5
:105DD00002C00C9458410E947D92F1CF0E945B5DFD
:105DE0000E94BB9581E080930B0288E50E94669932
:105DF000E82E89E50E946699082F8AE50E94669937
:105E0000F82EE11005C0011105C011E0182705C0EA
:105E1000011102C010E001C0182F80E1ECEBF4E0AA
:105E2000A3E8BCE001900D928A95E1F7111105C03D
:105E3000E11003C0002309F440C020E030E040EA54
:105E400050E46091730C7091740C8091750C90917A
:105E5000760C0E9422EA60938B0C70938C0C8093DA
:105E60008D0C90938E0C2091C4043091C504409108
:105E7000C6045091C7040E9448EC18165CF41982BD
:105E80001A821B821C82BE016F5F7F4F8BE89CE0F1
:105E90000E94BC96111105C0E11003C0011107C09A
:105EA0000CC080E090E00E9490901123B9F381E053
:105EB00090E00E949090111102C0FF2021F082E03A
:105EC00090E00E9490900E945B71809154048093B6
:105ED0000B020E94A1950E94C8D50C94584188E5F8
:105EE0000E946699882319F00E94289A0EC020E02B
:105EF00030E040E251E46091BC047091BD048091B7
:105F0000BE049091BF040E9422EA4B015C0189E526
:105F10000E946699882319F00E94289A0EC020E0FA
:105F200030E040E251E46091C0047091C10480917E
:105F3000C2049091C3040E9422EA2B013C012091EB
:105F4000730C3091740C4091750C5091760C2BAF02
:105F50003CAF4DAF5EAF20916B0C30916C0C40911B
:105F60006D0C50916E0CC501B4010E9421EA209184
:105F70006F0C3091700C4091710C5091720C239603
:105F80002CAF3DAF4EAF5FAF239720E030E040E253
:105F900051E40E9421EA6B017C0127E137EB41EDDE
:105FA00058EB0E9448EC87FF02C00C94584123E054
:105FB00030E046E953E4C701B6010E94FFE5181638
:105FC00014F40C94584123962CAD3DAD4EAD5FAD0D
:105FD0002397C301B2010E9421EA20E030E040E2B1
:105FE00051E40E9421EA6B017C0127E137EB41ED8E
:105FF00058EB0E9448EC87FF02C00C94584123E004
:1060000030E046E953E4C701B6010E94FFE51816E7
:1060100014F40C94584120E030E0A9016BAD7CAD44
:106020008DAD9EAD0E9422EA2BAD3CAD4DAD5EAD77
:106030000E9421EA6B017C0127E137EB41ED58EB2F
:106040000E9448EC87FF02C00C94584123E030E0E6
:1060500046E953E4C701B6010E94FFE5181614F49F
:106060000C9458410C94114110925B040C945841CB
:1060700081E080935B040C94594185E40E94669909
:10608000B82E811102C00E945B5D00EB802E02E001
:10609000902E8CEBC82E84E0D82E97E7E92E9CE05A
:1060A000F92E00E010E0A12CD4018D914D010E9449
:1060B0006699882309F44EC0F6012081318142811E
:1060C0005381C457DF4F2883CC58D040C357DF4F8C
:1060D0003883CD58D040C257DF4F4883CE58D04088
:1060E000C157DF4F5883CF58D0400E94289AD6011D
:1060F0006D937D938D939C931397C457DF4F2881A5
:10610000CC58D040C357DF4F3881CD58D040C2570C
:10611000DF4F4881CE58D040C157DF4F5881CF580C
:10612000D04003301105B1F00E9421EA9B01AC017F
:10613000F70160817181828193810E9422EAD701F7
:106140006D937D938D939C931397C8010E94129930
:10615000AA24A3940F5F1F4FB4E0CB0ED11CE4E040
:10616000EE0EF11C0430110509F09ECFAA2019F0A3
:106170000E945B7137C0BB20A9F1C090C804D090C9
:10618000C904E090CA04F090CB042091C912309168
:10619000CA124091CB125091CC12C701B6010E9495
:1061A00064E60E9453EC6093F90F7093FA0F8093AA
:1061B000FB0F9093FC0FC701B6010E9466EB2FB74F
:1061C000F89460939D0B70939E0B80939F0B90931C
:1061D000A00B2FBF1092E90F1092EA0F1092EB0F55
:1061E0001092EC0F0E94C8D50C945841F1E7EF16BD
:1061F000F10409F450C608F0D7C030E3E316F10407
:1062000009F433C508F068C058E1E516F10409F453
:1062100095C2B0F592E1E916F10409F42EC778F4BD
:10622000B2E0EB16F10408F4C2C1E1E1EE16F104AC
:1062300011F00C9458410E94A1A30C945841F5E12F
:10624000EF16F10409F470C248F434E1E316F104E6
:1062500011F00C945841EFE4F2E023C246E1E41659
:10626000F10409F465C257E1E516F10411F00C944C
:10627000584140E061E0C8010E94E6860C94584114
:106280008CE1E816F10409F4AEC268F4AAE1EA165A
:10629000F10409F45EC208F06AC210922D100E9447
:1062A000CC8B0C945841EFE1EE16F10409F4EFC3E6
:1062B00038F42EE1E216F10409F49CC20C94584122
:1062C00030E2E316F10409F498C34AE2E416F1045B
:1062D00009F483C40C9458415CE5E516F10409F413
:1062E0000EC768F591E5E916F10409F4A6C6A0F415
:1062F000BCE4EB16F10409F4BCC4EDE4EE16F104C1
:1063000009F4BBC4FBE4EF16F10411F00C945841FE
:106310000E948C8B0C94584123E5E216F10409F499
:10632000A7C608F4A1C644E5E416F10409F4A5C61D
:1063300055E5E516F10409F4CFC60C9458418CE6F6
:10634000E816F10409F4A3C5C8F4A9E6EA16F104B5
:1063500009F4E4C538F4E8E6EE16F10409F491C452
:106360000C945841FAE6EF16F10409F42EC62BE618
:10637000E216F10409F44FC60C9458413EE6E316C8
:10638000F10409F4CFC408F4E6C55FE6E516F104AC
:1063900009F4DBC480E7E816F10411F00C945841CD
:1063A00085E493E00E9415929DEDE916F10411F445
:1063B0000C942D3B08F065C0BEEBEB16F10409F41C
:1063C000E8C578F5F7E7EF16F10409F435C798F456
:1063D00033E7E316F10409F421C708F419C755E7B8
:1063E000E516F10411F00C94584160E0C8010E94D8
:1063F0005D560C94584189E7E816F10409F427C763
:1064000008F41EC7ACE8EA16F10409F470C5B1E956
:10641000EB16F10411F00C9458410E9487D60C94AD
:106420005841ECECEE16F10409F456C7A0F429EC3F
:10643000E216F10409F411C73BECE316F10409F488
:106440002EC748ECE416F10411F00C9458410E9458
:106450007BD50C9458415EECE516F10411F40C94D4
:10646000413A08F4A3C793EDE916F10411F40C9432
:10647000883AACEDEA16F10411F40C94203B0C942C
:106480005841B2E9EB16B1E0FB0611F40C94653FFC
:10649000F0F5FEE2EF16F1E0FF0611F40C94373C44
:1064A00090F43CE2E31631E0F30611F40C94723BF5
:1064B00010F00C94983B52EEE516F10411F40C9494
:1064C000463B0C94584183E6E81681E0F80611F447
:1064D0000C94CE4048F4AFE2EA16A1E0FA0611F4BB
:1064E0000C94AE3C0C945841B0E9EB16B1E0FB06BD
:1064F00011F40C94623FE1E9EE16E1E0FE0611F0C2
:106500000C94584181E00E942B970C945841F6EF6F
:10651000EF16F1E0FF0611F40C94894040F53CEAD7
:10652000E31631E0F30611F40C94693F58F45AE98C
:10653000E51651E0F50611F00C9458410E9444D53F
:106540000C94584184EFE81681E0F80611F40C949D
:10655000704095EFE91691E0F90611F00C9458415E
:106560000E9442B280E00E9487720C945841A3E5D9
:10657000EA16A3E0FA0611F40C94984048F4E7EF09
:10658000EE16E1E0FE0611F40C948C400C94584198
:10659000F0EAEF16F3E0FF0609F475C227EEE21603
:1065A00023E0F20611F40C94E7400C94584180E586
:1065B0000E946699882361F00E941D9A6B017C01FC
:1065C000BB24B394672B682B692B31F4B12C04C026
:1065D000B12CC12CD12C760183E50E9466998823C9
:1065E00099F00E94C09A6B017C01B1100FC0672B1B
:1065F000682B692B59F4D8018C91882339F061E01C
:10660000C8010E945D5607C0BB20A9F360E08DE27F
:1066100092E00E94485683E090E09093600C809353
:106620005F0C81E080939E060E945B5D0E946B710F
:10663000C114D104E104F104E9F08091630C90915C
:10664000640CA091650CB091660CC80ED91EEA1EB0
:10665000FB1E0E94A750DC01CB018C199D09AE09DD
:10666000BF09B7FF1AC080919E068823B1F00E942F
:106670007D92EFCF80919E06882319F00E947D9233
:10668000F9CF80912D1060E0882319F08EE192E01F
:1066900002C08AE092E00E94485610929E060C9436
:1066A000584184918F010F5F1F4F882321F00E9472
:1066B000C08EF801F6CF1092B3121092B21240E0E1
:1066C00050E0BA018EE590E10E948E788BE1EEE514
:1066D000F0E1DE01159601900D928A95E1F7809127
:1066E0005C1090915D109C838B838EE293E09A8383
:1066F000898340E050E0BE016F5F7F4F8FEE93E0F3
:106700000E94E0A8CE0101960E94E3B3E0E4F2E02B
:1067100084918F010F5F1F4F882311F40C9458410F
:106720000E94C08EF801F4CF0E94FB890C9458415E
:1067300010922D1010922E100C94584180912E1012
:10674000882319F081E080932D100E948C8B0C948B
:10675000584180912E10882311F40C94584183E500
:106760000E94669981110C947E410C94584180914D
:106770002E10882351F1E0E6F2E084918F010F5F43
:106780001F4F882321F00E94C08EF801F6CF609140
:10679000A9127091AA128091AB129091AC124AE0AA
:1067A0000E94C78E8FE20E94C08E6091A5127091E8
:1067B000A6128091A7129091A8124AE00E94C78E5B
:1067C0008AE00E94C08E0C945841E2E7F2E0849186
:1067D0008F010F5F1F4F882311F40C9458410E94C2
:1067E000C08EF801F4CF40E060E0C8010E94E68668
:1067F0000C94584180912E10882311F40C94584128
:1068000088EF91E10E945C7888EF91E10E94A57E7B
:1068100010922C1010922B10E0905C04F0905D040C
:1068200080912E10882311F40C9458410E949C866C
:10683000FE0131966F01CF010E94D3B38AE590E14A
:1068400090937A1080937910D7018C918F3209F050
:1068500060C06FE270E0C7010E945BED8C010F5FCA
:106860001F4F09F45CC06FE270E0C8010E945BED4D
:106870005C01009709F454C00817190708F050C0CC
:106880004C01801A910AA401B801CE0180960E94A1
:1068900084EDE0E2F0E0EC0FFD1FE80DF91D108241
:1068A0008E01005E1F4FF80181918F01882319F03E
:1068B0000E94C08EF8CF8AE00E94C08E609179104D
:1068C00070917A106115710511F06C5F7F4F21E0B6
:1068D000AE01405E5F4FCE0105960E94AD7E8111F4
:1068E00012C0BE01605E7F4F89EA92E00E9444764A
:1068F0008EE20E94C08E8AE00E94C08EC6010E9475
:10690000E3B30C945841D0927A10C092791085016B
:10691000A6CF8BE790E190937A108093791087014E
:106920006091791070917A106115710511F06C5FAA
:106930007F4F18A21BA222E0A801CE0180960E94E0
:10694000AD7E811102C0F12C14C0CE0180960E9450
:106950004EA88823C1F361E0CE0180960E9475D1D4
:10696000009789F325EEDC012C931BA20E946C7624
:10697000F82ECE0180960E94DDB3FF2009F1E3E8F6
:10698000F2E084917F01BFEFEB1AFB0A882321F02C
:106990000E94C08EF701F5CFF80181918F01882305
:1069A00019F00E94C08EF8CF8AE00E94C08E10922B
:1069B000A9121092AA121092AB121092AC1218C027
:1069C000E1E9F2E084917F012FEFE21AF20A8823D5
:1069D00021F00E94C08EF701F5CFD8018D918D0175
:1069E000882319F00E94C08EF8CF8EE20E94C08EDC
:1069F000C6010E94E3B30C94584180912D1081117F
:106A00000E945B5D00915C0410915D0461E270E0A6
:106A1000C8010E945BED009719F08C010F5F1F4FBA
:106A200080E50E946699882349F0FF24F3948091C1
:106A30005204909153048017910708F0F12C809133
:106A40002E10882311F40C9458414F2D61E0C80199
:106A50000E94E68683E50E946699882349F080912A
:106A60005204909153048017910710F40C948F41B5
:106A700080912E10882319F081E080932D10F11061
:106A80000C94584162CE0E9496A30C9458410E94E7
:106A9000F9A71CE3C12ED12CE12CF12CA701960102
:106AA0000E94C4E9762E672ECA01B901A70196019A
:106AB0000E94C4E96B017C01CA01B90128E130E000
:106AC00040E050E00E94C4E94B015C01C9016DE661
:106AD00071E00E94E6EC8E010F5F1F4F611571059A
:106AE00099F06F927F92DF92CF929F928F929F93B5
:106AF0008F937F936F9385EE92E09F938F931F9375
:106B00000F930E9498E512C00097B1F06F927F92A8
:106B1000DF92CF929F928F929F938F9385ED92E019
:106B20009F938F931F930F930E9498E50FB6F8944D
:106B3000DEBF0FBECDBF36C081149104A104B104E5
:106B400079F06F927F92DF92CF929F928F9289EC31
:106B500092E09F938F931F930F930E9498E5E6CF47
:106B6000C114D104E104F10469F06F927F92DF92C5
:106B7000CF9281EC92E09F938F931F930F930E948B
:106B800098E5D4CF6F927F928DEB92E09F938F9395
:106B90001F930F930E9498E50F900F900F900F9006
:106BA0000F900F9060E0C8010E945D56EEE7FBE297
:106BB00084917F019FEFE91AF90A882321F00E944E
:106BC000C08EF701F5CFB80189EF92E00E944476BC
:106BD0008AE00E94C08E0C94584183E50E94669919
:106BE000882311F40C9458410E94109A7C018F3F25
:106BF000910519F010F00C94584180E50E946699B7
:106C0000882339F00E94109A8C0197FF04C00C94DD
:106C100058410DE010E0D02EE4EBF2E0C8019927D6
:106C2000219131912817390731F0B3E0E430FB07A7
:106C3000B9F70C94A141E7E7F6E284918F010F5F69
:106C40001F4F882321F00E94C08EF801F6CFE6E0A6
:106C5000F3E084918F010F5F1F4F882311F40C9490
:106C600058410E94C08EF801F4CF0E94AF9D0C9451
:106C700058410E94CC8B0C9458410E94E0A70C9480
:106C8000584188E690E00E94A89981110C945841DF
:106C900080911B1383FF02C00C94584183E50E942E
:106CA00066998823D9F10E94109A9093890680935F
:106CB000880680E00E9413CE0E94109A86359105C6
:106CC0003CF40E94E0A760E08CE193E00E9448560B
:106CD0000E94109A8C0160915F0470916004809111
:106CE0006104909162040E9466EB60177107B4F42E
:106CF00084E893E09F938F938091550490E00196F0
:106D00009F938F9385E193E09F938F931F920E94AF
:106D1000718B0FB6F894DEBF0FBECDBF0E94F6E0B8
:106D20000C9458418EE40E946699882311F40C94C7
:106D300058410E9453DE60936114709362148093F3
:106D40006314909364140C94584183E50E946699EF
:106D5000882319F00E94799901C080E080931B1369
:106D6000EEE7FBE284918F010F5F1F4F882321F034
:106D70000E94C08EF801F6CFEEE3F3E084918F011C
:106D80000F5F1F4F882321F00E94C08EF801F6CFBD
:106D900080911B138823A1F1B0E3CB2EB3E0DB2E4F
:106DA000E12CF12C20E080911B1390E00E2C02C00E
:106DB000959587950A94E2F780FF17C0BB24B3949A
:106DC000B20E222319F08CE20E94C08EF6012591AA
:106DD0003491F901849189010F5F1F4F882321F0BD
:106DE0000E94C08E9801F5CF2B2DFFEFEF1AFF0AFE
:106DF00032E0C30ED11C45E0E416F104A1F642C016
:106E0000EAE3F3E084918F010F5F1F4F8823D1F1F4
:106E10000E94C08EF801F6CF8AE50E946699882309
:106E200011F40C94C0400E94289A6B017C0120E070
:106E300030E040EA51EC0E9448EC87FF02C00C941D
:106E4000B24020E030E040EA51E4C701B6010E94C0
:106E5000FFE5181614F40C94B240C0921113D092AE
:106E60001213E0921313F0921413C0928D02D09279
:106E70008E02E0928F02F092900242E0C701B601CA
:106E80000E94478F8AE00E94C08E0C945841109255
:106E900004020C94584183E50E946699882369F0A6
:106EA0000E947999809341028D3310F40C945841DB
:106EB0008CE3809341020C945841EEE7FBE284910D
:106EC0008F010F5F1F4F882321F00E94C08EF801B1
:106ED000F6CF4091410250E060E070E08EE493E034
:106EE0000E947E648AE00E94C08E0C94584180917A
:106EF0001B1383FF02C00C94584183E50E946699DE
:106F0000882311F40C9458410E94109A90938D0696
:106F100080938C060E94E0CD0C94584189E690E065
:106F20000E94A899811111C0E5E5F3E084918F01D9
:106F30000F5F1F4F882321F00E94C08EF801F6CF0B
:106F40000E94FCD68AE00E94C08E1092600C1092C3
:106F50005F0C0C94AA468DE690E00E94A8998111DE
:106F60000C94584180911B1383FF02C00C9458412C
:106F700083E50E94669928968FAF289781110C941B
:106F8000B64182E50E94669981110C94B6410C9439
:106F9000584180911B1383FF02C00C94584160E05C
:106FA00089E993E00E94485683E50E9466992896F5
:106FB0008FAF289781110C94594382E50E946699FE
:106FC00081110C9459430C94584183E50E946699B1
:106FD000882321F00E9447DE8C0102C00FEF10E0F1
:106FE00080E50E946699882319F00E9447DE02C05E
:106FF00080E090E098010F3F110519F010F02FEF9D
:1070000030E0892B11F00C94584130938B0620937B
:107010008A060C94584180E50E946699811106C049
:1070200010928B0610928A060C9458410E9447DEFB
:10703000892B11F00C945841F3CF0E9446CE0E9448
:107040005B5D0E94049210928B0610928A0668EE95
:1070500073E080E090E00E948E5560E086EA93E065
:107060000E9448560C94584110925A040C9458416E
:1070700081E080935A040C94594183E50E946699FB
:10708000882361F00E94C09A609342027093430289
:1070900080934402909345020C94584188E50E94E5
:1070A000669981110C94CA4489E50E946699811100
:1070B0000C94CA448AE50E94669981110C94CA44D2
:1070C00085E40E94669981110C94CA440E945B5D1C
:1070D0000E9404920C94584183E50E94669988238B
:1070E00011F40C9458410E94C09A6093670C7093FD
:1070F000680C8093690C90936A0C0C94584150EB87
:10710000C52E52E0D52E6DEBE62E62E1F62E10E094
:10711000D6018D916D010E946699882309F46DC096
:10712000133009F063C00E94289A4B015C0120E0F3
:1071300030E040EA51E40E94FFE587FF4EC0A50120
:1071400094016091C9127091CA128091CB129091F2
:10715000CC120E94FEEA2B013C019B01AC01609124
:10716000091370910A1380910B1390910C130E94D4
:1071700064E66093091370930A1380930B13909342
:107180000C13A30192016091F9127091FA1280918F
:10719000FB129091FC120E9464E66093F9127093C6
:1071A000FA128093FB129093FC1260915D1470911F
:1071B0005E1480915F14909160140E9403E6A30115
:1071C00092010E9464E60E946BEB60935D147093E1
:1071D0005E1480935F14909360148092C912909211
:1071E000CA12A092CB12B092CC1207C00E94289A69
:1071F000F70160837183828393831F5FF4E0EF0E56
:10720000F11C143009F084CF0E941AD50C94584117
:107210000E945B5D0E94C8D50C945841E8EBF3E0F6
:1072200084918F010F5F1F4F882311F40C945841F4
:107230000E94C08EF801F4CF0E9425720C94584130
:1072400081E080930B02809354040C945941109276
:107250000B02109254040C94584135EDE32E32E1A8
:10726000F32E00EB12E044E0D42ED00ED8018D9125
:107270008D010E946699882349F00E94289A0E94F5
:107280006BEBF7016083718382839383F4E0EF0EED
:10729000F11CD012EBCF0E94EDD30C9458419DEE1F
:1072A000E92E92E1F92E00EB12E024E0D22ED00E6E
:1072B000D8018D918D010E946699882339F00E9432
:1072C000289AF7016083718382839383F4E0EF0E41
:1072D000F11CD012EDCFECC783E50E94669988239C
:1072E000D9F00E94289AAB01BC0140930D13509332
:1072F0000E1360930F13709310134093CD1250939D
:10730000CE126093CF127093D01280EF94E00E945F
:10731000B8648AE00E94C08E80E50E946699882346
:1073200099F00E94289AAB01BC0140930D13509331
:107330000E1360930F137093101383ED94E00E946B
:10734000B8648AE00E94C08E82E50E946699882314
:1073500099F00E94289AAB01BC014093D11250933E
:10736000D2126093D3127093D41284EB94E00E94F3
:10737000B8648AE00E94C08E84E50E9466998823E2
:1073800009F496C70E94289AAB01BC014093CD1224
:107390005093CE126093CF127093D01286E994E08E
:1073A0000E94B8648AE00E94C08E82C783E50E9472
:1073B0006699882351F00E94289A6093E91270938D
:1073C000EA128093EB129093EC1284E50E94669986
:1073D000882351F00E94289A6093E5127093E61278
:1073E0008093E7129093E81282E40E9466998823C2
:1073F00051F00E941D9A6093171370931813809395
:10740000191390931A1388E50E946699882351F006
:107410000E94289A6093FD127093FE128093FF12CF
:107420009093001389E50E946699882351F00E9489
:10743000289A60930113709302138093031390931F
:1074400004138AE50E946699882351F00E94289AC5
:10745000609305137093061380930713909308139A
:1074600085E40E946699882309F422C70E94289A1D
:107470006093091370930A1380930B1390930C136A
:1074800017C710EBA12E12E0B12E0CEBC02E04E0BA
:10749000D02E80EBE82E84E0F82E00E010E0D5013D
:1074A0008D915D010E946699882311F10E94289AAE
:1074B0002B013C01F70120813181428153810E94DF
:1074C00021EA9B01AC01D6016D917D918D919C913A
:1074D0000E9422EAF6016083718382839383D7013D
:1074E0004D925D926D927C921397C8010E94129901
:1074F0000F5F1F4FB4E0CB0ED11CE4E0EE0EF11C89
:107500000330110561F60E945B710E94C8D5D0C698
:10751000EEE7FBE284918F010F5F1F4F882321F07C
:107520000E94C08EF801F6CF83E50E9466998823F9
:1075300021F00E94E59980932702E0E4F5E0849130
:107540008F010F5F1F4F882321F00E94C08EF8012A
:10755000F6CF80912702811103C0ECE3F5E002C071
:10756000E8E3F5E084918F010F5F1F4F882321F03E
:107570000E94C08EF801F6CFE0E3F5E084918F0120
:107580000F5F1F4F882321F00E94C08EF801F6CFB5
:107590004091F10B5091F20B6091F30B7091F40B51
:1075A0008EE295E00E94B8644091F50B5091F60B85
:1075B0006091F70B7091F80B8BE295E00E94B86434
:1075C0004091F90B5091FA0B6091FB0B7091FC0B01
:1075D00088E295E00E94B864E0E2F5E084918F01D2
:1075E0000F5F1F4F882321F00E94C08EF801F6CF55
:1075F00040911B0250911C0260911D0270911E026D
:107600008EE195E00E94B86440911F0250912002E3
:1076100060912102709122028BE195E00E94B86492
:10762000409123025091240260912502709126021C
:1076300088E195E00E94B8648AE00E94C08E38C656
:1076400083E50E946699882309F432C60E94109A45
:1076500090931A02809319022BC68DED90E00E9440
:10766000A899811125C683E50E946699882309F4AB
:107670001FC60091550410E00E94109A000F111FC0
:10768000F801E95EFD4F9183808312C680E50E9478
:107690006699882309F40CC60E94109A8C0183E530
:1076A0000E946699882321F00E94109A7C0103C0F1
:1076B000EE24EA94FE2CC7010196039708F0F8C562
:1076C00017FDF6C5E4EBF2E0C8019927219131914D
:1076D0002817390709F4ECC523E0E430F207B1F7C5
:1076E0000C94824683E50E946699882319F00E94D3
:1076F00047DE02C084E091E099A388A380E50E9460
:107700006699882349F00E9447DE893833E1930760
:1077100028F088E893E102C088EE93E09A83898399
:10772000BE01605E7F4FCE0101960E943D8BC0C5B9
:1077300085E40E946699811110C080E50E946699D7
:10774000882399F00E94289A609328027093290256
:1077500080932A0290932B0208C00E94109A181658
:1077600019065CF7E7E7F6E271C089E40E946699C2
:10777000882381F00E94289A2CEA35EC47E25EE3E8
:107780000E9464E66093300270933102809332026B
:107790009093330284E40E946699882381F00E94CA
:1077A000289A2CEA35EC47E25EE30E94FEEA6093F9
:1077B0002C0270932D0280932E0290932F02EEE7FD
:1077C000FBE284918F010F5F1F4F882321F00E94FD
:1077D000C08EF801F6CF40912802509129026091A5
:1077E0002A0270912B0288E595E00E94B8642CEA89
:1077F00035EC47E25EE36091300270913102809196
:107800003202909133020E94FEEAAB01BC0184E592
:1078100095E00E949B642CEA35EC47E25EE36091C0
:107820002C0270912D0280912E0290912F020E94C5
:1078300064E6AB01BC0180E595E00E949B648AE0B0
:107840000E94C08E35C50E94C08EF80184918F01C0
:107850000F5F1F4F8111F7CF0FE813E0D8018D9113
:107860008D01882309F40ECB0E94C08EF7CF83E5EB
:107870000E946699082F8823D1F00E94109ABC01BB
:10788000990F880B990B0E9405E660939102709303
:107890009202809393029093940211E020E030E0F2
:1078A000A9010E94FFE5811110E01093161380E5F5
:1078B0000E946699182F8823A9F020E030E0A901E2
:1078C0006091910270919202809193029091940242
:1078D0000E94FFE5882319F00E94E599182F109364
:1078E0001613E6C40111E4C4EEE7FBE284918F01B4
:1078F0000F5F1F4F882321F00E94C08EF801F6CF42
:1079000080911613811103C060E873E002C062EF3A
:1079100073E081E795E00E94447620E030E040E0AB
:107920005FE3609191027091920280919302909135
:1079300094020E9422EA0E9466EB80E695E00E9493
:107940002B76ECE5F5E084918F010F5F1F4F8823C4
:1079500009F4AEC40E94C08EF801F5CF85E40E9400
:107960006699882321F00E94109A8C0102C000E0E1
:1079700010E083E40E946699882349F00E94109ADF
:10798000CA57DF4F99838883C658D04008C0E5E0C6
:10799000F0E0CA57DF4FF983E883C658D04085E549
:1079A0000E946699ED968FAFED97882329F00E948B
:1079B000E599ED968FAFED9783E50E946699882350
:1079C00019F00E94109A04C017FD08C086E990E0E3
:1079D0000115110529F41092550402C086E490E0C7
:1079E0001092600C10925F0CBC01990F880B990BE0
:1079F0000E9405E624966FAF24972C967FAF2C97B4
:107A000060968FAF609764969FAF64970E94A7506F
:107A10004B015C01012B19F400EA13E00EC003EBEB
:107A200013E0D8018D918D01882319F00E94C08E3A
:107A3000F8CF8AE00E94C08E3BC4F80181918F018B
:107A4000882319F00E94C08EF8CF8AE00E94C08E71
:107A50000E9446CE8FE780932F1381E0809304022B
:107A6000C258DF4F88829982AA82BB82CE57D0400B
:107A7000C857DF4F88829982AA82BB82C858D040FB
:107A800068961FAE6897F0E46C96FFAF6C972CE198
:107A9000A0962FAFA09736E4AC963FAFAC97E09698
:107AA0001FAEE097A4961FAEA497A8961FAEA89706
:107AB000E4961FAEE497EC961CAE1DAE1EAE1FAE54
:107AC000EC97E8961CAE1DAE1EAE1FAEE897C12C1B
:107AD000D12C7601FFE74F2E512C612C712C8FE7B2
:107AE00090E0A0E0B0E023968CAF9DAFAEAFBFAF0B
:107AF0002397CE57DF4F188219821A821B82C258F1
:107B0000D04091E0EE969FAFEE9729961FAE1EAE45
:107B10002997212C312C00E010E080910402882369
:107B200009F4C9C10E94A7506BAF7CAF8DAF9EAF67
:107B300080912D13882309F4CBC00E946DCE209034
:107B40005F0430906004009161041091620491011F
:107B5000A801E0966FADE097A4967FADA497A89694
:107B60008FADA897E4969FADE4970E94FFE587FF4D
:107B70000CC0E0962FAEE097A4963FAEA497A896CF
:107B80000FAFA897E4961FAFE4979101A8016896FC
:107B90006FAD68976C967FAD6C97A0968FADA097F0
:107BA000AC969FADAC970E9448EC181664F46896AA
:107BB0002FAE68976C963FAE6C97A0960FAFA097CC
:107BC000AC961FAFAC97EE96AFADEE9724962FAD67
:107BD00024972C963FAD2C9760964FAD6097649696
:107BE0005FAD6497B101C801AA2309F455C00E9492
:107BF00048EC18160CF06CC04BAD5CAD6DAD7EADB5
:107C0000481959096A097B09DB01CA01885893415F
:107C1000A109B109B7FD5CC023968CAD9DADAEAD99
:107C2000BFAD239784199509A609B709B595A795FE
:107C30009795879580932F13CE57DF4F48835983AD
:107C40006A837B83C258D0402496BFAD2497E096C8
:107C5000BFAFE0972C96EFAD2C97A496EFAFA4970B
:107C60006096FFAD6097A896FFAFA89764962FAD7A
:107C70006497E4962FAFE4978BAD9CADADADBEADF0
:107C8000C258DF4F88839983AA83BB83CE57D040E5
:107C9000EE961FAEEE971CC00E94FFE587FF18C04E
:107CA0008BAD9CADADADBEADC258DF4F28813981E3
:107CB0004A815B81CE57D040821B930BA40BB50B3E
:107CC000AC01BD01485853416109710977FF8BC66A
:107CD00020E030E040EA51E424966FAD24972C96E2
:107CE0007FAD2C9760968FAD609764969FAD64973B
:107CF0000E9422EA9B01AC01B101C8010E9448EC3C
:107D000018166CF4EEE3F6E084918F010F5F1F4FBD
:107D1000882309F4CDC20E94C08EF801F5CF80E31C
:107D200098EFAFEFBFEFC857DF4F288139814A8105
:107D30005B81C858D040821B930BA40BB50B2BADB5
:107D40003CAD4DAD5EAD820F931FA41FB51FB7FDB7
:107D500011C00E94FCD68AE00E94C08E8BAD9CAD03
:107D6000ADADBEADC857DF4F88839983AA83BB836F
:107D7000C858D0408BAD9CADADADBEAD880F991F3E
:107D8000AA1FBB1FC258DF4F288139814A815B81FE
:107D9000CE57D040821B930BA40BB50B88199909C1
:107DA000AA09BB0981389F44A241B10568F0E0E20D
:107DB000F6E084918F010F5F1F4F882309F478C28A
:107DC0000E94C08EF801F5CF29964EAD5FAD299780
:107DD000CA57DF4F88819981C658D04084179507CC
:107DE0000CF066C0E3ECF5E084918F010F5F1F4F4C
:107DF000882321F00E94C08EF801F6CFB701A601BA
:107E00008EEA95E00E94B8648AE00E94C08EE896EF
:107E10004CAD5DAD6EAD7FADE89789E995E00E9410
:107E2000B8648AE00E94C08EEC964CAD5DAD6EAD3C
:107E30007FADEC9784E895E00E94B8648AE00E94E8
:107E4000C08EED969FADED97992309F431C2C09293
:107E50002802D0922902E0922A02F0922B022CEA08
:107E600035EC47E25EE3E8966CAD7DAD8EAD9FAD3F
:107E7000E8970E9464E66093300270933102809329
:107E80003202909333022CEA35EC47E25EE3EC9643
:107E90006CAD7DAD8EAD9FADEC970E94FEEA609318
:107EA0002C0270932D0280932E0290932F0200C219
:107EB0000E946E5632CE809104028111F9C10E9457
:107EC00046CEF6C10E945B5DF3C180E00E942B9715
:107ED000EFC1A0EBB4E0BCAFABAF8CEB282E84E0DD
:107EE000382EE7E6F4E02196FFAFEEAF219700E0F1
:107EF00010E021962EAD3FAD2197275634402996AC
:107F00003FAF2EAF29972196AEADBFAD21978D9192
:107F10002196BFAFAEAF2197882309F4ACC0F8011A
:107F2000E55EFD4F2081318142815381F801EF50A0
:107F3000F44F60817181828193810E9422EA20E066
:107F400030E040E05FE30E9464E69B01AC01F10198
:107F500060817181828193810E9448EC181634F40B
:107F6000C8018958984D0E94657103C060E070E0B7
:107F7000CB01D1018D909D90AD90BC90F801E55959
:107F8000F34F20813181428153810E9422EA9B017B
:107F9000AC01C501B4010E9421EA6B017C0120E023
:107FA00030E040EA51EC0E9448EC87FD35C020E00B
:107FB00030E040EA51E4C701B6010E94FFE518161F
:107FC0005CF1EBADFCAD4080518062807380A70115
:107FD0009601C301B2010E9421EA6B017C01A30159
:107FE00092010E9421EA9B01AC01C501B4010E94EB
:107FF00022EAD1016D937D938D939C931397EBAD02
:10800000FCADC082D182E282F38229968EAD9FAD13
:1080100029970E9412992FC0E7E7F6E284918F0119
:108020000F5F1F4F882321F00E94C08EF801F6CF0A
:10803000E0EDF6E084918F010F5F1F4F882321F060
:108040000E94C08EF801F6CF61E082EC96E00E94BB
:1080500048560E94244C88E290E09A83898388ECF9
:1080600090E099A388A3BE016F5F7F4FCE018096F9
:108070000E943D8B1DC12BAD3CAD2C5F3F4F3CAFF3
:108080002BAF0C5F1F4F34E0230E311C0C30110559
:1080900009F02FCF0E945B710E94C8D560E082EB8F
:1080A00096E00E94485683E992E099A388A304E6EB
:1080B00010E01A830983BE01605E7F4FCE010196F6
:1080C0000E943D8B8AEB92E099A388A31A830983CF
:1080D000BE01605E7F4FCE0101960E943D8BE8C0DD
:1080E000E7E7F6E284918F010F5F1F4F882321F0AD
:1080F0000E94C08EF801F6CFEEEEF6E084918F017B
:108100000F5F1F4F882309F4D3C00E94C08EF8016F
:10811000F5CF0E9442B2CCC083E50E9466998823C5
:1081200021F00E94E59991E089270E948772C0C0E2
:10813000EEE7FBE284918F010F5F1F4F882321F050
:108140000E94C08EF801F6CFE9E1F7E084918F013B
:108150000F5F1F4F882311F40C940C370E94C08EC0
:10816000F801F4CFE2E0F7E084918F010F5F1F4F39
:10817000882311F40C9442370E94C08EF801F4CF8A
:1081800040911113509112136091131370911413B5
:108190008FEF96E00E94B8640C944237E7E7F6E26E
:1081A00084918F010F5F1F4F882321F00E94C08EA2
:1081B000F801F6CFE3E2F7E084918F010F5F1F4FE4
:1081C000882309F475C00E94C08EF801F5CF81E0C4
:1081D000809316021092500C83E50E9466998823C2
:1081E00009F48DC50E94E599811162C088C5E092AD
:1081F0005604EEE7FBE284918F010F5F1F4F882347
:1082000021F00E94C08EF801F6CFB701772782E3F4
:1082100097E00E942B768AE00E94C08E49C080E0E1
:1082200048C00E94BB9583E50E946699882309F4A3
:1082300063C00E94E599EE24E394F12C082FA3017A
:108240009201C501B4010E9474976B017C012CEA74
:1082500035EC47E257E3C501B4010E9422EAAB01C5
:10826000BC0182E092E00E949B642CEA35EC47E27C
:1082700057E3C301B2010E9422EAAB01BC018DEFBA
:1082800091E00E949B642CEA35EC47E257E3C7017A
:10829000B6010E9422EAAB01BC0188EF91E00E9486
:1082A0009B648AE00E94C08E0E94A1950E94C8D55E
:1082B00081E01092600C10925F0C81111AC00C9436
:1082C000F02884918F010F5F1F4F882321F00E94B7
:1082D000C08EF801F6CF6091610C7091620C84E45D
:1082E00097E00E94447682E20E94C08E8AE00E945B
:1082F000C08E0E9401952EC581E09DCF0E9453DE65
:10830000AB01BC014093A9125093AA126093AB1227
:108310007093AC1288EF91E10E948E78C9CF0E94D1
:1083200053DEAB01BC014093A9125093AA12609393
:10833000AB127093AC1288EF91E10E948E780C948E
:10834000383561E08D2D0E946C4F6E2D8D2D0E9471
:10835000244EB7018D2D0E94A84F0930110509F058
:10836000A7CFF0928B06E0928A06A2CF0E94109AC5
:10837000909389068093880680E00E9413CE0E9425
:10838000109A8635910544F40E94E0A760E084E7E6
:1083900093E00E94485602C00E948C8B6091880630
:1083A00070918906072E000C880B990B0E9405E638
:1083B00020915F0430916004409161045091620407
:1083C0000E9448EC1816B4F484E893E09F938F93CE
:1083D0008091550490E001969F938F938DE693E0F2
:1083E0009F938F931F920E94718B0FB6F894DEBFFC
:1083F0000FBECDBF0E94F6E081E080930402109290
:10840000600C10925F0C23961CAE1DAE1EAE1FAE0C
:10841000239727961CAE1DAE1EAE1FAE27971BAE30
:108420002C961FAE2C979CE360969FAF6097ACE1B3
:108430006496AFAF6497B6E46896BFAF6897C12CF7
:10844000D12CF0E8EF2EAFEBFA2E812C912C5401B9
:108450006091880670918906072E000C880B990B95
:108460000E9405E6162F072F782E692E262F372F0C
:10847000482F592FB601C7010E94FFE5882311F14B
:1084800020915F0430916004409161045091620436
:10849000612F702F872D962D0E94FFE5881F88275A
:1084A000881F8BAF2896EFAD2897EE2379F08823AD
:1084B00069F080910402882309F4FACE60E088E52F
:1084C00093E06EC11C2D0D2D7E2C6F2C0E94A750A9
:1084D0006B017C01DC01CB0127962CAD3DAD4EAD8F
:1084E0005FAD2797821B930BA40BB50BB7FD47C05D
:1084F000D701C60188519C4FAF4FBF4F27968CAF15
:108500009DAFAEAFBFAF27970E94FCD6E9E6F3E080
:1085100084912F019FEF491A590A882321F00E9464
:10852000C08EF201F5CF81149104A104B104D1F001
:10853000D501C401805F984DAF4FBF4FBC01CD0145
:108540006C197D098E099F0928EE33E040E050E068
:108550000E94C4E9CA01B9010E942D8F8AE00E94DD
:10856000C08E0DC0E6E6F3E084912F01AFEF4A1A0A
:108570005A0A882321F00E94C08EF201F5CF0E9492
:108580007D920E946B7160915F0470916004809194
:108590006104909162040E9466EB072E000C880B28
:1085A000990B0E9405E61B012C019B01AC01612F78
:1085B000702F872D962D0E9421EA9F7781149104B8
:1085C000A104B10449F420E030E040E85FE30E94F8
:1085D000FFE587FF0BC008C020E030E040E450E436
:1085E0000E9448EC181614F446015701BBADBB239A
:1085F00009F443C023962CAD3DAD4EAD5FAD23973E
:10860000211531054105510541F0D701C601821BF5
:10861000930BA40BB50BB7FD30C09101A2012C96B2
:108620006FAD2C9760967FAD609764968FAD649721
:1086300068969FAD68970E9421EA20E030E040EC08
:108640005FE30E94FFE587FD34CFD701C601805A62
:108650009541AF4FBF4F23968CAF9DAFAEAFBFAF2D
:1086600023972C962FAE2C9760963FAE609764961A
:108670004FAE649768965FAE689780910402882336
:1086800009F417CF81149104A104B10429F4C12E77
:10869000D02EE72CF62CDCCE90E1C91A97E2D90A4D
:1086A000E108F108C818D908EA08FB08F7FE01CF6D
:1086B000EECF0E94109A90938D0680938C060E94B4
:1086C000E0CD0E94109A069714F00E948C8B81E0F6
:1086D000809304021092600C10925F0C80915604FB
:1086E0008093550423961CAE1DAE1EAE1FAE23977D
:1086F00027961CAE1DAE1EAE1FAE27971BAE2C9646
:108700001FAE2C97ACE36096AFAF6097BCE1649668
:10871000BFAF6497E6E46896EFAF6897C12CD12CA1
:1087200070E8E72EEFEBFE2E812C912C5401609126
:108730008C0670918D06072E000C880B990B0E94F9
:1087400005E6162F072F782E692E262F372F482F54
:10875000592FB601C7010E94FFE5882321F120911E
:108760006304309164044091650450916604612F64
:10877000702F872D962D0E94FFE5881F8827881F60
:108780008BAF2896FFAD2897FF2389F0882379F0D7
:1087900080910402882309F48BCD60E088E893E09F
:1087A0000E94485685CD1C2D0D2D7E2C6F2C0E94CD
:1087B000A7506B017C01DC01CB0127962CAD3DADB0
:1087C0004EAD5FAD2797821B930BA40BB50BB7FD86
:1087D00047C0D701C60188519C4FAF4FBF4F279666
:1087E0008CAF9DAFAEAFBFAF27970E94FCD6E5E937
:1087F000F3E084912F019FEF491A590A882321F051
:108800000E94C08EF201F5CF81149104A104B1043D
:10881000D1F0D501C401805F984DAF4FBF4FBC016F
:10882000CD016C197D098E099F0928EE33E040E0E7
:1088300050E00E94C4E9CA01B9010E942D8F8AE06C
:108840000E94C08E0DC0E2E9F3E084912F01AFEFEA
:108850004A1A5A0A882321F00E94C08EF201F5CFED
:108860000E947D920E946B71609163047091640418
:1088700080916504909166040E9466EB072E000CBF
:10888000880B990B0E9405E61B012C019B01AC0192
:10889000612F702F872D962D0E9421EA9F778114DA
:1088A0009104A104B10449F420E030E040E85FE322
:1088B0000E94FFE587FF0BC008C020E030E040E4E5
:1088C00050E40E9448EC181614F446015701BBAD61
:1088D000BB2309F443C023962CAD3DAD4EAD5FAD37
:1088E0002397211531054105510541F0D701C601F6
:1088F000821B930BA40BB50BB7FD30C09101A201F5
:108900002C966FAD2C9760967FAD609764968FAD77
:10891000649768969FAD68970E9421EA20E030E056
:1089200040EC5FE30E94FFE587FD32CFD701C6012F
:10893000805A9541AF4FBF4F23968CAF9DAFAEAFDE
:10894000BFAF23972C962FAE2C9760963FAE6097C3
:1089500064964FAE649768965FAE68978091040204
:10896000882309F415CF81149104A104B10429F4DA
:10897000C12ED02EE72CF62CDACE90E1C91A97E260
:10898000D90AE108F108C818D908EA08FB08F7FE77
:10899000FFCEEECF0E945B5D88E50E94669988233A
:1089A00019F05F9A1092AC0489E50E9466998823B9
:1089B00019F08A9A1092AD048AE50E94669988237C
:1089C00051F09FB7F894809108018160809308016D
:1089D0009FBF1092AE0485E40E946699882309F433
:1089E00067CC129A65CC29964EAD5FAD29971416C7
:1089F00015060CF049C1CE57DF4F88809980AA80B8
:108A0000BB80C258D040880E991EAA1EBB1ECE57EE
:108A1000DF4F288139814A815B81C258D040281BB1
:108A2000390B4A0B5B0BCA01B901A30192010E94E9
:108A3000B5E9A50194010E94E6E923964CAC5DAC32
:108A40006EAC7FAC2397420E531E641E751E34E13C
:108A500043165104610471041CF14CEE4416510498
:108A6000610471043CF450E845165104610471043A
:108A70003CF105C05BEE452E512C612C712C2396E8
:108A80004CAE5DAE6EAE7FAE23978EEF90E0A0E071
:108A9000B0E084199509A609B7092C013D0116C05B
:108AA00024E130E040E050E023962CAF3DAF4EAFE4
:108AB0005FAF239744E1442E512C612C712C06C0EA
:108AC00023964CAE5DAE6EAE7FAE239723964CAD33
:108AD0005DAD6EAD7FAD23978AEA96E00E94FFDD23
:108AE000B301A20185EA96E00E94FFDD68964FADD2
:108AF00068976C965FAD6C97A0966FADA097AC969B
:108B00007FADAC978EE996E00E94B864E0964FADD9
:108B1000E097A4965FADA497A8966FADA897E4964A
:108B20007FADE49787E996E00E94B86429964EAD40
:108B30005FAD2997433051050CF4A6C0C301B201C3
:108B40000E9405E620E030E040E850E40E9464E640
:108B50006B017C0168962FAD68976C963FAD6C9762
:108B6000A0964FADA097AC965FADAC97E0966FAD79
:108B7000E097A4967FADA497A8968FADA897E496AA
:108B80009FADE4970E9421EA2BED3FE049E450E4D9
:108B90000E9464E620E030E040E05FE30E9464E68B
:108BA0009B01AC01C701B6010E94FEEA6B017C018A
:108BB000C501B4010E9405E62FE632E143E85AE31D
:108BC0000E9464E64B015C01B701A60181E996E0D1
:108BD0000E94B864B501A4018BE896E00E94B864D5
:108BE0002AE939E949E15FE3C701B6010E9464E679
:108BF0006B017C019B01AC010E9422EAA50194015A
:108C00000E94FEEAE8966CAF7DAF8EAF9FAFE8970B
:108C1000A5019401C701B6010E9464E620E030E09E
:108C200040E05EE30E9464E6EC966CAF7DAF8EAFF1
:108C30009FAFEC97EBE7F6E084915F015FEFA51A39
:108C4000B50A882321F00E94C08EF501F5CFB70147
:108C5000A60185E796E00E94B864E8964CAD5DAD4C
:108C60006EAD7FADE8978FE696E00E94B864EC9613
:108C70004CAD5DAD6EAD7FADEC9789E696E00E94A0
:108C8000B8648AE00E94C08E23968CAD9DADAEADD7
:108C9000BFAD2397840D951DA61DB71DB595A7954E
:108CA0009795879580932F1329968EAD9FAD299721
:108CB000019629969FAF8EAF299724969FAD249752
:108CC00068969FAF68972C96AFAD2C976C96AFAF18
:108CD0006C976096BFAD6097A096BFAFA097649663
:108CE000EFAD6497AC96EFAFAC978BAC9CACADACF2
:108CF000BEACF1E0EE96FFAFEE970C94683E0E949A
:108D000088D7D6CA0E945B5DD02E60E0802F0E947B
:108D10006C4F4FEFE416F40659F4802F0E949BD954
:108D200031E020E0892B09F030E0032F122F05C03D
:108D3000EA94EF2861F000E010E08D2D0E949BD9AD
:108D40008017910709F4B4CA0E947D92F6CF01E022
:108D500010E0F3CFC157DF4F0FB6F894DEBF0FBE60
:108D6000CDBFDF91CF911F910F91FF90EF90DF90DA
:108D7000CF90BF90AF909F908F907F906F905F90BB
:108D80004F903F902F9008954F925F926F927F92F5
:108D90008F929F92AF92BF92CF92DF92EF92FF920B
:108DA0000F931F93CF93DF93CDB7DEB762970FB6C4
:108DB000F894DEBF0FBECDBF10929B060E94A75055
:108DC00000919004109191042091920430919304A9
:108DD0006B017C01C01AD10AE20AF30AF7FC13C046
:108DE00020918F04209520938F04DC01CB018A54BD
:108DF0009C4FAF4FBF4F8093900490939104A093EA
:108E00009204B0939304FF24F39480918F04811112
:108E100001C0F12C0E94ED558091D30F853198F45B
:108E2000FF2049F080918A0690918B06892B19F0DA
:108E30000DE918E002C000E817E023E14FE061E02F
:108E400089E00E941DA58091D30F8D3108F093C158
:108E50008830D0F56091880670918906072E000C45
:108E6000880B990B0E9405E620E030E040E05FE3CC
:108E70000E9422EA0E9466EB7C876B87643671054C
:108E80002CF46A30710524F426E003C022E101C00D
:108E90002CE082E190E0821B910997FD0196959567
:108EA00087959195819591098B5F8093D60F87E087
:108EB0008093D70FCE010B960E9455550E94C7D0C4
:108EC0008DE797E00E94BAD08091D30F8D3108F0E2
:108ED00044C08091D50F853108F43FC060915F0494
:108EE0007091600480916104909162040E9466EB2D
:108EF000072E000C880B990B0E9405E620E030E05D
:108F000040E05FE30E9422EA0E9466EB9B017E87BD
:108F10006D87643671050CF06BC32A3031050CF097
:108F200065C326E082E190E0821B910997FD0196DE
:108F3000959587959195819591098B5F8093D60F33
:108F40008CE18093D70FCE010D960E9455550E945B
:108F5000C7D08DE797E00E94BAD08091D30F8531BA
:108F600040F58091D50F813120F160918806709194
:108F70008906072E000C880B990B0E9405E62091AC
:108F80005F043091600440916104509162040E943A
:108F900048EC18160CF02EC31092BF0F02E022E02E
:108FA00041E16DE08FE99FE00E94C8B581E08093C8
:108FB000BF0F8091D30F8830D0F560918C067091EF
:108FC0008D06072E000C880B990B0E9405E620E009
:108FD00030E040E05FE30E9422EA0E9466EB788B7B
:108FE0006F87643671052CF46A30710524F426E02D
:108FF00003C022E101C02CE082E190E0821B9109D4
:1090000097FD0196959587959195819591098F5A30
:109010008093D60F87E08093D70FCE010F960E94E2
:1090200055550E94C7D08DE797E00E94BAD0809135
:10903000D30F8D3108F044C08091D50F853108F4ED
:109040003FC06091630470916404809165049091C5
:1090500066040E9466EB072E000C880B990B0E9499
:1090600005E620E030E040E05FE30E9422EA0E9453
:1090700066EB9B017A8B698B643671050CF0C5C277
:109080002A3031050CF0BFC226E082E190E0821B5D
:10909000910997FD019695958795919581959109EF
:1090A0008F5A8093D60F8CE18093D70FCE014196D3
:1090B0000E9455550E94C7D08DE797E00E94BAD014
:1090C0008091D30F853140F58091D50F813120F10A
:1090D00060918C0670918D06072E000C880B990B01
:1090E0000E9405E620916304309164044091650478
:1090F000509166040E9448EC18160CF088C2109239
:10910000BF0F02E022E042E168E58FE99FE00E94A4
:10911000C8B581E08093BF0F8091D30F8C3158F593
:109120008091D50F843138F120918A0630918B06D9
:109130002F5F3F4F44E6429FC001439F900D112493
:1091400097FF02C081509F4F292F392F330F330BC8
:109150003A832983232B79F088E68093D60F8BE11D
:109160008093D70FCE0101960E9455550E94C7D01B
:1091700085E20E94A6868091D30F843328F48091E3
:10918000D50F8A3208F04CC28091D30F853328F472
:109190008091D50F813308F06BC280912D10882308
:1091A00009F44BC08091D30F843308F046C08091FE
:1091B000D50F823308F441C02091FB11222319F10D
:1091C0008091A5129091A612A091A712B091A81219
:1091D0000097A105B10509F452C2BC01CD016D593A
:1091E0007F4F8F4F9F4F24E630E040E050E00E94D9
:1091F000C4E96091A9127091AA128091AB1290916A
:10920000AC120E94C4E948E4249FB0011124072E47
:10921000000C880B990B0E9405E62AE037ED43E22B
:109220005CE30E9464E60E946BEB262F02E042E3BF
:1092300067E38FE99FE00E94C8B58091D30F813327
:1092400008F060C08091D50F893208F45BC00E949D
:10925000F9A72B013C018CE3882E912CA12CB12C79
:10926000C301B201A50194010E94C4E9CA01B90178
:10927000A50194010E94C4E9CA01962E872E5901C6
:109280008E010F5F1F4F41E8441641E5540641E04F
:109290006406710408F4F5C1B90128E130E040E04A
:1092A00050E00E94C4E929013A018F929F92C501C2
:1092B00068E170E00E94E6EC9F938F935F924F927B
:1092C00089E697E09F938F931F930F930E9498E5F1
:1092D0000FB6F894DEBF0FBECDBF9AE04916510419
:1092E0006104710408F0FCC197E0892F880F980F82
:1092F0009195955A9093D60F80E38093D70FC8012C
:109300000E94C7D0E091990FF0919A0F848181114A
:10931000D4C06091BC047091BD048091BE04909152
:10932000BF040E9466EB7A836983CE0101960E9496
:10933000E954BC0180EA94E00E946FED6091C004A2
:109340007091C1048091C2049091C3040E9466EBA5
:109350007A836983CE0101960E94E954BC018BE9AE
:1093600094E00E946FED2CEA35EC47E257E3609100
:10937000C4047091C5048091C6049091C7040E94F2
:1093800022EA20E030E048EC52E40E9464E60E94C9
:1093900066EB4B015C0197FD19C090E1891697E2DD
:1093A0009906A104B104E4F0C501B40120E137E25B
:1093B00040E050E00E94E6E9CA01B9012AE030E04D
:1093C00040E050E00E94E6E9605D0BC0B094A094DC
:1093D00090948094811C911CA11CB11C6DE201C071
:1093E00060E26093490C28EE821623E09206A10405
:1093F000B10494F0C501B40128EE33E040E050E040
:109400000E94E6E9CA01B9012AE030E040E050E0FC
:109410000E94E6E9605D01C060E260934A0CC5010C
:10942000B40124E630E040E050E00E94E6E99AE032
:10943000492E512C612C712CCA01B901A301920152
:109440000E94E6E9605D60934B0CC501B401A30185
:1094500092010E94E6E94B015C01672B682B692BA6
:1094600079F08EE280934C0CCA01B901A3019201FC
:109470000E94E6E9605D60934D0C80E3880D15C0A5
:10948000CA01B901A30192010E94E6E9662339F0FD
:109490008EE280934C0C605D60934D0C05C080E2C1
:1094A00080934D0C80934C0C80E280934E0C69E4C9
:1094B0007CE084E994E00E946FED8091D30F8832C4
:1094C00098F48091D50F8D3178F02BE040E86DE174
:1094D00080E00E9448A68091D30F873228F48091C3
:1094E000D50F8F3108F0FEC08091D30F823328F45E
:1094F0008091D50F8B3208F060C18091D30F8034FA
:1095000028F48091D50F883308F074C180919D06AE
:10951000882349F00E94F6CF40E050E0BA0181E490
:109520009CE40E948ACF2091190230911A02409146
:109530007606509177066091780670917906C90198
:10954000840F951F2436310524F4853691053CF4AB
:1095500016C02436310531F08436910584F484E652
:1095600090E00DC04B3051056105710514F00A976C
:1095700006C0463F5F4F6F4F7F4F6CF40A96909343
:109580001A028093190210927606109277061092B2
:109590007806109279068091190290911A028A3009
:1095A00091053CF0883E43E094072CF087EE93E071
:1095B00002C08AE090E090931A02809319026296AA
:1095C0000FB6F894DEBF0FBECDBFDF91CF911F91D4
:1095D0000F91FF90EF90DF90CF90BF90AF909F9052
:1095E0008F907F906F905F904F9008952CE09ACC71
:1095F00022E198CC02E022E041E16DE08FE99FE0BA
:109600000E94C8B5D6CC2CE040CD22E13ECD02E090
:1096100022E042E168E58FE99FE00E94C8B57CCD79
:1096200007E028E04AE26AE28FE99FE00E94C8B5BD
:1096300005E022E04CE262E38FE99FE00E94C8B5BA
:1096400024E04AE061E38AE20E9448A66091A10F0B
:109650007091A20F82E38093BB0F8BE28093BC0FCB
:109660002BEB3FE042E38FE99FE00E94B0B48CCD4A
:1096700024E04AE461E386E30E9448A68ECD20E020
:10968000C2CD44E6A416B104C0F48F929F92C501E6
:1096900068E170E00E94E6EC9F938F938FE597E07E
:1096A0009F938F931F930F930E9498E50FB6F894A2
:1096B000DEBF0FBECDBF95E018CE8F929F923F9335
:1096C0002F9387E597E09F938F931F930F930E94AB
:1096D00098E50FB6F894DEBF0FBECDBF96E005CE7D
:1096E00098E003CE83E08093D60F86E28093D70F75
:1096F000FF2029F08BE797E00E94BAD00DC080913F
:109700006704811102C08FE305C08091AC04811110
:10971000F1CF80E20E94A6868BE08093D60F16E2FE
:109720001093D70F80EA94E00E94C7D08BE2809319
:10973000D60F1093D70FFF2029F089E797E00E94FA
:10974000BAD00DC080916804811102C08FE305C0BA
:109750008091AD048111F1CF80E20E94A68683E35F
:109760008093D60F16E21093D70F8BE994E00E94F6
:10977000C7D083E58093D60F1093D70FFF2029F031
:1097800087E797E00E94BAD00DC0809169048111EB
:1097900002C08FE305C08091AE048111F1CF80E259
:1097A0000E94A6868BE58093D60F86E28093D70F22
:1097B00084E994E00E94C7D097CE84E00E94DCCF79
:1097C00083E08093D60F12E31093D70F86E00E94B8
:1097D000A6D00E94ED558CE08093D60F1093D70F42
:1097E00089E192E00E9455550E94C7D085E20E940F
:1097F000A68683CE1092D60F8FE38093D70F86E490
:1098000092E00E94C7D082CE80915E048630D8F468
:1098100096E0899FF0011124E559FB4F20910D023C
:1098200030910E0231832083409176065091770665
:1098300060917806709179064283538364837583BF
:109840008F5F80935E04089540E050E0BA0184EC9D
:1098500096E40C948ACFE0915E04EE2389F0E15007
:10986000E0935E0486E0E89FF0011124E559FB4F88
:109870004281538164817581808191810C948ACF6A
:10988000E3CF0F931F93CF93DF9310929B068091AA
:10989000760690917706A0917806B091790681308E
:1098A0009048A105B10540F0109276061092770617
:1098B0001092780610927906C09176068091A504E0
:1098C0001816DCF4282F082E000C330B2150310918
:1098D0004C2F0C2E000C550B4217530774F0CFEF92
:1098E000C80F8C2F90E0A0E0B0E0809376069093B4
:1098F0007706A0937806B09379061092BA128091F9
:10990000B912C81714F4C093B9128091B912082E75
:10991000000C990B04962C2F0C2E000C330B821785
:10992000930724F48CEF8C0F8093B9121091B91225
:10993000D0E001E0112341F08091FD0F9091FE0FE6
:10994000891B8F70B9F519C080914002882349F0B6
:1099500081E0C11180E024E04AE15AE06D2F0E94CD
:10996000AE5580919D06882339F3C111E5CF73DF91
:109970008091BA12882301F30EC180912D108111BC
:1099800019C01130D1F480914002882351F081E058
:10999000C13009F080E023E04DE05AE06D2F0E94D5
:1099A000AE5580919D06882331F1C13021F583ECBD
:1099B00096E61BC0113009F4D6C01230E1F4809154
:1099C0004002882351F081E0C23009F080E023E0BA
:1099D00045E05AE06D2F0E94AE5580919D06882388
:1099E00051F0C23041F482E094E80E9442598091E3
:1099F000BA128111D0C080912E10882309F48BC037
:109A00008091FB11882309F476C080912D10882362
:109A1000E9F01330D9F580914002882351F081E0BC
:109A2000C33009F080E020E249EF59E06D2F0E9439
:109A3000AE5580919D06882309F48CC0C33009F08F
:109A400089C010922D100E94CC8B50C01330F1F4BD
:109A500080914002882351F081E0C33009F080E01A
:109A600020E24CEE59E06D2F0E94AE5580919D068C
:109A7000882309F46FC0C33009F06CC080912E10A8
:109A8000811100932D100E948C8B30C0143009F08E
:109A900061C080914002882351F081E0C43009F018
:109AA00080E020E241EE59E06D2F0E94AE5580919A
:109AB0009D06882309F44EC0C43009F04BC00E94B3
:109AC0009C8680916A0480936D0610926E060E94B7
:109AD00044D50E94E0A710928B0610928A0610923D
:109AE000040260E08AEB99E00E9448568091BA1225
:109AF000882381F150C0133011F084E02CC0809194
:109B000040028823C1F081E0C33009F080E023E007
:109B100043ED59E00DC0133081F780914002882356
:109B200051F081E0C33009F080E023E048EC59E0D7
:109B30006D2F0E94AE5580919D068823F1F2C330AF
:109B4000E1F683E79EEA0E9442598091BA12882387
:109B5000A1F221C085E0DF5F1F5FD53009F0EACEBA
:109B60008093A50418C080914002882349F081E0C9
:109B7000C13009F080E023E045E15AE06D2FEED7D7
:109B800080919D06882309F436CFC13009F033CF88
:109B900082E19AE62ACFDF91CF911F910F9108952C
:109BA000CF92DF92EF92FF920F931F93CF93DF93A9
:109BB0006C017A018B01C0E0D0E0CE15DF0589F0A1
:109BC000D8016D918D01D601ED91FC910190F0814C
:109BD000E02DC6011995892B11F47E0102C0219652
:109BE000ECCFC701DF91CF911F910F91FF90EF90C4
:109BF000DF90CF9008950E941BED0F931F93CF939A
:109C0000DF93EB018A01181619066CF4843121E008
:109C1000920714F083E191E090938906809388067F
:109C200080E00E9413CED7FD06C0D0938D06C0936E
:109C30008C060E94E0CD10938B0600938A06DF917C
:109C4000CF911F910F9100CE1F93CF93DF93282FB9
:109C500030E0F901EE58F44F8491F901E45DF44FDE
:109C6000D491F901EA51F54FC491CC23C1F0162FDC
:109C70008111DCD0EC2FF0E0EE0FFF1FEE54F54F1A
:109C8000A591B4918FB7F894111105C09C91ED2F57
:109C9000E095E92302C0EC91ED2BEC938FBFDF91AF
:109CA000CF911F9108951F920F920FB60F9211241A
:109CB0000BB60F922F933F934F935F936F937F93C6
:109CC0008F939F93AF93BF93EF93FF93809172060F
:109CD00090917306A0917406B0917506892B8A2B1A
:109CE0008B2B59F180917106E0916F06F09170060F
:109CF0009081892780838091720690917306A0914C
:109D00007406B0917506181619061A061B060CF093
:109D100055C08091720690917306A0917406B0911F
:109D200075060197A109B109809372069093730695
:109D3000A0937406B093750641C080910C02E1E2D5
:109D4000FDE0E4919FEF90930C02E230C9F050F4F3
:109D5000EE2399F0E13081F590916F009D7F909313
:109D60006F002AC0E43019F1E0F0E53029F5909158
:109D700073009D7F909373001FC010926E001CC0F3
:109D8000909170009D7F9093700091E09093B0004F
:109D90009091B100987F94609093B1001092B300BD
:109DA0000BC0909171009D7F9093710005C09091C0
:109DB00072009D7F9093720060E046DFFF91EF910B
:109DC000BF91AF919F918F917F916F915F914F91D3
:109DD0003F912F910F900BBE0F900FBE0F901F90D1
:109DE00018953FB7F8948091B8069091B906A09164
:109DF000BA06B091BB0626B5A89B05C02F3F19F047
:109E00000196A11DB11D3FBFBA2FA92F982F8827FA
:109E1000820F911DA11DB11DBC01CD0142E0660F55
:109E2000771F881F991F4A95D1F7089590E0FC018C
:109E30003197E231F10508F04EC08827EE58FF4F08
:109E40008F4F0C940DED809180008F7703C080912F
:109E500080008F7D80938000089580918000877FAF
:109E6000F9CF84B58F7702C084B58F7D84BD089506
:109E70008091B0008F7703C08091B0008F7D809378
:109E8000B0000895809190008F7707C08091900076
:109E90008F7D03C080919000877F8093900008950C
:109EA0008091A0008F7707C08091A0008F7D03C0B4
:109EB0008091A000877F8093A00008958091200169
:109EC0008F7707C0809120018F7D03C08091200192
:109ED000877F809320010895CF93DF9390E0FC016A
:109EE000E45DF44F2491FC01EA51F54F84918823FD
:109EF00061F190E0880F991FFC01E35CF24FC5917E
:109F0000D491FC01EE54F54FA591B491611109C0B3
:109F10009FB7F8948881209582238883EC912E2323
:109F20000BC0623061F49FB7F8943881822F80951E
:109F300083238883EC912E2B2C939FBF06C08FB771
:109F4000F894E8812E2B28838FBFDF91CF9108955D
:109F50001F93CF93DF93182FEB0161E0BDDF2097B4
:109F600011F460E004C0CF3FD10531F461E0812FEE
:109F7000DF91CF911F9168CEE12FF0E0EE58F44FC2
:109F8000E4914E2F50E0FA013197E231F10508F0EB
:109F90009DC08827EC57FF4F8F4F0C940DED84B573
:109FA000806884BDC7BD97C084B5806284BDC8BDCC
:109FB00092C080918000806880938000D093890057
:109FC000C093880088C08091800080628093800068
:109FD000D0938B00C0938A007EC0809180008860FF
:109FE00080938000D0938D00C0938C0074C08091CA
:109FF000B00080688093B000C093B3006CC08091C3
:10A00000B00080628093B000C093B40064C08091BF
:10A010009000806880939000D0939900C09398003E
:10A020005AC080919000806280939000D0939B00F2
:10A03000C0939A0050C080919000886080939000F7
:10A04000D0939D00C0939C0046C08091A000806882
:10A050008093A0008091A0008F7B8093A000D0937C
:10A06000A900C093A80037C08091A00080628093AF
:10A07000A000D093AB00C093AA002DC08091A00097
:10A0800088608093A000D093AD00C093AC0023C043
:10A0900080912001806880932001D0932901C09392
:10A0A000280119C080912001806280932001D09303
:10A0B0002B01C0932A010FC08091200188608093FA
:10A0C0002001D0932D01C0932C0105C0C038D105CB
:10A0D0000CF04CCF46CFDF91CF911F9108958F9216
:10A0E0009F92AF92BF92CF92DF92EF92FF926B015D
:10A0F0007C0177DE4B015C01C114D104E104F10461
:10A10000E9F06FDEDC01CB0188199909AA09BB09C6
:10A11000883E9340A105B10578F321E0C21AD10829
:10A12000E108F10888EE880E83E0981EA11CB11C9E
:10A13000C114D104E104F10421F7DECFFF90EF90C8
:10A14000DF90CF90BF90AF909F908F9008952FB7E2
:10A15000F8946091B4067091B5068091B60690911E
:10A16000B7062FBF08951F920F920FB60F921124BA
:10A170002F933F938F939F93AF93BF938091B40698
:10A180009091B506A091B606B091B7063091B3068E
:10A1900023E0230F2D3720F40196A11DB11D05C02A
:10A1A00026E8230F0296A11DB11D2093B3068093CC
:10A1B000B4069093B506A093B606B093B706809107
:10A1C000B8069091B906A091BA06B091BB06019667
:10A1D000A11DB11D8093B8069093B906A093BA064D
:10A1E000B093BB06BF91AF919F918F913F912F91FB
:10A1F0000F900FBE0F901F9018958F929F92AF9265
:10A20000BF92CF92DF92EF92FF92CF93FC01C0807A
:10A21000D180E280F38020E030E0A901C701B601DF
:10A220000E94FFE587FF08C0C701B601905820E0F3
:10A2300030E048EC52E406C020E030E048EC52E464
:10A24000C701B6010E9464E60E9466EB6B017C01C7
:10A25000603AF6E87F07F1E08F07910584F020EA85
:10A2600036E841E050E00E94E6E9CA01B9012AE07F
:10A2700030E040E050E00E94E6E9605D01C060E24D
:10A280006093480C80E1C81687E2D806E104F10427
:10A2900094F0C701B60120E137E240E050E00E94AF
:10A2A000E6E9CA01B9012AE030E040E050E00E944E
:10A2B000E6E9605D01C060E26093490CE8EECE160D
:10A2C000E3E0DE06E104F10494F0C701B60128EEF4
:10A2D00033E040E050E00E94E6E9CA01B9012AE01B
:10A2E00030E040E050E00E94E6E9605D01C060E2DD
:10A2F00060934A0CC701B60124E630E040E050E02C
:10A300000E94E6E98AE0882E912CA12CB12CCA018A
:10A31000B901A50194010E94E6E9605D60934B0CD0
:10A320008EE280934C0CC701B601A50194010E94F6
:10A33000E6E9C62FCA01B901A50194010E94E6E928
:10A34000605D60934D0CC05DC0934E0C88E49CE052
:10A35000CF91FF90EF90DF90CF90BF90AF909F9004
:10A360008F9008950F931F93CF93DF9300D01F9288
:10A37000CDB7DEB78091760690917706A0917806EA
:10A38000B0917906B7FF08C0109276061092770652
:10A39000109278061092790680917A0690917B0649
:10A3A000A0917C06B0917D0640917606509177068B
:10A3B000609178067091790684179507A607B7070C
:10A3C00044F48093760690937706A0937806B09332
:10A3D000790680914002882371F140917606509170
:10A3E0007706609178067091790680917E0690914B
:10A3F0007F06A0918006B09181068A019B01080F1B
:10A40000191F2A1F3B1FC901B8010E9405E62AE057
:10A4100037ED43E25CE30E9464E669837A838B83D1
:10A420009C83CE010196E9DEBC0180918406909167
:10A4300085060E94D9D080919D06882381F14091A4
:10A440007606509177066091780670917906809132
:10A450007E0690917F06A0918006B09181068A01C8
:10A460009B01080F191F2A1F3B1FC901B8010E9439
:10A4700005E62AE037ED43E25CE30E9464E6E09102
:10A480008206F0918306309721F060837183828386
:10A490009383E1D9E0918606F091870619950F9094
:10A4A0000F900F900F90DF91CF911F910F91089512
:10A4B0008F929F92AF92BF92CF92DF92EF92FF92D4
:10A4C000CF9320E030E048EC52E4FC0160817181E0
:10A4D000828193810E9464E60E9466EB6B017C019D
:10A4E00097FF0AC0F094E094D094C094C11CD11C92
:10A4F000E11CF11C8DE201C08BE28093480CC70186
:10A50000B60120E137E240E050E00E94E6E98AE04F
:10A51000882E912CA12CB12CCA01B901A50194015E
:10A520000E94E6E9605D6093490CC701B60128EE20
:10A5300033E040E050E00E94E6E9CA01B901A5011C
:10A5400094010E94E6E9605D60934A0CC701B60180
:10A5500024E630E040E050E00E94E6E9CA01B9019B
:10A56000A50194010E94E6E9605D60934B0C8EE2C8
:10A5700080934C0CC701B601A50194010E94E6E945
:10A58000C62FCA01B901A50194010E94E6E9605DE8
:10A5900060934D0CC05DC0934E0C88E49CE0CF915D
:10A5A000FF90EF90DF90CF90BF90AF909F908F90F3
:10A5B00008958F929F92AF92BF92CF92DF92EF92C7
:10A5C000FF92FC01C080D180E280F38020E030E087
:10A5D000A901C701B6010E94FFE587FF04C0C701BA
:10A5E000B601905802C0C701B6010E9466EB6B012C
:10A5F0007C016031F7E27F078105910584F020E15D
:10A6000037E240E050E00E94E6E9CA01B9012AE0E1
:10A6100030E040E050E00E94E6E9605D01C060E2A9
:10A6200060934A0C88EEC81683E0D806E104F10472
:10A6300094F0C701B60128EE33E040E050E00E94FC
:10A64000E6E9CA01B9012AE030E040E050E00E94AA
:10A65000E6E9605D01C060E260934B0CE4E6CE1673
:10A66000D104E104F10494F0C701B60124E630E01E
:10A6700040E050E00E94E6E9CA01B9012AE030E07A
:10A6800040E050E00E94E6E9605D01C060E2609356
:10A690004C0CFAE0CF16D104E104F1049CF08AE0FE
:10A6A000882E912CA12CB12CC701B601A5019401D3
:10A6B0000E94E6E9CA01B901A50194010E94E6E9F8
:10A6C000605D01C060E260934D0CC701B6012AE0F5
:10A6D00030E040E050E00E94E6E9605D60934E0C9F
:10A6E0008AE49CE0FF90EF90DF90CF90BF90AF9016
:10A6F0009F908F9008950F931F93CF93DF9300D077
:10A700001F92CDB7DEB78091760690917706A09123
:10A710007806B0917906B7FF08C0109276061092BD
:10A720007706109278061092790680917A069091B9
:10A730007B06A0917C06B0917D06409176065091F3
:10A740007706609178067091790684179507A607B9
:10A75000B70744F48093760690937706A093780623
:10A76000B093790680914002882371F1409176067A
:10A7700050917706609178067091790680917E06F7
:10A7800090917F06A0918006B09181068A019B017D
:10A79000080F191F2A1F3B1FC901B8010E9403E6B9
:10A7A00020E030E048EC52E40E9464E669837A835A
:10A7B0008B839C83CE010196FCDEBC0180918406D4
:10A7C000909185060E94D9D080919D06882391F1B1
:10A7D00040917606509177066091780670917906DF
:10A7E00080917E0690917F06A0918006B0918106AF
:10A7F0008A019B01080F191F2A1F3B1FC901B801BD
:10A800000E9403E620E030E048EC52E40E9464E657
:10A810000E946BEBE0918206F0918306309721F065
:10A82000608371838283938316D8E0918606F091CA
:10A83000870619950F900F900F900F90DF91CF9191
:10A840001F910F91089520E030E040E251E4FC01B7
:10A8500060817181828193810E9464E60E9466EB2F
:10A860009B0177FF06C022273327261B370B8DE27B
:10A8700001C08BE28093490CC90168EE73E00E942D
:10A88000FAECCB01EAE0F0E0BF010E94FAEC805D57
:10A8900080934A0CC90164E670E00E94FAECCB0197
:10A8A000BF010E94FAEC805D80934B0CC901BF018F
:10A8B0000E94FAEC282FCB01BF010E94FAEC805DC8
:10A8C00080934C0C8EE280934D0C205D20934E0CB7
:10A8D00089E49CE008958F929F92AF92BF92CF92AD
:10A8E000DF92EF92FF92CF9320E030E048EC52E409
:10A8F000FC0160817181828193810E9464E60E94E3
:10A9000066EB6B017C0197FD10C020E137E240E06F
:10A9100050E00E94E6E9CA01B9012AE030E040E0D7
:10A9200050E00E94E6E9605D09C0F094E094D094A4
:10A93000C094C11CD11CE11CF11C6DE26093490C58
:10A94000C701B60128EE33E040E050E00E94E6E99E
:10A950008AE0882E912CA12CB12CCA01B901A50145
:10A9600094010E94E6E9605D60934A0CC701B6015C
:10A9700024E630E040E050E00E94E6E9CA01B90177
:10A98000A50194010E94E6E9605D60934B0C8EE2A4
:10A9900080934C0CC701B601A50194010E94E6E921
:10A9A000C62FCA01B901A50194010E94E6E9605DC4
:10A9B00060934D0CC05DC0934E0C89E49CE0CF9138
:10A9C000FF90EF90DF90CF90BF90AF909F908F90CF
:10A9D0000895FC0140815181852F881F8827881F99
:10A9E00029F022273327241B350B01C09A01483E4A
:10A9F0005340ACF0C90168EE73E00E94FAECCB0161
:10AA0000EAE0F0E0BF010E94FAEC805D80934B0C1D
:10AA1000C90164E670E00E94FAECCB0112C0243652
:10AA20003105B4F0811102C080E201C08DE2809353
:10AA30004B0CC90164E670E00E94FAECCB01EAE03D
:10AA4000F0E0BF010E94FAEC805D80934C0C11C0D5
:10AA500090E290934B0C90934C0C2A3031059CF073
:10AA6000811102C080E201C08DE280934C0CEAE0CB
:10AA7000F0E0C901BF010E94FAECCB01BF010E94C6
:10AA8000FAEC805D05C0811102C080E201C08DE258
:10AA900080934D0CC9016AE070E00E94FAEC805D81
:10AAA00080934E0C8BE49CE00895FC012081318161
:10AAB00037FD0FC0243631058CF0C90164E670E023
:10AAC0000E94FAECCB016AE070E00E94FAEC805D33
:10AAD00006C03195219531098DE201C080E2809355
:10AAE0004C0C2A30310564F0EAE0F0E0C901BF0106
:10AAF0000E94FAECCB01BF010E94FAEC805D01C01C
:10AB000080E280934D0CC9016AE070E00E94FAEC8B
:10AB1000805D80934E0C8CE49CE00895CF92DF9290
:10AB2000EF92FF926B017C0183E3C816D104E1042C
:10AB3000F10460F082E3C81AD108E108F10862E389
:10AB400070E080E090E0CBDA21D6EECFC701B6010D
:10AB5000C6DAFF90EF90DF90CF9018C60F931F9347
:10AB6000CF93DF93982F862F8A01D22F692F0E94CF
:10AB7000ADCF9091D30F8091470C891748F19091F8
:10AB8000D50F8091460C981718F1C4E1F801849113
:10AB9000882331F00E948FD0C81B0F5F1F4FF6CF64
:10ABA000CC2329F080E20E94A686C150F9CF809183
:10ABB000470C9AE79093D60F8093D70F8D2F0E9462
:10ABC000A6D080E2DF91CF911F910F910C94A686C1
:10ABD000DF91CF911F910F91089587E59DE00E942D
:10ABE000A8A581E080939F0608950F931F93AFDA85
:10ABF0000091AF061091B0062091B1063091B206D7
:10AC0000DC01CB01801B910BA20BB30BB7FD0CC079
:10AC100086B186FB992790F981E08927349B826071
:10AC2000329B84608093AE068091AE0681709091D5
:10AC3000AE0691FD82609091AD06891731F18130A9
:10AC4000A9F028F0823041F0833059F01CC09130D7
:10AC500089F0923099F017C0992361F0933071F028
:10AC600012C0913059F0923071F404C0992331F040
:10AC7000933049F49091AC06915003C09091AC068A
:10AC80009F5F9093AC068093AD061F910F9108953E
:10AC90009C018091500C681778F0962FB901909321
:10ACA000500C42E450E086E492E00E946FE50E947E
:10ACB0002FA883E08093400208952091500C211129
:10ACC0000CC0BC0142E450E086E492E00E9484EDB6
:10ACD0000E942FA883E08093400208954F925F92D4
:10ACE0006F927F928F929F92AF92BF92CF92DF929C
:10ACF000EF92FF920F931F93CF93DF9300D01F9299
:10AD0000CDB7DEB710910F021F3FF1F020DAC090EF
:10AD10008E06D0908F06E0909006F0909106DC01B0
:10AD2000CB018C199D09AE09BF09B7FD0DC020915B
:10AD3000FE0F8091FD0F30E090E001968F70992713
:10AD40002817390709F011C250DF8091AE0682FF43
:10AD50003EC08091AB0681113CC081E08093AB0680
:10AD600090919E06892780939D0610929E0683E00F
:10AD7000809340021092AE06EAD9DC01CB018C50E0
:10AD80009E4FAF4FBF4F8093AF069093B006A093F6
:10AD9000B106B093B20680ED97E09C838B8382E38B
:10ADA00090E09A838983BE016D5F7F4FCE0101964B
:10ADB0000E943D8B16E0115061F08FEF9FE00E94E2
:10ADC000E96C62E070E080E090E089D9F4CF109205
:10ADD000AB0610910901109511708091AA06181701
:10ADE000A1F0112309F4E2C10E94FB898091AA0617
:10ADF000823021F060E08FE29DE04ADF1093AA06E6
:10AE000083E0809340020E94F6CFA1D96B017C01C0
:10AE10008091A6069091A706A091A806B091A906D8
:10AE2000A7019601281B390B4A0B5B0B57FF05C086
:10AE300080919C06882309F4F4C1D701C6018C597E
:10AE40009F4FAF4FBF4F8093A6069093A706A09346
:10AE5000A806B093A9068091AC0618162CF4809130
:10AE6000AC06843074F408C08091AC0699278195B3
:10AE70000CF4909504972CF480919D0681119FC04D
:10AE8000AFC080919B06882309F472C08091AC0604
:10AE9000181664F48091AC06082E000C990B97FDEF
:10AEA000039695958795959587950EC08091AC06EC
:10AEB000082E000C990B97FD03969595879595950F
:10AEC0008795919581959109809097069090980625
:10AED000A0909906B0909A0681149104A104B1043F
:10AEE000D1F1BC01990F880B990B0E9405E62B014B
:10AEF0003C01C701B601681979098A099B090E94BA
:10AF000003E69B01AC01C301B2010E94FEEA20E00E
:10AF100030E04AE754E40E9464E64B015C0120E023
:10AF200030E040E253E40E9448EC87FF0FC020E08D
:10AF300030E046E952E4C501B4010E9448EC87FDC7
:10AF40000AC02AE030E040E050E009C024E630E0EA
:10AF500040E050E004C021E030E040E050E0C0922A
:10AF60009706D0929806E0929906F0929A0604C04D
:10AF700021E030E040E050E0A091AC060A2E000C49
:10AF8000BB0B0E940CEA24E030E040E050E00E945D
:10AF9000E6E98091760690917706A0917806B091C7
:10AFA0007906820F931FA41FB51F80937606909396
:10AFB0007706A0937806B09379061092AC06D70175
:10AFC000C6018856954CAF4FBF4F8093A206909311
:10AFD000A306A093A406B093A50682E08093400246
:10AFE00080910D0290910E02845C964441F4809110
:10AFF0001002882309F4E5C08150809310022FB716
:10B00000F8948091920690919306A0919406B09145
:10B0100095062FBF3AE0B695A795979587953A95EF
:10B02000D1F7009741E0A407B10520F08FEF9FEF23
:10B03000A0E0B0E09695879520914002211105C0CF
:10B0400030919C063111E9C053C0009741F0409106
:10B05000A0065091A1064817590708F049C08091F1
:10B060009C06811111C0223050F0243028F0243089
:10B0700031F41092400203C081E0809340020E94AC
:10B08000B18681E080939C0684E00E94DCCF81E061
:10B090008093BF0FE0910D02F0910E02199510926E
:10B0A0009D0680919C06882351F00E94F5A591E0B1
:10B0B000811101C090E090939C06911192C0809004
:10B0C000A0069090A106A12CB12C41D8DC01CB01A7
:10B0D0008C199D09AE09BF0988169906AA06BB06F8
:10B0E00038F435D86C197D097093A1066093A006D9
:10B0F00080910D0290910E02845C964421F0809123
:10B100009606882379F088E9C80E8AE3D81EE11CE8
:10B11000F11CC092A206D092A306E092A406F0927F
:10B12000A5060FC08091A2069091A306A091A40647
:10B13000B091A506C81AD90AEA0AFB0AF7FE0E94CE
:10B14000244C80919C0681116CC08091400281301A
:10B1500049F008F466C0843008F063C081E0809351
:10B1600040025FC0109240025CC024E01202F00175
:10B170001124EC5FFC4F20E030E040E752E46081B6
:10B180007181828193810E94FEEAC12C7B018C0136
:10B1900028EC34E044EC54E060EC74E08CEB94E098
:10B1A0000E94FBBC8FEF80930F02CECD10922D102A
:10B1B00010922E10823009F421CE60E082E29DE0F0
:10B1C0001CCE8CE0809310028091A0069091A10685
:10B1D00001979093A1068093A00681E0809340029E
:10B1E0000ECF8090A0069090A106A12CB12C0E94B9
:10B1F000A750DC01CB018C199D09AE09BF09881647
:10B200009906AA06BB0668F40E94A7506C197D092E
:10B210007093A1066093A00604C0009709F434CF90
:10B2200016CF0F900F900F900F90DF91CF911F913D
:10B230000F91FF90EF90DF90CF90BF90AF909F90D5
:10B240008F907F906F905F904F9008950E94F6CFFF
:10B250003E98469A3C98449A3A98429AEAE0F1E03D
:10B2600080818E7F80839FB7F894EBE0F1E080814E
:10B27000816080839FBF82E08093AA06B6DC109233
:10B28000AC060895CF93DF931F921F92CDB7DEB720
:10B2900089839A830E94044C40E050E0BA0189817E
:10B2A0009A810F900F90DF91CF910C948ACF2F92BB
:10B2B0003F924F925F926F927F928F929F92AF9246
:10B2C000BF92CF92DF92EF92FF92CF93DF9300D0A5
:10B2D0001F92CDB7DEB76090880670908906809087
:10B2E0005F0490906004A0906104B0906204B30188
:10B2F000072C000C880B990B0E9405E6A501940110
:10B300000E9421EA6B017C016093DD0B7093DE0BE0
:10B310008093DF0B9093E00B20ED3CEC4CE45DE37D
:10B3200060912C0270912D0280912E0290912F023B
:10B330000E9464E61B012C012091D90B3091DA0B9D
:10B340004091DB0B5091DC0BC501B4010E9421EA56
:10B350009B01AC01C201B1010E9464E61B012C01FA
:10B3600023E333E343E75FE36091D50B7091D60BA2
:10B370008091D70B9091D80B0E9464E69B01AC01A1
:10B38000C201B1010E9422EA69837A838B839C8384
:10B390006093D50B7093D60B8093D70B9093D80BFB
:10B3A0008092D90B9092DA0BA092DB0BB092DC0B5F
:10B3B00020E030E040E251E4C701B6010E9448ECD1
:10B3C000181624F481E08093D40B89C020E030E08B
:10B3D00040E251ECC701B6010E94FFE587FD02C0C3
:10B3E000672821F481E08093D40B9DC08091D40B19
:10B3F000882351F01092D00B1092D10B1092D20BE7
:10B400001092D30B1092D40B209128023091290274
:10B4100040912A0250912B02C701B6010E9464E6B6
:10B420002B013C016093CC0B7093CD0B8093CE0B22
:10B430009093CF0B2091D00B3091D10B4091D20B38
:10B440005091D30BC701B6010E9422EA4B015C0167
:10B450006093D00B7093D10B8093D20B9093D30B4E
:10B4600020913002309131024091320250913302EA
:10B470000E9464E69B01AC016093C80B7093C90BFA
:10B480008093CA0B9093CB0BC301B2010E9422EAB6
:10B4900029813A814B815C810E9421EA2B013C0188
:10B4A00020E030E04FE753E40E9448EC20E030E039
:10B4B000A9011816DCF4C701B6010E9448EC181661
:10B4C00074F4A7019601C501B4010E9421EA6093BA
:10B4D000D00B7093D10B8093D20B9093D30B412C54
:10B4E000512C8FE7682E83E4782E20C0C301B2016F
:10B4F0000E94FFE587FF1AC020E030E0A901C701E4
:10B50000B6010E94FFE587FF0EC0A7019601C501A5
:10B51000B4010E9421EA6093D00B7093D10B809309
:10B52000D20B9093D30B412C512C3201C301B201A9
:10B530000F900F900F900F90DF91CF91FF90EF90B1
:10B54000DF90CF90BF90AF909F908F907F906F9043
:10B550005F904F903F902F90089560916304709199
:10B56000640480916504909166040E9466EBCB01AF
:10B5700008952F923F924F925F926F927F928F9297
:10B580009F92AF92BF92CF92DF92EF92FF920F9372
:10B590001F93CF93DF93EC014EED5DE281E090E0ED
:10B5A000FA0125913491C217D3070CF05DC09C01BC
:10B5B00021503109220F331F220F331FD901A4520A
:10B5C000B24DFD01659174912652324DF901A5905D
:10B5D000B490FC01EE0FFF1FEE0FFF1FE452F24D7F
:10B5E000E590F490FD01C590D490FA010591149175
:10B5F000F90125903490072E000C880B990B0E94BE
:10B6000005E62B013C01CA19DB09BE01DD0F880BE1
:10B61000990B0E9405E64B015C01B7016C197D098D
:10B62000072E000C880B990B0E9405E69B01AC01CC
:10B63000C501B4010E9464E66B017C01B801621986
:10B640007309072E000C880B990B0E9405E69B01DD
:10B65000AC01C701B6010E94FEEA9B01AC01C30127
:10B66000B2010E9422EA11C001964C5F5F4F803404
:10B67000910509F095CFE8EDFEE265917491072EF2
:10B68000000C880B990B0E9405E6DF91CF911F916A
:10B690000F91FF90EF90DF90CF90BF90AF909F9071
:10B6A0008F907F906F905F904F903F902F90089574
:10B6B000CF92DF92EF92FF920F931F93CF93DF937E
:10B6C0001F921F92CDB7DEB77C018A0180911602CE
:10B6D000882309F443C0E7E7F6E284916F019FEF06
:10B6E000C91AD90A882341F069837A830E94C08EDF
:10B6F000F60169817A81F1CFFB0184916F019FEF9F
:10B70000C91AD90A882321F00E94C08EF601F5CF0C
:10B71000E8E8FFE184916F019FEFC91AD90A8823F5
:10B7200021F00E94C08EF601F5CFF7FC0AC0B701E8
:10B73000FF0C880B990B0E942D8F8AE00E94C08E0F
:10B740000DC0E3E8FFE184917F019FEFE91AF90A58
:10B75000882321F00E94C08EF701F5CF8091C70B9E
:10B76000811108C01092160281E08093C70BC801B6
:10B770000E9415920F900F90DF91CF911F910F9122
:10B78000FF90EF90DF90CF900C9446CE4F925F9257
:10B790006F927F928F929F92AF92BF92CF92DF92E1
:10B7A000EF92FF920F931F9380912D1381110FC081
:10B7B0001F910F91FF90EF90DF90CF90BF90AF90CF
:10B7C0009F908F907F906F905F904F9008950E9410
:10B7D0006DCE0E94A7502B013C01609188067091AC
:10B7E0008906072E000C880B990B0E9405E6209114
:10B7F0005F0430916004409161045091620412E151
:10B80000812E912C08E2A02EB12CC12CD12C7B01D1
:10B810008C016DEE7BE08BEE9BE00E94F3CC80E030
:10B8200090E045DD4B015C01C0905F04D090600466
:10B83000E0906104F09062046091AA047091AB04FE
:10B84000072E000C880B990B0E9405E69B01AC01AA
:10B85000C701B6010E9448EC1816CCF460910902A9
:10B8600070910A02072E000C880B990B0E9405E6C6
:10B870009B01AC01C701B6010E94FFE587FF07C02D
:10B88000C501B4010E9466EB7595679501C060E043
:10B8900060932F138091211390912213A091231371
:10B8A000B09124130097A105B105A9F0A30192015D
:10B8B000281B390B4A0B5B0B57FD0DC00E9463CB55
:10B8C0002091251330912613821793070CF4A8C0FA
:10B8D00080E00E9413CE8091271390912813A091AD
:10B8E0002913B0912A130097A105B10599F0A3017E
:10B8F0009201281B390B4A0B5B0B57FD0BC02DDE49
:10B9000020912B1330912C13821793070CF480C0D5
:10B910000E94E0CD8091E70B9091E80BA091E90B9C
:10B92000B091EA0BA3019201281B390B4A0B5B0B68
:10B9300057FD3ECF38E8430E33E1531E611C711CA6
:10B940004092E70B5092E80B6092E90B7092EA0B81
:10B9500060918C0670918D06072E000C880B990B58
:10B960000E9405E6209163043091640440916504CF
:10B9700050916604EFE08E2E912CFCE3AF2EB12C9B
:10B98000CC24CA94DC2C7B018C0161EE7BE085EE3B
:10B990009BE00E94F3CCC0906304D0906404E090DC
:10B9A0006504F090660420E030E040EA50E4C7010E
:10B9B000B6010E9448EC87FD20C020E030E046E15F
:10B9C00053E4C701B6010E94FFE51816B4F0609178
:10B9D0008C0670918D06072E000C880B990B0E9427
:10B9E00005E69B01AC01C701B6010E94FFE587FD9A
:10B9F0001FC080E080932E13DBCE10922E139FB7D2
:10BA0000F894809102018F7D809302019FBFD0CE78
:10BA100046EA5FE165EB7FE18FEF9FEF49DE7ACF8A
:10BA200044EC5FE163ED7FE180E090E041DE53CFE5
:10BA30008FE7E0CF880F991F880F991FFC01EF5601
:10BA4000F44F4081518162817381FC01E052FB4FD0
:10BA50004083518362837383E0918F0BF091900B4D
:10BA600082899389A489B5898093C30B9093C40B71
:10BA7000A093C50BB093C60B0895CF93DF932FB758
:10BA8000F894EC01CC0FDD1FCC0FDD1FFE01EF564B
:10BA9000F44F60817181828193812FBF0E9405E6FE
:10BAA000C053DB4F288139814A815B810E9464E663
:10BAB000DF91CF9108959091FD0F8091FE0F98171F
:10BAC00019F00E947D92F7CF089580918C0B80FF32
:10BAD00003C0899A8FEF02C0899881E08093110298
:10BAE00080918C0B81FF03C08F988FEF02C08F9ADB
:10BAF00081E08093120280918C0B9FB782FF09C076
:10BB0000F89480910B01826080930B019FBF8FEFAF
:10BB100008C0F89480910B018D7F80930B019FBF2B
:10BB200081E08093130280918C0B83FF03C01698F1
:10BB30008FEF02C0169A81E08093140208959091CD
:10BB4000FD0F8091FE0F981731F08091FE0F8F5FEF
:10BB50008F708093FE0F08951F920F920FB60F9271
:10BB600011240BB60F92BF92CF92DF92EF92FF9209
:10BB70000F931F932F933F934F935F936F937F93F5
:10BB80008F939F93AF93BF93EF93FF93CF93DF93E5
:10BB900000D01F92CDB7DEB780916E008B7F80936F
:10BBA0006E0080916F008D7F80936F007894C090BD
:10BBB000BF0BD090C00BE090C10BF090C20BC11432
:10BBC000D104E104F10409F442C080910B02811117
:10BBD00004C08091AF048823D1F10E947671F9EB03
:10BBE000CF16FBE0DF06E104F10488F008EBC01A91
:10BBF0000BE0D00AE108F108C092BF0BD092C00B55
:10BC0000E092C10BF092C20B88EB9BE009C0C60129
:10BC10001092BF0B1092C00B1092C10B1092C20B6E
:10BC2000909389008093880020918800309189004A
:10BC3000809184009091850040962817390708F07C
:10BC40006EC0809184009091850040961FC08091C5
:10BC50008D0B90918E0B009709F494C08C010150CC
:10BC6000110910938E0B00938D0B1092900B109274
:10BC70008F0B65DF012B41F487E79FE19093520C16
:10BC80008093510C0E94FC7088EC90E090938900A6
:10BC90008093880044C0C8010E94E68B24E630E00F
:10BCA00080910B02882309F4B6C4C901293BBBE08B
:10BCB0003B0708F0EAC59093890080938800809143
:10BCC000B10B9091B20BA091B30BB091B40B820F5A
:10BCD000931FA11DB11D8093B10B9093B20BA09344
:10BCE000B30BB093B40B2091880030918900809100
:10BCF00084009091850040962817390748F4809178
:10BD000084009091850040969093890080938800EC
:10BD1000BB2029F01092900B10928F0B10DFF8943B
:10BD200080913013882321F080916E008B7F03C0B7
:10BD300080916E00846080936E0080916F008260BD
:10BD400080936F000F900F900F900F90DF91CF9125
:10BD5000FF91EF91BF91AF919F918F917F916F91E3
:10BD60005F914F913F912F911F910F91FF90EF9015
:10BD7000DF90CF90BF900F900BBE0F900FBE0F9033
:10BD80001F901895C0908F0BD090900BC114D104C8
:10BD900009F0ADC19091FD0F8091FE0F981749F108
:10BDA0009091FE0F1DE4919F900111242454394F6E
:10BDB0008091920690919306A0919406B091950679
:10BDC000F901E75BFF4F4081518162817381841BE0
:10BDD000950BA60BB70B8093920690939306A093B6
:10BDE0009406B0939506D9018C9188608C93690173
:10BDF0000BC08FB7F894109292061092930610928F
:10BE00009406109295068FBFD092900BC0928F0B24
:10BE1000C114D10409F468C1F60152A180918C0BC0
:10BE2000418158130AC0242F30E080911502082E5A
:10BE3000000C990B2817390729F050938C0B40936D
:10BE4000150243DE1092BB0B1092BC0B1092BD0B7F
:10BE50001092BE0BD601D7968D919C91D8978134C4
:10BE6000BCE99B0728F48132EEE49E0748F002C04B
:10BE700080E49CE9969587959695879524E007C080
:10BE80008131F7E29F0730F09695879522E0209365
:10BE9000BA0B08C021E02093BA0B8032910510F450
:10BEA00080E290E08C0100521109011528E0120790
:10BEB000D8F0E12FFF27EE0FFF1FEE0FFF1FCF017E
:10BEC0008958944EFC01329645915491AA27059FBA
:10BED0009001049F210D3A1F06942A1F3A1F112436
:10BEE000FC01859194911CC09801369527952C7F73
:10BEF0002958384EF90185919491F901329665914E
:10BF00007491A80147705527649F9001659F300D7B
:10BF1000749F300D112443E0369527954A95E1F73B
:10BF2000821B930B8436910588F48CEDE82E83E018
:10BF3000F82ED7018D917D01882319F00E94C08EC3
:10BF4000F8CFC8010E94E68B84E690E09093B90B8D
:10BF50008093B80B8091BA0B8093B70BF60183AD39
:10BF600094AD9093B60B8093B50B8134FCE99F0799
:10BF700028F481320EE4900748F002C080E49CE986
:10BF8000969587959695879524E007C0813117E2AD
:10BF9000910730F09695879522E02093BA0B08C060
:10BFA00021E02093BA0B8032910510F480E290E0FA
:10BFB0008C0100521109011528E01207D8F0E12F79
:10BFC000FF27EE0FFF1FEE0FFF1FCF018958944E82
:10BFD000FC01329645915491AA27059F9001049F38
:10BFE000210D3A1F06942A1F3A1F1124FC01859146
:10BFF00094911CC09801369527952C7F2958384E6E
:10C00000F90185919491F901329665917491A80195
:10C0100047705527649F9001659F300D749F300DC8
:10C02000112473E0369527957A95E1F7821B930BDF
:10C030008436910588F45CEDE52E53E0F52ED701AA
:10C040008D917D01882319F00E94C08EF8CFC80120
:10C050000E94E68B84E690E0AC0160E070E04093E3
:10C06000B10B5093B20B6093B30B7093B40B9093DE
:10C07000890080938800F60182899389A489B58913
:10C08000B695A79597958795B095A095909581952C
:10C090009F4FAF4FBF4F8093AD0B9093AE0BA093CC
:10C0A000AF0BB093B00B8093A90B9093AA0BA09306
:10C0B000AB0BB093AC0B8093A50B9093A60BA09306
:10C0C000A70BB093A80B8093A10B9093A20BA09306
:10C0D000A30BB093A40B1092C30B1092C40B10923D
:10C0E000C50B1092C60B03C080ED97E0CFCD8091B9
:10C0F0000B028111C7C38091AF048111C3C320918A
:10C10000BA0B222309F4AFC1E0918F0BF091900B91
:10C110004091A10B5091A20B6091A30B7091A40BC5
:10C1200082819381A481B581840F951FA61FB71FBB
:10C130008093A10B9093A20BA093A30BB093A40B9D
:10C14000181619061A061B060CF4889AE0918F0B34
:10C15000F091900B4091A50B5091A60B6091A70B0D
:10C160007091A80B86819781A085B185840F951F5A
:10C17000A61FB71F8093A50B9093A60BA093A70BA8
:10C18000B093A80B181619061A061B060CF48E9A03
:10C19000E0918F0BF091900B4091A90B5091AA0B5D
:10C1A0006091AB0B7091AC0B82859385A485B585AE
:10C1B000840F951FA61FB71F8093A90B9093AA0BFE
:10C1C000A093AB0BB093AC0B181619061A061B06FE
:10C1D00044F49FB7F89480910B01886080930B0121
:10C1E0009FBFE0918F0BF091900B4091AD0B509160
:10C1F000AE0B6091AF0B7091B00B86859785A089CF
:10C20000B189840F951FA61FB71F8093AD0B909324
:10C21000AE0BA093AF0BB093B00B181619061A060D
:10C220001B060CF4149A8091A10B9091A20BA09183
:10C23000A30BB091A40B181619061A061B0684F559
:10C24000E0918F0BF091900B428953896489758935
:10C25000841B950BA60BB70B8093A10B9093A20B9D
:10C26000A093A30BB093A40B809111024091910B6A
:10C270005091920B6091930B7091940B082E000CCF
:10C28000990BAA0BBB0B840F951FA61FB71F80939A
:10C29000910B9093920BA093930BB093940B88986F
:10C2A0008091A50B9091A60BA091A70BB091A80B24
:10C2B000181619061A061B0684F5E0918F0BF091EB
:10C2C000900B4289538964897589841B950BA60B51
:10C2D000B70B8093A50B9093A60BA093A70BB093DD
:10C2E000A80B809112024091950B5091960B609192
:10C2F000970B7091980B082E000C990BAA0BBB0B97
:10C30000840F951FA61FB71F8093950B9093960BD4
:10C31000A093970BB093980B8E988091A90B909156
:10C32000AA0BA091AB0BB091AC0B181619061A060C
:10C330001B06BCF5E0918F0BF091900B428953895D
:10C3400064897589841B950BA60BB70B8093A90B89
:10C350009093AA0BA093AB0BB093AC0B80911302FC
:10C360004091990B50919A0B60919B0B70919C0B93
:10C37000082E000C990BAA0BBB0B840F951FA61F50
:10C38000B71F8093990B90939A0BA0939B0BB0933C
:10C390009C0B9FB7F89480910B01877F80930B01D2
:10C3A0009FBF8091AD0B9091AE0BA091AF0BB09160
:10C3B000B00B181619061A061B0684F5E0918F0BB0
:10C3C000F091900B4289538964897589841B950B80
:10C3D000A60BB70B8093AD0B9093AE0BA093AF0B56
:10C3E000B093B00B8091140240919D0B50919E0B25
:10C3F00060919F0B7091A00B082E000C990BAA0B5B
:10C40000BB0B840F951FA61FB71F80939D0B9093A6
:10C410009E0BA0939F0BB093A00B14988091C30B1D
:10C420009091C40BA091C50BB091C60B0196A11DB4
:10C43000B11D8093C30B9093C40BA093C50BB09315
:10C44000C60B2150E0918F0BF091900B42895389DC
:10C450006489758984179507A607B70708F451CE34
:10C46000BB24B39401C0B12C4091C30B5091C40BB9
:10C470006091C50B7091C60BE0908F0BF090900B04
:10C48000F70186899789A08DB18D84179507A60736
:10C49000B70708F4C6C04091B10B5091B20B609140
:10C4A000B30B7091B40B068D178D20A131A1AA2773
:10C4B000419FB12D529FC001629F900D619F800DE1
:10C4C000911D429FB00D811D9A1F519FB00D811D7E
:10C4D0009A1F609FB00D811D9A1F509FB10D8A1F3A
:10C4E0009A1FB6958A1F9A1F349F800D911D359F04
:10C4F000900D112423AD34AD820F931F9093B60B92
:10C500008093B50B47A950AD61AD72ADA0E0B0E02E
:10C51000481759076A077B0720F45093B60B4093DE
:10C52000B50B8091B50B9091B60B8134BCE99B079C
:10C5300028F48132EEE49E0748F002C080E49CE9D2
:10C54000969587959695879524E007C08131F7E207
:10C550009F0730F09695879522E02093BA0B08C08C
:10C5600021E02093BA0B8032910510F480E290E034
:10C570008C0100521109011528E01207E8F0E12FA3
:10C58000FF27EE0FFF1FEE0FFF1FCF018958944EBC
:10C59000FC01329625913491AA27039FA001029FA6
:10C5A000410D5A1F06944A1F5A1F1124FC01259160
:10C5B0003491241B350B1EC0A801569547954C7F1E
:10C5C0004958584EFA0125913491FA0132966591F5
:10C5D0007491A80147705527649FC001659F900D15
:10C5E000749F900D1124B3E096958795BA95E1F765
:10C5F000281B390B2436310508F052CBFCEDEF2E09
:10C60000F3E0FF2ED7018D917D01882309F443CB00
:10C610000E94C08EF7CF8091AF04811146CBC90133
:10C620004ACB4091C30B5091C40B6091C50B7091E4
:10C63000C60BF701828D938DA48DB58D8417950758
:10C64000A607B70708F0EBC00091BB0B1091BC0B1D
:10C650002091BD0B3091BE0B09831A832B833C8341
:10C66000468D578D60A171A1AA27059FB12D169FF8
:10C670006001269FD00C259FC00CD11C069FB00DD9
:10C68000C11CDA1E159FB00DC11CDA1E249FB00D0F
:10C69000C11CDA1E149FB10DCA1EDA1EB695CA1E41
:10C6A000DA1E709FC00CD11C719FD00C1124809198
:10C6B000B50B9091B60BFF96C816D90680F48C196D
:10C6C0009D0940815181628173816C01E12CF12CC3
:10C6D000C416D506E606F70620F4CA0102C080811A
:10C6E000918181341CE9910728F481322EE492076C
:10C6F00048F002C080E49CE99695879596958795C9
:10C7000024E007C0813137E2930730F09695879592
:10C7100022E02093BA0B08C021E02093BA0B8032AC
:10C72000910510F480E290E08C010052110901158E
:10C7300048E01407E8F0E12FFF27EE0FFF1FEE0F90
:10C74000FF1FCF018958944EFC01329625913491F8
:10C75000AA27039FA001029F410D5A1F06944A1F5A
:10C760005A1F1124FC0125913491241B350B1EC046
:10C77000C801969587958C7F8958984EFC01259124
:10C780003491FC01329665917491A8014770552748
:10C79000649FC001659F900D749F900D112443E02C
:10C7A000969587954A95E1F7281B390B2436310574
:10C7B00088F48CEDE82E83E0F82ED7018D917D0171
:10C7C000882319F00E94C08EF8CFC8010E94E68B22
:10C7D00024E630E080910B02811104C08091AF0407
:10C7E000882339F0C901293BBBE03B0708F068C04A
:10C7F00001C0C901909389008093880089819A8142
:10C80000AB81BC81820F931FA11DB11D8093BB0B17
:10C810009093BC0BA093BD0BB093BE0B64CA209148
:10C82000B80B3091B90B80910B02811104C080913B
:10C83000AF048823F1F0293BEBE03E07D0F0C901BB
:10C8400068EB7BE00E94E6EC883E43E0940708F04A
:10C8500052C08854944FA901481B590B60E070E006
:10C860004093BF0B5093C00B6093C10B7093C20BEE
:10C870009C0130938900209388008091B70B8093AE
:10C88000BA0B31CA0E9476713ACC68EB7BE00E9409
:10C89000E6EC883E03E0900780F48854944FA901A9
:10C8A000481B590B60E070E04093BF0B5093C00BE6
:10C8B0006093C10B7093C20BFEC988EB9BE0EFCF76
:10C8C00068EB7BE00E94E6EC883E13E0910780F481
:10C8D0008854944FA901481B590B60E070E04093C5
:10C8E000BF0B5093C00B6093C10B7093C20B82CFF0
:10C8F00088EB9BE0EFCF88EB9BE0ADCFCF92DF9250
:10C90000EF92FF92CF93DF936A017B01FC01849148
:10C91000EF012196882321F00E94C08EFE01F7CFFF
:10C920004AE0C701B601DF91CF91FF90EF90DF9011
:10C93000CF900C94C78ECF92DF92EF92FF92CF935D
:10C94000DF936A017B01FC018491EF01219688232A
:10C9500021F00E94C08EFE01F7CF42E0C701B60170
:10C96000DF91CF91FF90EF90DF90CF900C94478FA5
:10C97000CF92DF92EF92FF92CF93DF936A017B0118
:10C98000FC018491EF012196882321F00E94C08E42
:10C99000FE01F7CF42E0C701B601DF91CF91FF90D2
:10C9A000EF90DF90CF900C94478F80E090E0A0E272
:10C9B000B1E48093010C9093020CA093030CB0930C
:10C9C000040C40E050E0BA018091060C9091070CF5
:10C9D0000C948ACF80E090E0A0E8BFE38093010C44
:10C9E0009093020CA093030CB093040C40E050E031
:10C9F000BA018091060C9091070C0C948ACF8DECB3
:10CA00009CECACECBDE38093010C9093020CA093E2
:10CA1000030CB093040C40E050E0BA018091060C86
:10CA20009091070C0C948ACFCF92DF92EF92FF92F5
:10CA3000CF93C82F0E94A7506B017C0124EA30E7F6
:10CA40004DE75FE36091010C7091020C8091030C43
:10CA50009091040C0E94FFE587FD05C046E950E077
:10CA600060E070E003C040E050E0BA01C40ED51EA3
:10CA7000E61EF71EC0928E06D0928F06E0929006B8
:10CA8000F0929106C0930F02CF91FF90EF90DF904C
:10CA9000CF90089580919D0681110C942B4C60914C
:10CAA00076067091770680917806909179066115E7
:10CAB00071058105910571F10E9405E62091010C37
:10CAC0003091020C4091030C5091040C0E9464E6DA
:10CAD0009B01AC016091C8047091C9048091CA04A3
:10CAE0009091CB040E9422EA6093C8047093C90419
:10CAF0008093CA049093CB04109276061092770626
:10CB0000109278061092790683E090E08DDF81E044
:10CB10008093400280914002882349F088EC94E0A1
:10CB20000E942354BC018DE091E20C94D9D0089569
:10CB30002F923F924F925F926F927F928F929F922D
:10CB4000AF92BF92CF92DF92EF92FF920F931F931B
:10CB5000CF93DF9300D000D0CDB7DEB720919D06F4
:10CB60002223D1F026960FB6F894DEBF0FBECDBFBC
:10CB7000DF91CF911F910F91FF90EF90DF90CF90B9
:10CB8000BF90AF909F908F907F906F905F904F90ED
:10CB90003F902F900C942B4C8B011C0180917606BA
:10CBA00090917706A0917806B0917906892B8A2B0F
:10CBB0008B2B09F497C00E946B719801220F331FD1
:10CBC000220F331F3E832D83F901E454FB4F408035
:10CBD00051806280738080912702811115C020E00E
:10CBE00030E04AE754E4C301B2010E9421EA4B015C
:10CBF0005C0120E030E04AE754E4C301B2010E9446
:10CC000022EA6B017C0110C0ED81FE81EF50F44FF0
:10CC100080809180A280B380ED81FE81E55EFD4F32
:10CC2000C080D180E280F380809176069091770673
:10CC3000A0917806B091790689839A83AB83BC83EF
:10CC4000BC01CD010E9405E62091010C3091020C3F
:10CC50004091030C5091040C0E9464E69B01AC01CE
:10CC6000C301B2010E9422EAAD81BE81A454BB4F30
:10CC70003D01FD01608371838283938329813A8121
:10CC80004B815C8157FF0DC0A50194010E94FFE517
:10CC900087FF1BC0D3018D929D92AD92BC921397DA
:10CCA00014C029813A814B815C81232B242B252BB5
:10CCB00061F0A70196010E9448EC181634F4D301E4
:10CCC000CD92DD92ED92FC921397C801ADDE1092E9
:10CCD000760610927706109278061092790681E017
:10CCE0008093400280914002882329F1C801880F77
:10CCF000991F880F991F84549B4F0E942354BC0195
:10CD0000C10126960FB6F894DEBF0FBECDBFDF91EE
:10CD1000CF911F910F91FF90EF90DF90CF90BF9038
:10CD2000AF909F908F907F906F905F904F903F90CB
:10CD30002F900C94D9D026960FB6F894DEBF0FBE74
:10CD4000CDBFDF91CF911F910F91FF90EF90DF90BA
:10CD5000CF90BF90AF909F908F907F906F905F909B
:10CD60004F903F902F90089562E070E086E091E24E
:10CD7000DFCE61E070E08FEF90E2DACE60E070E04D
:10CD800088EF90E2D5CEAF92BF92CF92DF92EF9232
:10CD9000FF920F931F93CF93DF9310929B06809186
:10CDA000760690917706A0917806B0917906813049
:10CDB0009048A105B10540F01092760610927706D2
:10CDC0001092780610927906C09176068091000C38
:10CDD0001816DCF4282F082E000C330B21503109D3
:10CDE0004C2F0C2E000C550B4217530774F0CFEF4D
:10CDF000C80F8C2F90E0A0E0B0E08093760690936F
:10CE00007706A0937806B09379061092BA128091B3
:10CE1000B912C81714F4C093B9128091B912082E30
:10CE2000000C990B04962C2F0C2E000C330B821740
:10CE3000930724F48CEF8C0F8093B912D091B91220
:10CE400010E085EBE82E80E2F82E9FE8C92E90E2F4
:10CE5000D92E2BEDA22E20E2B22ED11117C0809137
:10CE60004002882349F081E0C11180E024E043EFD3
:10CE700050E2612F0E94AE5580919D06882309F4EF
:10CE80007EC0C1117CC00E942B4C75C0D130D9F43A
:10CE900080914002882351F081E0C13009F080E0A8
:10CEA00023E049EE50E2612F0E94AE5580919D062D
:10CEB000882309F464C0C13009F061C08CEC9FE79D
:10CEC0000E94425958C0D230D9F480914002882340
:10CED00051F081E0C23009F080E020E24FED50E2F5
:10CEE000612F0E94AE5580919D06882309F447C0AA
:10CEF000C23009F044C0B092520CA092510C39C01B
:10CF0000D330E9F480914002882351F081E0C330AE
:10CF100009F080E020E24AEC50E2612F0E94AE5519
:10CF200080919D06882359F1C33049F5D092520C67
:10CF3000C092510C0E94FC700E94244C1CC0D43042
:10CF4000F1F480914002882351F081E0C43009F06F
:10CF500080E020E249EB50E2612F0E94AE558091C3
:10CF60009D06882361F0C43051F4F092520CE09297
:10CF7000510C0E94FC708091BA12811180C0809186
:10CF800088069091890620918C0630918D06232B7E
:10CF900011F4892B31F1D53031F58091400288238D
:10CFA00051F081E0C53009F080E020E24CEA50E227
:10CFB000612F0E94AE5580919D06882309F45DC0C3
:10CFC000C53009F05AC010928B0610928A060E9452
:10CFD00046CE0E94244C8091BA12882309F44DC099
:10CFE0004EC005E001C006E0D0131EC08091400293
:10CFF000882349F081E0CD1380E023E040EA50E24D
:10D00000612F0E94AE5580919D06882361F0CD135B
:10D010000AC08EE299E60E9442598091BA128111AB
:10D020002EC00C2F01C00D2F81E0800FD81749F0C2
:10D030001F5FDF5F153009F010CF0E5F0093000C0B
:10D040001EC080914002882349F081E0CD1380E02A
:10D0500023E044E950E2612F0E94AE5580919D0685
:10D06000882331F3CD13E4CF8AE498E60E94425935
:10D070008091BA128823E1F202C006E0D5CFDF9199
:10D08000CF911F910F91FF90EF90DF90CF90BF90C5
:10D09000AF9008951F93CF93DF9310929B068091DA
:10D0A000760690917706A0917806B0917906813046
:10D0B0009048A105B10540F01092760610927706CF
:10D0C0001092780610927906C09176068091FF0B37
:10D0D0001816DCF4282F082E000C330B21503109D0
:10D0E0004C2F0C2E000C550B4217530774F0CFEF4A
:10D0F000C80F8C2F90E0A0E0B0E08093760690936C
:10D100007706A0937806B09379061092BA128091B0
:10D11000B912C81714F4C093B9128091B912082E2D
:10D12000000C990B04962C2F0C2E000C330B82173D
:10D13000930724F48CEF8C0F8093B9121091B912DD
:10D14000D0E0111117C080914002882349F081E09E
:10D15000C11180E024E047E850E26D2F0E94AE55F7
:10D1600080919D06882309F46DC0C1116BC00E9497
:10D170002B4C64C01130F9F480914002882351F0A7
:10D1800081E0C13009F080E020E24BE750E26D2FF2
:10D190000E94AE5580919D06882309F453C0C1308A
:10D1A00009F050C04091380C5091390C6091300C0E
:10D1B0007091310C1CC01230F9F480914002882328
:10D1C00051F081E0C23009F080E020E24BE650E20D
:10D1D0006D2F0E94AE5580919D06882399F1C23033
:10D1E00089F54091380C5091390C6FEF7FEF8091A9
:10D1F000340C9091350C20C0133021F58091400201
:10D20000882351F081E0C33009F080E020E24BE553
:10D2100050E26D2F0E94AE5580919D06882391F0BB
:10D22000C33081F44091380C5091390C6091300C2E
:10D230007091310C80E090E00E94FD4D8091BA1217
:10D24000811108C0DF5F1F5FD53009F07ACF84E01D
:10D250008093FF0BDF91CF911F9108951F93CF9380
:10D26000DF9310929B068091760690917706A091AD
:10D270007806B091790681309048A105B10540F05B
:10D280001092760610927706109278061092790620
:10D29000C09176068091FE0B1816DCF4282F082E1C
:10D2A000000C330B215031094C2F0C2E000C550B68
:10D2B0004217530774F0CFEFC80F8C2F90E0A0E017
:10D2C000B0E08093760690937706A0937806B093AB
:10D2D00079061092BA128091B912C81714F4C0934B
:10D2E000B9128091B912082E000C990B04962C2FBC
:10D2F0000C2E000C330B8217930724F48CEF8C0F49
:10D300008093B9121091B912D0E0111117C0809119
:10D310004002882349F081E0C11180E024E043E528
:10D3200050E26D2F0E94AE5580919D06882309F42E
:10D330006DC0C1116BC00E942B4C64C01130F9F458
:10D3400080914002882351F081E0C13009F080E0F3
:10D3500020E247E450E26D2F0E94AE5580919D0679
:10D36000882309F453C0C13009F050C04091360CF5
:10D370005091370C60912E0C70912F0C1CC0123004
:10D38000F9F480914002882351F081E0C23009F025
:10D3900080E020E247E350E26D2F0E94AE5580917D
:10D3A0009D06882399F1C23089F54091360C509141
:10D3B000370C6FEF7FEF8091320C9091330C20C0CF
:10D3C000133021F580914002882351F081E0C33071
:10D3D00009F080E020E247E250E26D2F0E94AE5556
:10D3E00080919D06882391F0C33081F44091360CE2
:10D3F0005091370C60912E0C70912F0C80E090E0D2
:10D400000E94FD4D8091BA12811108C0DF5F1F5F3D
:10D41000D53009F07ACF84E08093FE0BDF91CF9175
:10D420001F910895FF920F931F93CF93DF93109254
:10D430009B068091760690917706A0917806B09130
:10D44000790681309048A105B10540F0109276062A
:10D45000109277061092780610927906C09176069F
:10D460008091FD0B1816DCF4282F082E000C330BCE
:10D47000215031094C2F0C2E000C550B421753072D
:10D4800074F0CFEFC80F8C2F90E0A0E0B0E0809355
:10D49000760690937706A0937806B093790610925B
:10D4A000BA128091B912C81714F4C093B9128091BE
:10D4B000B912082E000C990B04962C2F0C2E000C80
:10D4C000330B8217930724F48CEF8C0F8093B912DF
:10D4D0001091B912D0E0FF24F394111117C080917C
:10D4E0004002882349F081E0C11180E024E042E25B
:10D4F00050E26D2F0E94AE5580919D06882309F45D
:10D50000E4C0C111E2C00E942B4CDBC0113021F5F8
:10D5100080914002882379F089E192E00E9455557C
:10D520009C0181E0C13009F080E000E04CE150E274
:10D530006D2F0E9464E080919D06882309F4C5C088
:10D54000C13009F0C2C027EE33E04AE050E069E1A3
:10D5500072E086E190E2B3C0123071F58091400232
:10D56000882379F088E896E00E9455559C0181E077
:10D57000C23009F080E000E04FE050E26D2F0E94E1
:10D5800064E080919D06882309F49FC0C23009F0B1
:10D590009CC0F0929B0610929706109298061092EB
:10D5A000990610929A0623E73BE644E051E068E8CA
:10D5B00076E088E090E22FC0133081F58091400240
:10D5C000882379F08CE896E00E9455559C0181E013
:10D5D000C33009F080E000E044E050E26D2F0E948B
:10D5E00064E080919D06882309F46FC0C33009F080
:10D5F0006CC0F0929B0610929706109298061092BB
:10D60000990610929A0626E73BE647E850E06CE858
:10D6100076E080E090E20E94B3D753C0143061F509
:10D6200080914002882379F08AE896E00E9455555F
:10D630009C0181E0C43009F080E000E046EF5FE14A
:10D640006D2F0E9464E080919D068823F1F1C43023
:10D65000E1F5F0929B0610929706109298061092B0
:10D66000990610929A062FEF30E040E050E06AE809
:10D6700076E08CEE9FE123C0153039F580914002B1
:10D68000882379F087E192E00E9455559C0181E062
:10D69000C53009F080E000E047EE5FE16D2F0E94A9
:10D6A00064E080919D06882381F0C53071F427EEF7
:10D6B00033E04AE050E067E172E082EE9FE10E94D1
:10D6C0000EE08091BA12811108C0DF5F1F5FD53074
:10D6D00009F003CF86E08093FD0BDF91CF911F917E
:10D6E0000F91FF90089580E00C9413CE0C94E0CD40
:10D6F000EF92FF921F93CF93DF937C017093070CFF
:10D700006093060C10929B068091760690917706A6
:10D71000A0917806B091790681309048A105B105B5
:10D7200040F01092760610927706109278061092CA
:10D730007906C09176068091050C1816DCF4282F26
:10D74000082E000C330B215031094C2F0C2E000CED
:10D75000550B4217530774F0CFEFC80F8C2F90E092
:10D76000A0E0B0E08093760690937706A0937806C9
:10D77000B09379061092BA128091B912C81714F4B6
:10D78000C093B9122091B912022E000C330B2C5FFA
:10D790003F4F8C2F0C2E000C990B2817390724F4BF
:10D7A0008CEF8C0F8093B9121091B912D0E091E0F8
:10D7B00081E0E816F10459F122E0E216F10409F4DF
:10D7C00048C0E114F10409F066C0111189C0992321
:10D7D000B1F01C16A4F08091760690917706A09186
:10D7E0007806B09179060196A11DB11D8093760649
:10D7F00090937706A0937806B0937906CF5F8091D7
:10D800004002882309F4D7C065E571E265C01111B3
:10D8100067C09923B1F01C16A4F080917606909110
:10D820007706A0917806B09179060196A11DB11DE9
:10D830008093760690937706A0937806B093790646
:10D84000CF5F80914002882309F4B5C06EE471E295
:10D8500043C0111145C09923B1F01C16A4F080916A
:10D86000760690917706A0917806B0917906019698
:10D87000A11DB11D8093760690937706A09378063C
:10D88000B0937906CF5F80914002882309F493C05A
:10D8900067E471E221C0111123C09923B1F01C1675
:10D8A000A4F08091760690917706A0917806B091C9
:10D8B00079060196A11DB11D809376069093770697
:10D8C000A0937806B0937906CF5F809140028823B9
:10D8D00009F471C06EE371E28D2F0E9450D96BC0C4
:10D8E0001130C9F480914002882351F081E0C130A9
:10D8F00009F080E024E044E351E26D2F0E94AE5530
:10D9000080919D06882309F456C0C13009F053C0A8
:10D910000E942B4C4CC01230B9F4809140028823F5
:10D9200051F081E0C23009F080E023E04AE251E2A8
:10D930006D2F0E94AE5580919D068823E1F1C23083
:10D94000D1F585ED94E631C01330B9F480914002F1
:10D95000882351F081E0C33009F080E023E041E208
:10D9600051E26D2F0E94AE5580919D06882319F1DA
:10D97000C33009F58AEE94E618C01430E1F48091C2
:10D980004002882351F081E0C43009F080E023E0B8
:10D9900046E151E26D2F0E94AE5580919D0688238D
:10D9A00051F0C43041F48FEF94E60E9442598091C7
:10D9B000BA12811108C0DF5F1F5F90E0D53009F017
:10D9C000F7CED093050CDF91CF911F91FF90EF9090
:10D9D00008952F923F924F925F926F927F928F9213
:10D9E0009F92AF92BF92CF92DF92EF92FF920F93EE
:10D9F0001F93CF93DF9300D000D0CDB7DEB78C015B
:10DA00000E94A750F801C680D780E084F184C11439
:10DA1000D104E104F10409F0F6C22485222309F4BB
:10DA200060C332852150248721E0230F228745855A
:10DA3000241301C01286F80124E0329FE00DF11D8D
:10DA40001124C684D784E088F188F801C282D38289
:10DA5000E482F582DC01CB018C0D9D1DA11DB11D61
:10DA600086839783A087B18784819581892B09F468
:10DA700038C3FFB7FD83F894F80122803380048116
:10DA8000158180910C02853221F08F3F09F0B8C2D8
:10DA900005C0E1E2FDE024912E83EDC085E2809394
:10DAA0000C02E1E2FDE0E491EF3F09F4A9C2E230AB
:10DAB00009F474C054F5EE2309F453C0E13009F0C1
:10DAC000D9C01092800010928100809181008860FE
:10DAD0008093810080918100816080938100EBE0E0
:10DAE000FBE0E491F0E0EE0FFF1FEE54F54F85915F
:10DAF00094919093150C8093140CE1E5FBE0E49174
:10DB0000E093130C81E08E83B9C0E43009F48EC039
:10DB10000CF468C0E53009F0ADC0109220011092FD
:10DB20002101809121018860809321018091210150
:10DB3000816080932101EBE0FBE0E491F0E0EE0FE7
:10DB4000FF1FEE54F54F8591949190930C0C8093A8
:10DB50000B0CE1E5FBE0E491E0930A0C25E02E8359
:10DB60008DC014BC15BC84B5826084BD85B5816050
:10DB700085BDEBE0FBE0E491F0E0EE0FFF1FEE541B
:10DB8000F54F859194919093180C8093170CE1E5D3
:10DB9000FBE0E491E093160C1E8270C01092B0007E
:10DBA0001092B1008091B00082608093B0008091AB
:10DBB000B10081608093B100EBE0FBE0E491F0E024
:10DBC000EE0FFF1FEE54F54F8591949190937006E0
:10DBD00080936F06E1E5FBE0E491E093710692E04B
:10DBE0009E834CC010929000109291008091910001
:10DBF0008860809391008091910081608093910072
:10DC0000EBE0FBE0E491F0E0EE0FFF1FEE54F54F88
:10DC1000859194919093120C8093110CE1E5FBE0B7
:10DC2000E491E093100CE3E0EE8328C01092A00092
:10DC30001092A1008091A10088608093A100809142
:10DC4000A10081608093A100EBE0FBE0E491F0E0B3
:10DC5000EE0FFF1FEE54F54F8591949190930F0CAA
:10DC600080930E0CE1E5FBE0E491E0930D0CF4E011
:10DC7000FE8304C0EE838E8187FDC2C12101612C29
:10DC8000712C61E085E20E946C4F4801A12CB12CFF
:10DC90008E818D7F09F0BDC060E072E18AE790E07F
:10DCA000A50194010E94E6E929833A834B835C83B2
:10DCB00069017A0191E0C91AD108E108F108EFEF92
:10DCC000CE16D104E104F10409F008F44DC060E47B
:10DCD00072E48FE090E0A50194010E94E6E96901F9
:10DCE0007A01F1E0CF1AD108E108F1082E81223043
:10DCF00001F58FEFC816D104E104F10409F008F42E
:10DD0000EEC160E970ED83E090E0A50194010E940E
:10DD1000E6E969017A0191E0C91AD108E108F10840
:10DD2000EFEFCE16D104E104F10409F0E0F583E051
:10DD300069C0FFEFCF16D104E104F104B9F0B0F0EF
:10DD400068E478EE81E090E0A50194010E94E6E9A4
:10DD500069017A0181E0C81AD108E108F1089E81C1
:10DD6000992309F49AC190C181E001C082E09E81AB
:10DD70009923A1F047C089819A81AB81BC812AE0B7
:10DD8000B595A795979587952A95D1F76C017D0153
:10DD9000E1E0CE1AD108E108F10885E095B5987F59
:10DDA000892B85BDA1C068E478EE81E090E0A501F3
:10DDB00094010E94E6E969017A01F1E0CF1AD108E5
:10DDC000E108F1082FEFC216D104E104F10409F0D3
:10DDD00008F428C164E274EF80E090E0A5019401AA
:10DDE0000E94E6E969017A01E1E0CE1AD108E10872
:10DDF000F108FFEFCF16D104E104F10411F008F0AF
:10DE000013C185E09091B100987F892B8093B10078
:10DE10006BC060E072E18AE790E0A50194010E9486
:10DE2000E6E969017A01E1E0CE1AD108E108F108DA
:10DE3000C114D104F1E0EF06F10488F068E478EE53
:10DE400081E090E0A50194010E94E6E969017A0170
:10DE500081E0C81AD108E108F10883E001C081E03F
:10DE60009E81913071F490918100987F892B8093ED
:10DE70008100452846284728D9F52FEF3FEFA90113
:10DE800068C0EE81E33071F490919100987F892B06
:10DE90008093910045284628472851F52FEF3FEF02
:10DEA000A90179C0FE81F43071F49091A100987FAE
:10DEB000892B8093A100452846284728C9F42FEFD5
:10DEC0003FEFA9017AC02E81253071F49091210194
:10DED000987F892B8093210145284628472841F4C3
:10DEE0002FEF3FEFA9017BC045284628472869F05E
:10DEF0009801220F331FD1010E9412EA28EE33E06D
:10DF000040E050E00E94C4E903C02FEF3FEFA901B9
:10DF10008E81823081F12CF4882361F08130C9F048
:10DF20006FC09E81943009F448C0ACF1953009F47B
:10DF300056C066C0C7BC2093290C30932A0C40936E
:10DF40002B0C50932C0C80916E00826080936E009D
:10DF500057C0D0928900C09288002093250C30933E
:10DF6000260C4093270C5093280C80916F00826000
:10DF700080936F0045C0C092B30020937206309327
:10DF8000730640937406509375068091700082600A
:10DF90008093700035C0D0929900C0929800209371
:10DFA000210C3093220C4093230C5093240C80912D
:10DFB000710082608093710023C0D092A900C0924A
:10DFC000A80020931D0C30931E0C40931F0C5093FF
:10DFD000200C8091720082608093720011C0D092F8
:10DFE0002901C09228012093190C30931A0C4093F8
:10DFF0001B0C50931C0C8091730082608093730003
:10E00000ED81EFBF6EC0DC01CB018C199D09AE091B
:10E01000BF09B7FD66C04098F801168217821086C6
:10E0200011865FC084E0EECE62E17AE780E090E0A6
:10E03000A50194010E94E6E969017A0181E0C81A0C
:10E04000D108E108F1089FEFC916D104E104F104F9
:10E05000C9F0C0F089819A81AB81BC815AE0B59545
:10E06000A795979587955A95D1F76C017D0121E089
:10E07000C21AD108E108F1088E81882309F48DCEF7
:10E0800087E0C0CE86E073CEEFEFCE16D104E10478
:10E09000F10409F048F684E06ACE8FEFC816D10487
:10E0A000E104F104D1F0C8F062E17AE780E090E0A9
:10E0B000A50194010E94E6E969017A01F1E0CF1A15
:10E0C000D108E108F1082FEFC216D104E104F104F0
:10E0D00011F008F050CE84E061CE83E05FCE82E0A4
:10E0E00091CE26960FB6F894DEBF0FBECDBFDF915E
:10E0F000CF911F910F91FF90EF90DF90CF90BF9045
:10E10000AF909F908F907F906F905F904F903F90D7
:10E110002F900895EF92FF920F931F93CF93DF9369
:10E120001F92CDB7DEB7082F162FE7E7F6E28491EE
:10E130007F012FEFE21AF20A882331F099830E94BF
:10E14000C08EF7019981F3CFE02FF92F84917F01E1
:10E150009FEFE91AF90A882321F00E94C08EF70187
:10E16000F5CF609161147091621480916314909165
:10E1700064140E942D8F8AE00E94C08E11110E94AB
:10E1800088D71092200D10921F0D0F90DF91CF9124
:10E190001F910F91FF90EF90089520916A0430E055
:10E1A000F901E453FB4F80832F5F3F4F23703327E8
:10E1B00020936A0480916E068F5F80936E060895A7
:10E1C000CF93FC0180818B33A1F080916E06843067
:10E1D00080F4C62FBF0180916A0420E6829FC001AF
:10E1E000112483519B4F0E946FED8C2FD6DF81E06D
:10E1F00001C080E0CF910895DF92EF92FF920F93DC
:10E200001F93CF93DF93CDB7DEB76E970FB6F89419
:10E21000DEBF0FBECDBF6091510C7091520C6115E5
:10E22000710501F14DE150E0CE0101967C010E94A3
:10E230006FE51E8EF7018F010E191F09D190DD20A9
:10E2400019F09AE0D912F7CFF701E00FF11F108211
:10E2500060E0C701B5DF882329F0C7010E94E6917D
:10E26000811109C081E02091510C3091520C232B77
:10E27000A1F480E012C0DD2049F00F5F1F4F8091B4
:10E28000510C9091520C080F191F02C000E010E0D1
:10E290001093520C0093510CE5CF6E960FB6F89484
:10E2A000DEBF0FBECDBFDF91CF911F910F91FF90C9
:10E2B000EF90DF90089528EC34E044EC54E060ECFB
:10E2C00074E08CEB94E00C9457D4FC01659175914B
:10E2D0008591949108950E94A7506093630C709368
:10E2E000640C8093650C9093660C08950F931F93B4
:10E2F000CF93DF93E0918F0BF091900B428153818C
:10E3000064817581141615061606170604F520910A
:10E310008C0B20FF1CC03CB12091090C3295369526
:10E32000377041E03427832F81702E7F822B8093BA
:10E33000090C9091080C9170892349F08091EC04AC
:10E3400081608093EC0480E090E00E941A5DE0918F
:10E350008F0BF091900B86819781A085B18518165F
:10E3600019061A061B0654F580918C0B81FF26C0F6
:10E37000809103012091090C422F50E0869591E095
:10E380008927082F017010E022273327201B310B2B
:10E390002427352722703327242735272093090C7B
:10E3A0008091080C8270282349F08091EC048260EF
:10E3B0008093EC0481E090E00E941A5DE0918F0B65
:10E3C000F091900B82859385A485B5851816190662
:10E3D0001A061B068CF580918C0B82FF2DC0809154
:10E3E000AF04882349F199B18091090C282F30E0BE
:10E3F000892F86958695869591E089278170C82F0B
:10E4000080E0D82F882799278C1B9D0B8227932784
:10E4100084709927822793278093090C9091080C88
:10E420009470892349F08091EC0484608093EC041B
:10E4300082E090E00E941A5D8091090C8093080CA4
:10E44000DF91CF911F910F910895CF93DF93E3EB6D
:10E45000F3E28491EF012196882321F00E94C08E7F
:10E46000FE01F7CFEBEAF3E28491EF0121968823D6
:10E4700021F00E94C08EFE01F7CF659B03C0C0EF64
:10E48000D3E002C0C5EFD3E08991882319F00E9440
:10E49000C08EFACF8AE00E94C08EE3EAF3E2849154
:10E4A000EF012196882321F00E94C08EFE01F7CF54
:10E4B0008091030181FF03C0C0EFD3E002C0C5EF2C
:10E4C000D3E08991882319F00E94C08EFACF8AE0A8
:10E4D0000E94C08EEBE9F3E28491EF01219688233C
:10E4E00021F00E94C08EFE01F7CF4B9B03C0C0EF0E
:10E4F000D3E002C0C5EFD3E08991882319F00E94D0
:10E50000C08EFACF8AE0DF91CF910C94C08EAF928B
:10E51000BF92CF92DF92EF92FF920F931F93CF9310
:10E52000C82F882319F0E5E8F3E20CC0EEE7FBE220
:10E5300084918F010F5F1F4F8823A9F30E94C08E23
:10E54000F801F6CF84918F010F5F1F4F882321F0D0
:10E550000E94C08EF801F6CF8AE00E94C08EC111E1
:10E560002CC0EEE7FBE284918F010F5F1F4F8823E1
:10E5700021F00E94C08EF801F6CFE2E7F3E2849129
:10E580008F010F5F1F4F882321F00E94C08EF8017A
:10E59000F6CF8091B812882321F08AE00E94C08EC5
:10E5A0003AC0E7E6F3E284918F010F5F1F4F8823A3
:10E5B00091F10E94C08EF801F6CF409189025091EE
:10E5C0008A0260918B0270918C028EE593E20E9428
:10E5D000B8648AE00E94C08E8091B812811127C071
:10E5E000CC2319F0E3E5F3E20CC0EEE7FBE2849103
:10E5F0008F010F5F1F4F8823A9F30E94C08EF8017F
:10E60000F6CF84918F010F5F1F4F882381F00E9406
:10E61000C08EF801F6CFEEE7FBE284918F010F5F29
:10E620001F4F882351F20E94C08EF801F6CFC1110E
:10E6300024C0EEE7FBE284918F010F5F1F4F882318
:10E6400021F00E94C08EF801F6CFE2E4F3E284915B
:10E650008F010F5F1F4F882321F00E94C08EF801A9
:10E66000F6CFEEE7FBE284918F010F5F1F4F882307
:10E6700021F00E94C08EF801F6CF4091BD1250915A
:10E68000BE126091BF127091C0128AE393E20E94A1
:10E69000B8644091C1125091C2126091C31270913E
:10E6A000C41287E393E20E94B8644091C51250916E
:10E6B000C6126091C7127091C81284E393E20E945F
:10E6C000B8644091C9125091CA126091CB127091F6
:10E6D000CC1281E393E20E94B8648AE00E94C08E6B
:10E6E000C11124C0EEE7FBE284918F010F5F1F4F41
:10E6F000882321F00E94C08EF801F6CFE3E1F3E217
:10E7000084918F010F5F1F4F882321F00E94C08EDC
:10E71000F801F6CFEEE7FBE284918F010F5F1F4F08
:10E72000882321F00E94C08EF801F6CF4091ED12AF
:10E730005091EE126091EF127091F0128AE093E224
:10E740000E94B8644091F1125091F2126091F3125C
:10E750007091F41287E093E20E94B8644091F51240
:10E760005091F6126091F7127091F81284E093E2E2
:10E770000E94B8644091F9125091FA126091FB1214
:10E780007091FC1281E093E20E94B8648AE00E94DA
:10E79000C08EC11124C0EEE7FBE284918F010F5FB0
:10E7A0001F4F882321F00E94C08EF801F6CFEFEDB5
:10E7B000F2E284918F010F5F1F4F882321F00E94A6
:10E7C000C08EF801F6CFEEE7FBE284918F010F5F78
:10E7D0001F4F882321F00E94C08EF801F6CF409190
:10E7E000D5125091D6126091D7127091D81286ED41
:10E7F00092E20E947E644091D9125091DA126091A7
:10E80000DB127091DC1283ED92E20E947E644091F3
:10E81000DD125091DE126091DF127091E01280EDF6
:10E8200092E20E947E644091E1125091E212609166
:10E83000E3127091E4128DEC92E20E947E648AE011
:10E840000E94C08EC11124C0EEE7FBE284918F01CB
:10E850000F5F1F4F882321F00E94C08EF801F6CF72
:10E86000E3E8F2E284918F010F5F1F4F882321F0CC
:10E870000E94C08EF801F6CFEEE7FBE284918F0193
:10E880000F5F1F4F882321F00E94C08EF801F6CF42
:10E8900040910D1350910E1360910F13709110134E
:10E8A0008AE792E20E94B8644091D1125091D2124C
:10E8B0006091D3127091D41287E792E20E94B864FB
:10E8C0004091CD125091CE126091CF127091D01222
:10E8D00084E792E20E94B8648AE00E94C08EC1116F
:10E8E00024C0EEE7FBE284918F010F5F1F4F882366
:10E8F00021F00E94C08EF801F6CFE0E0F2E28491B0
:10E900008F010F5F1F4F882321F00E94C08EF801F6
:10E91000F6CFEEE7FBE284918F010F5F1F4F882354
:10E9200021F00E94C08EF801F6CF4091E91250917B
:10E93000EA126091EB127091EC1287EF91E20E9463
:10E94000B8644091E5125091E6126091E71270911F
:10E95000E81284EF91E20E94B8644091171350913D
:10E9600018136091191370911A1381EF91E20E94AC
:10E970007E644091FD125091FE126091FF127091E1
:10E9800000138EEE91E20E94B86440910113509101
:10E99000021360910313709104138BEE91E20E94B5
:10E9A000B86440910513509106136091071370915C
:10E9B000081388EE91E20E94B864409109135091C7
:10E9C0000A1360910B1370910C1385EE91E20E9473
:10E9D000B8648AE00E94C08EC11124C0EEE7FBE259
:10E9E00084918F010F5F1F4F882321F00E94C08EFA
:10E9F000F801F6CFE7EDF1E284918F010F5F1F4F31
:10EA0000882321F00E94C08EF801F6CFEEE7FBE2EA
:10EA100084918F010F5F1F4F882321F00E94C08EC9
:10EA2000F801F6CF4091B0045091B1046091B20466
:10EA30007091B3048EEC91E20E94B8644091B404EA
:10EA40005091B5046091B6047091B7048BEC91E2DB
:10EA50000E94B8644091B8045091B9046091BA041E
:10EA60007091BB0488EC91E20E94B8648AE00E9435
:10EA7000C08ECC2379F082E3A82E8CE0B82E9EE2E3
:10EA8000C92E9CE0D92E26E3E22E2CE0F22E00E0E7
:10EA900010E024C0EEE7FBE284918F010F5F1F4F6F
:10EAA000882321F00E94C08EF801F6CFEBEAF1E254
:10EAB00084918F010F5F1F4F882321F00E94C08E29
:10EAC000F801F6CFEEE7FBE284918F010F5F1F4F55
:10EAD000882389F20E94C08EF801F6CFB80182EA3D
:10EAE00091E2B9D0F501619171915F018FE991E2F5
:10EAF000B2D0F601619171916F018CE991E2ABD0D6
:10EB0000F701619171917F0189E991E2A4D08AE0D6
:10EB10000E94C08E0130110519F001E010E0DECF37
:10EB2000C11124C0EEE7FBE284918F010F5F1F4FFC
:10EB3000882321F00E94C08EF801F6CFEAE8F1E2C6
:10EB400084918F010F5F1F4F882321F00E94C08E98
:10EB5000F801F6CFEEE7FBE284918F010F5F1F4FC4
:10EB6000882321F00E94C08EF801F6CF4091280240
:10EB70005091290260912A0270912B0281E891E262
:10EB80000E94B8642CEA35EC47E25EE36091300203
:10EB90007091310280913202909133020E94FEEA1C
:10EBA000AB01BC018EE791E20E949B642CEA35EC3C
:10EBB00047E25EE360912C0270912D0280912E025B
:10EBC00090912F020E9464E6AB01BC018BE791E2B9
:10EBD0000E949B648AE00E94C08EC11124C0EEE7AF
:10EBE000FBE284918F010F5F1F4F882321F00E9469
:10EBF000C08EF801F6CFE5E6F1E284918F010F5F58
:10EC00001F4F882321F00E94C08EF801F6CFEEE757
:10EC1000FBE284918F010F5F1F4F882321F00E9438
:10EC2000C08EF801F6CF40911113509112136091EC
:10EC30001313709114138CE591E20E94B8648AE07A
:10EC4000CF911F910F91FF90EF90DF90CF90BF90E9
:10EC5000AF900C94C08E0F931F93CF93DF938B01D3
:10EC6000FC018491EF012196882321F00E94C08E3F
:10EC7000FE01F7CFB801110F880B990BDF91CF91EF
:10EC80001F910F910C942D8F0F931F93CF93DF93B0
:10EC90001F921F92CDB7DEB7FC0184918F010F5FE9
:10ECA0001F4F811102C08B0108C069837A830E94C3
:10ECB000C08EF80169817A81F0CFF80181918F01CE
:10ECC000882319F00E94C08EF8CF0F900F90DF912B
:10ECD000CF911F910F910895CF938091960F882324
:10ECE000B9F140918E0F50918F0F6091900F7091FC
:10ECF000910F2EE83DE08091970F9091980F0E9420
:10ED000030D3C82F811102C0C0E023C04091920FC0
:10ED10005091930F6091940F7091950F411551058B
:10ED20006105710591F02EE83DE08091970F90917B
:10ED3000980F0E9430D3882339F31092920F1092CB
:10ED4000930F1092940F1092950F1092960F01C08E
:10ED5000C1E08C2FCF910895CF92DF92EF92FF9276
:10ED6000CF936B017C01C42F80918E0F90918F0FF8
:10ED7000A091900FB091910F8C159D05AE05BF0528
:10ED8000C9F0AADF811102C080E018C02EE83DE082
:10ED9000B701A6018091970F9091980F0E9492D38E
:10EDA000882391F3C0928E0FD0928F0FE092900F34
:10EDB000F092910F81E0C1118093960FCF91FF9057
:10EDC000EF90DF90CF9008954F925F926F927F9275
:10EDD0008F929F92AF92BF92CF92DF92EF92FF926B
:10EDE0000F931F93CF93DF93EC016A017B012801FE
:10EDF0003901423051056105710510F480E064C0AD
:10EE000089859A85AB85BC850196A11DB11D8417A6
:10EE10009507A607B70790F38F89803149F48D2CA9
:10EE20009E2CAF2CBB248B899C89AD89BE890FC0D9
:10EE3000803221F78B889C88AD88BE88DB01CA01AF
:10EE400057E0B695A795979587955A95D1F7880E6F
:10EE5000991EAA1EBB1E41E0C501B4017DDF8823B7
:10EE600069F29F89903161F4DD24EE24FF2496013C
:10EE7000220F331FF901E257F24F5182408211C035
:10EE8000E894C7F8DD24EE24FF249601220F331FF7
:10EE9000220F331FF901E257F24F40825182628202
:10EEA00073829A89923080F04D815E816F8178857E
:10EEB000840E951EA61EB71E8092920F9092930FFD
:10EEC000A092940FB092950FDF91CF911F910F9167
:10EED000FF90EF90DF90CF90BF90AF909F908F907A
:10EEE0007F906F905F904F900895CF92DF92EF9256
:10EEF000FF920F931F93CF93DF93FC01818592853F
:10EF0000A385B4850196A11DB11D84179507A60799
:10EF1000B70710F480E061C08789803149F4BB27CE
:10EF2000A72F962F852FC388D488E588F6880FC031
:10EF3000803281F783899489A589B6896A017B012A
:10EF4000C7E0F694E794D794C794CA95D1F78C0D8F
:10EF50009D1DAE1DBF1DE9016A017B018F0140911E
:10EF60008E0F50918F0F6091900F7091910F8417B9
:10EF70009507A607B70799F4F80187898031B1F49E
:10EF8000B701A601552766277727440F551FFA01B9
:10EF9000E257F24F80819181A0E0B0E019C040E0DB
:10EFA000BC01CD01D9DE8111E7CFB4CFB701A601F5
:10EFB0004F77552766277727440F551F440F551F56
:10EFC000FA01E257F24F80819181A281B381BF7033
:10EFD00088839983AA83BB8381E0DF91CF911F91BE
:10EFE0000F91FF90EF90DF90CF9008954F925F9236
:10EFF0006F927F92AF92BF92CF92DF92EF92FF9289
:10F000000F931F93CF93DF9300D01F92CDB7DEB73E
:10F010008C0149835A836B837C835901C12CD12C89
:10F020007601412C82E0582E612C712C49815A8145
:10F030006B817C819E012F5F3F4FC80156DF882383
:10F0400041F1D301C201F801058404C0880F991F62
:10F05000AA1FBB1F0A94D2F7C80ED91EEA1EFB1EB8
:10F0600049815A816B817C818789803139F481E0C3
:10F07000483F5F4F6105710538F4D8CF81E0483FC4
:10F080005F4F6F4F7F4090F2F501C082D182E282E4
:10F09000F3820F900F900F900F90DF91CF911F91FF
:10F0A0000F91FF90EF90DF90CF90BF90AF907F9047
:10F0B0006F905F904F900895CF93DF93EC018B8119
:10F0C000882331F1898187FF20C061E0CE010E9451
:10F0D00075D1FC01892BE1F08081853EC9F08B81DF
:10F0E000823040F489899A89AB89BC89848F958F55
:10F0F000A68FB78F8D899E89AF89B88D938F828FA8
:10F10000B58BA48B89818F778983DF91CF91E4CDF3
:10F1100081E0888380E0DF91CF9108958F929F9264
:10F12000AF92BF92CF92DF92EF92FF920F931F9315
:10F13000CF93DF93EC018B81811102C080E076C018
:10F1400009891A892B893C8904171507260737076F
:10F15000A8F36A017B01823029F4C886D986EA8641
:10F16000FB860DC0C114D104E104F10451F41C82EA
:10F170001D821E821F82188619861A861B8681E0D0
:10F1800055C088849984AA84BB84E98DFA8D25852D
:10F1900030E0275F3F4FB501A4014150510961099B
:10F1A0007109022E04C076956795579547950A9484
:10F1B000D2F7D701C6010197A109B10904C0B695DC
:10F1C000A795979587952A95D2F784179507A6074F
:10F1D000B70720F089288A288B2849F44D895E8951
:10F1E0006F89788D4C835D836E837F8304C0841B1D
:10F1F000950BA60BB70B4C015D018E010C5F1F4FE9
:10F2000081149104A104B10409F4A7CF4C815D815C
:10F210006E817F819801898D9A8D67DE91E0891AD0
:10F220009108A108B1088111EBCF88CFDF91CF9170
:10F230001F910F91FF90EF90DF90CF90BF90AF9014
:10F240009F908F9008952F923F924F925F926F926E
:10F250007F928F929F92AF92BF92CF92DF92EF9266
:10F26000FF920F931F93CF93DF9300D01F92CDB7E0
:10F27000DEB78C014B011A01DC0113968C911397B8
:10F280008130C1F411968C9181FF14C082FF18C0A7
:10F29000F801418952896389748980859185A285A5
:10F2A000B38584179507A607B70751F0C80136DF65
:10F2B000811106C081E0F80180838FEF9FEF2CC1A0
:10F2C000610185C0D80159968D919C915A97FC0196
:10F2D000248121502A013B0139E0769467945794A8
:10F2E00047943A95D1F7722E74207A01F1E0FF220B
:10F2F000772009F478C080E092E08E199F095601CA
:10F300008C159D0508F45C01D80159962D913C910E
:10F310005A9714968D919D910D90BC91A02D0297B6
:10F32000A109B109F901058404C0880F991FAA1F1A
:10F33000BB1F0A94D2F74685578560897189840F6F
:10F34000951FA61FB71F9C01AD01270D311D411D43
:10F35000511D29013A01A11432E0B30609F089C018
:10F3600080918E0F90918F0FA091900FB091910F7F
:10F3700084159505A605B70569F41092960F8FEFD1
:10F380009FEFDC0180938E0F90938F0FA093900FCF
:10F39000B093910F9401B301A2018091970F9091C6
:10F3A000980F0E9430D3882309F484CFF801808518
:10F3B0009185A285B3858A0D9B1DA11DB11D8087F6
:10F3C0009187A287B3878A0C9B1CCA18DB08D801D7
:10F3D00018964D915D916D917C911B97C114D1044C
:10F3E00009F070CF7AC0E114F10409F084CF1496CB
:10F3F0004D915D916D917C91179741155105610576
:10F40000710559F455968D919D910D90BC91A02D4B
:10F410000097A105B10539F520C09E012F5F3F4F30
:10F4200064DD882309F446CF89819A81AB81BC8150
:10F43000F801218D328DF9012789203139F4883F77
:10F44000FFEF9F07A105B10540F40DC0883F2FEFE6
:10F450009207A2072FE0B20730F0C8010E9491D1B5
:10F46000811149CF27CFF80184839583A683B78381
:10F4700042CFE114F10411F5D80118964D915D9138
:10F480006D917C911B9751968D919D910D90BC91A2
:10F49000A02D481759076A077B0780F01DDC8823D9
:10F4A00009F408CF81E08093960F40928E0F50921E
:10F4B0008F0F6092900F7092910F07C041E0C301CF
:10F4C000B2014ADC882309F4F5CEA501B401C701D5
:10F4D0008257924F0E9434ED69CF51968D919D9144
:10F4E0000D90BC91A02D84179507A607B70740F48F
:10F4F000F801418B528B638B748B8181806881838F
:10F50000D80111968C9183FD02C0C10105C0C801CC
:10F51000D3DD8111FACFCECE0F900F900F900F90C8
:10F52000DF91CF911F910F91FF90EF90DF90CF90DF
:10F53000BF90AF909F908F907F906F905F904F9013
:10F540003F902F900895CF93DF931F92CDB7DEB7F2
:10F55000698341E050E0BE016F5F7F4F049673DE28
:10F560000F90DF91CF9108952F923F924F925F922B
:10F570006F927F928F929F92AF92BF92CF92DF92C3
:10F58000EF92FF920F931F93CF93DF9300D01F92C0
:10F59000CDB7DEB79C838B834B015A01DC011396F8
:10F5A0008C91811103C08FEF9FEFE9C0EB81FC814B
:10F5B000818180FFF8CFAB81BC8151960D911D9167
:10F5C0002D913C91549718964D915D916D917C9140
:10F5D0001B97C501A0E0B0E068017901C41AD50A03
:10F5E000E60AF70AC816D906EA06FB0618F4580117
:10F5F000A41AB50A75018B819C8104969A8389832C
:10F60000612C92E0792EE114F10409F48AC0AB81F7
:10F61000BC8118964D915D916D917C911B976A010B
:10F62000B1E0DB22EB81FC8123811A012B0189E00F
:10F6300056944794379427948A95D1F7818D928D6B
:10F64000223061F4FC01828D938DA48DB58DBC01B7
:10F65000CD01620D731D841D951D49C0DC011496FA
:10F660001C9111501221C114D104F9F411111DC0C3
:10F67000452B462B472B59F4EB81FC8185899689D4
:10F68000A789B08D84839583A683B7830EC0AB8191
:10F69000BC8114964D915D916D917C911797298154
:10F6A0003A8123DC882309F47ECFEB81FC81218D14
:10F6B000328D84819581A681B7810297A109B10914
:10F6C000F901058404C0880F991FAA1FBB1F0A9463
:10F6D000D2F74685578560897189840F951FA61FCB
:10F6E000B71FBC01CD01610F711D811D911D9301DB
:10F6F0002C193D0987012E153F0508F489010115D4
:10F70000F2E01F0779F520918E0F30918F0F409115
:10F71000900F5091910F621773078407950719F4A2
:10F7200021C0C5012CC09401AB01BC018091970F91
:10F730009091980F0E9492D3882309F434CF800EC1
:10F74000911EEB81FC8180859185A285B385800F18
:10F75000911FA11DB11D80879187A287B387E01AF1
:10F76000F10A51CF40E0F8DA882309F41CCFB60142
:10F770006257724FA801C4010E9434EDE0CF0F9090
:10F780000F900F900F90DF91CF911F910F91FF90ED
:10F79000EF90DF90CF90BF90AF909F908F907F9031
:10F7A0006F905F904F903F902F900895DF92EF926F
:10F7B000FF920F931F93CF93DF937C01EB018A019C
:10F7C0008DE0D82E40E250E0BE01C701CDDE803290
:10F7D000910539F021E0892B09F420E0822F8195F1
:10F7E0003EC02881222399F1253E61F32E3251F348
:10F7F0000115110541F13B853F733F3021F54A8DDD
:10F800005B8D452B01F52F713FEF320F3230D8F46D
:10F8100030E021503109D29EC001D39E900D1124B9
:10F82000D801A80FB91FFE0120E0AD01253088F4F2
:10F8300031813D932F5F32962D30C1F7288126FF0D
:10F8400002C0FA0115862B8523FDBCCF08C080E0DD
:10F8500006C02B3010F43481ECCF3681EACFDF9133
:10F86000CF911F910F91FF90EF90DF9008954F92ED
:10F870005F926F927F92AF92BF92CF92DF92EF92A0
:10F88000FF920F931F93CF93DF931F92CDB7DEB7F5
:10F890008C017B015A01D22EDB0159968D919C91EE
:10F8A0005A97F801928F818F40E050E0BA01C7016A
:10F8B00035DCC12CF70180859185A285B38541890E
:10F8C00052896389748984179507A607B70708F0DA
:10F8D00062C025E0B695A795979587952A95D1F7AB
:10F8E000F82FFF707F2ED70113968C91823008F489
:10F8F00063C041E050E0BE016F5F7F4FC70134DE5F
:10F90000019719F4898190E002C08FEF9FEF019673
:10F9100009F452C0F70180859185A285B3854F9681
:10F92000A11DB11D80879187A287B387F0E27F9EDA
:10F93000C0011124BC016257724F61157105E1F1DC
:10F94000DB012C91222319F0253ED1F465C1C110B1
:10F950000EC040918E0F50918F0F6091900F70915B
:10F96000910FF8014487558766877787708AFC0175
:10F97000E257F24F8081882361F0CC24C3949ACF60
:10F980004BE050E0C5010E9427ED892B09F092CF92
:10F9900015C0CC24C3948D2D8274823469F4CC209C
:10F9A00009F489C0D80150967C9061E0C8010E949A
:10F9B00075D1009709F005C180E031C1D7FCFCCFBB
:10F9C000F0E27F9EA00111249A012257324FD90103
:10F9D0001B968C91817121F08D2D827109F067C089
:10F9E00080918E0F90918F0FA091900FB091910FF9
:10F9F000F80184879587A687B787708AFA01E2574E
:10FA0000F24F4489558960E070E0BA0155274427D8
:10FA1000D80155964D935D936D937C935897828D45
:10FA2000938DA0E0B0E0482B592B6A2B7B2BD8019B
:10FA300055964D935D936D937C935897D9011B9682
:10FA40008C91887159F4848D958DA68DB78DF801B0
:10FA5000818B928BA38BB48B81E00FC0803139F501
:10FA600098012F5E3F4FD80159968D919C915A97DE
:10FA7000BDDA8823E1F084E0F80183838D2D8F7057
:10FA8000D80111968C931197F80114821582168271
:10FA9000178218961D921D921D921C921B97D4FEE0
:10FAA000AFC0C8010E944EA88111AAC085CFD8015D
:10FAB00013961C9281CFF7018381823009F47CCFA9
:10FAC00081899289A389B489803E9F4FAF41B10556
:10FAD00008F072CFC7010E9491D1882309F46CCF3E
:10FAE000FBD8882309F468CFD70159962D913C9112
:10FAF0005A9714968D919D910D90BC91A02D0297CF
:10FB0000A109B109F901058404C0880F991FAA1F32
:10FB1000BB1F0A94D2F74684578460887188480EC8
:10FB2000591E6A1E7B1E81E08093960F40928E0FB5
:10FB300050928F0F6092900F7092910F80E092E040
:10FB4000EEE8FDE0DF019C011D9221503040E1F71D
:10FB5000CC24C394D7015996ED91FC915A97848196
:10FB6000C81698F42EE83DE0B301A2014C0D511DDA
:10FB7000611D711D8091970F9091980F0E9430D355
:10FB8000882309F419CFC394E5CF80E092E0A0E088
:10FB9000B0E0058404C0880F991FAA1FBB1F0A94F8
:10FBA000D2F7F7014189528963897489840F951FBF
:10FBB000A61FB71F818B928BA38BB48B8EE89DE021
:10FBC000712C20E2DC011D922A95E9F72BE0F5016A
:10FBD000DC0101900D922A95E1F721E238E2FC0167
:10FBE000318B208B40E058E057874687338B228B40
:10FBF000318F208F578B468B6FD88111E1CEDCCEB1
:10FC0000D5FE08C0F8014189528963897489C80109
:10FC100085DA05C081E003C0C110AFCE9ACE0F9047
:10FC2000DF91CF911F910F91FF90EF90DF90CF90D8
:10FC3000BF90AF907F906F905F904F9008950F931B
:10FC40001F93CF93DF93FC012381222311F080E0E7
:10FC500043C08B01EC01FB018789803131F1803297
:10FC6000B1F783E08B83F801428D538D648D758DE0
:10FC70004D8B5E8B6F8B788F9E012F5E3F4FC8013F
:10FC8000B5D9882321F31A8F098F81E089831C82DB
:10FC90001D821E821F82188619861A861B861C8664
:10FCA0001D861E861F86188A17C082E08B831D8AD8
:10FCB0001E8A1F8A188EFB01808D918DA0E0B0E016
:10FCC00025E0880F991FAA1FBB1F2A95D1F7898BA2
:10FCD0009A8BAB8BBC8BD7CFDF91CF911F910F91BC
:10FCE0000895CF93DF93EB01FC012381211102C022
:10FCF00080E028C02250223020F48FE288831982CD
:10FD000020C060E00E9475D1009791F3FC0190E063
:10FD100080E02EE23081303269F0883029F4DE0153
:10FD2000A90FB11D2C939F5FDE01A90FB11D30817A
:10FD30003C939F5F8F5F31968B3061F7C90FD11D68
:10FD4000188281E0DF91CF910895CF93DF93EC018A
:10FD5000B3D91B82DF91CF9108952F923F924F929A
:10FD60005F926F927F928F929F92AF92BF92CF924B
:10FD7000DF92EF92FF920F931F93CF93DF93CDB754
:10FD8000DEB7C554D1090FB6F894DEBF0FBECDBFA4
:10FD90003C015B018A01322E1C8E1F8E19821C824F
:10FDA000672B11F410E0A7C0FC0183818111FACF09
:10FDB000FA0180818F3261F4CA018C010196F80149
:10FDC00020812F32D1F3F50183818250823010F4EB
:10FDD00075010AC0618D728DCE01019630DF8823D6
:10FDE00009F3CE0101967C016E019CE1C90ED11C84
:10FDF00026014E01E7E38E0E911CFBE0F80D2596DF
:10FE0000FFAF2597CE01019624969FAF8EAF249722
:10FE10002696CFAE26972D2C35C080E2819325966D
:10FE20009FAD25979E13F9CFD80190E027E04A2F88
:10FE30003B2F8D91811128C08FA9803209F4B2CF58
:10FE4000842F932F8C01FC01208101962F32D1F356
:10FE5000222309F44AC021E0A401B701C60107DD4D
:10FE6000882309F49FCFEA14FB0411F0C7016DDF6A
:10FE7000C414D50499F126969FAD2697822D76015C
:10FE8000C92ED82EF401C9CF8F32B1F28E3219F0BB
:10FE9000EDECF3E20AC02A3009F484CF98E02AE0BE
:10FEA000C6CF3196381709F47DCF34913111F9CF8F
:10FEB000291708F477CF813208F474CF8F3709F40B
:10FEC00071CF31E0390FF401E90FF11D9FE9980F6F
:10FED0009A3108F480528083932FA9CF23969FAD47
:10FEE000239724968FAD2497CACF232DA401B70161
:10FEF000C301BDDC182FCE0101960E94DDB3CE01F7
:10FF00004C960E94DDB3812FCB5BDF4F0FB6F89488
:10FF1000DEBF0FBECDBFDF91CF911F910F91FF903C
:10FF2000EF90DF90CF90BF90AF909F908F907F9099
:10FF30006F905F904F903F902F9008952CEA35EC92
:10FF400047E25EE360913C0C70913D0C80913E0C69
:10FF500090913F0C0E94FEEA60932C0270932D0258
:10FF600080932E0290932F0208952CEA35EC47E2FD
:10FF70005EE36091400C7091410C8091420C909135
:10FF8000430C0E9464E660933002709331028093C8
:10FF900032029093330208951F93CF93DF93109210
:10FFA0009B068091760690917706A0917806B09195
:10FFB000790681309048A105B10540F0109276068F
:10FFC000109277061092780610927906C091760604
:10FFD00080913A0C1816DCF4282F082E000C330BF5
:10FFE000215031094C2F0C2E000C550B4217530792
:10FFF00074F0CFEFC80F8C2F90E0A0E0B0E08093BA
:020000021000EC
:10000000760690937706A0937806B09379061092BF
:10001000BA128091B912C81714F4C093B912809122
:10002000B912082E000C990B04962C2F0C2E000CE4
:10003000330B8217930724F48CEF8C0F8093B91243
:100040001091B912D0E0111117C08091400288239D
:1000500049F081E0C11180E024E04BEF53E26D2FC5
:100060000E94AE5580919D06882309F470C0C1118D
:100070006EC00E942B4C67C01130C9F480914002C1
:10008000882351F081E0C13009F080E023E044EFA3
:1000900053E26D2F0E94AE5580919D06882309F48E
:1000A00056C0C13009F053C087E295E84AC012300B
:1000B000B9F480914002882351F081E0C23009F008
:1000C00080E023E04DEE53E26D2F0E94AE5580910B
:1000D0009D068823E1F1C230D1F58DE295E831C06B
:1000E0001330B9F480914002882351F081E0C3308D
:1000F00009F080E023E046EE53E26D2F0E94AE55FA
:1001000080919D06882319F1C33009F583E395E8B2
:1001100018C01430E1F480914002882351F081E04E
:10012000C43009F080E023E04DED53E26D2F0E94D2
:10013000AE5580919D06882351F0C43041F489E387
:1001400095E80E9442598091BA12811107C0DF5F81
:100150001F5FD53009F077CFD0933A0CDF91CF9164
:100160001F9108953F924F925F926F927F928F926C
:100170009F92AF92BF92CF92DF92EF92FF920F9336
:100180001F93CF93DF9310929B06809176069091F8
:100190007706A0917806B091790681309048A10544
:1001A000B10540F01092760610927706109278060C
:1001B00010927906C09176068091440C1816DCF4F2
:1001C000282F082E000C330B215031094C2F0C2EF8
:1001D000000C550B4217530774F0CFEFC80F8C2F4C
:1001E00090E0A0E0B0E08093760690937706A0932D
:1001F0007806B09379061092BA128091B912C81796
:1002000014F4C093B9128091B912082E000C990B06
:1002100004962C2F0C2E000C330B8217930724F41A
:100220008CEF8C0F8093B9123090B912D0E054E665
:10023000452E512C612C712C6DE5C62E6BEAD62E05
:100240007EE9A72E7FE7B72EE5EB8E2EEFE79E2EF9
:10025000311017C080914002882349F081E0C1111C
:1002600080E024E040EF54E26D2F0E94AE55809173
:100270009D06882309F4A7C1C111A5C10E942B4C7A
:100280009EC181E038122EC080914002882379F00F
:1002900088E896E00E9455559C0181E0C13009F044
:1002A00080E000E049EE54E26D2F0E9464E080910E
:1002B0009D06882309F487C1C13009F084C1C09329
:1002C0009B0610929706109298061092990610922B
:1002D0009A0623E73BE644E051E068E876E082EEE8
:1002E00094E231C092E0391231C0809140028823FB
:1002F00079F08CE896E00E9455559C0181E0C2306F
:1003000009F080E000E04EED54E26D2F0E9464E0C1
:1003100080919D06882309F456C1C23009F053C16B
:1003200081E080939B061092970610929806109297
:10033000990610929A0626E73BE647E850E06CE8FB
:1003400076E08AED94E20E94B3D739C1A3E03A1275
:1003500031C080914002882379F08AE896E00E94BB
:1003600055559C0181E0C33009F080E000E040ED8C
:1003700054E26D2F0E9464E080919D06882309F469
:1003800022C1C33009F01FC181E080939B06109207
:100390009706109298061092990610929A062FEFDF
:1003A00030E040E050E06AE876E086EC94E20E94BB
:1003B0000EE005C1B4E03B1229C0809140028823C1
:1003C00099F080912D0C811103C025EB34E202C01D
:1003D00029EB34E281E0C43009F080E001E04DEB2C
:1003E00054E26D2F0E9464E080919D06882309F4F9
:1003F000EAC0C43009F0E7C090912D0C81E0892754
:1004000080932D0C83E080934002D9C025E0321206
:100410003AC080914002882311F181E08F9384E0FB
:100420008F931F921F928CE392E09F938F93A7EA82
:10043000B4E2BF93AF93AEEAB4E2BF93AF93DF935E
:1004400081E0C53009F080E08F930E94D4E08DB741
:100450009EB70C960FB6F8949EBF0FBE8DBF8091CD
:100460009D06882309F4AFC0C53009F0ACC0E12C6B
:10047000F12C02E813E420E030E0A9016CE372E023
:1004800080EA94E23CC096E039123CC08091400280
:10049000882311F181E08F9384E08F931F921F9244
:1004A00088E392E09F938F93A2E9B4E2BF93AF9366
:1004B000A9E9B4E2BF93AF93DF9381E0C63009F0BE
:1004C00080E08F930E94D4E08DB79EB70C960FB654
:1004D000F8949EBF0FBE8DBF80919D06882309F4BE
:1004E00072C0C63009F06FC0E12CF12C02E813E4B1
:1004F00020E030E0A90168E372E08BE894E20E941A
:1005000098DF5DC097E039125EC080914002882379
:1005100079F084E392E00E946B549C0181E0C73043
:1005200009F080E000E043E854E26D2F0E9464E0AF
:1005300080919D06882309F446C0C73009F043C066
:100540000E94044C83E080934002ABE7B4E2B09396
:100550008506A093840684E392E0909383068093BB
:10056000820610927E0610927F06109280061092EC
:10057000810640927A0650927B0660927C067092C9
:100580007D0620E030E048EC52E460913402709146
:10059000350280913602909137020E9464E60E94F3
:1005A0006BEB609376067093770680937806909352
:1005B0007906A4E6BDEAB0930E02A0930D028091E5
:1005C000BA1281110DC12CEA35EC47E25EE360916D
:1005D00030027091310280913202909133020E9478
:1005E000FEEA6093400C7093410C8093420C909310
:1005F000430C2CEA35EC47E25EE360912C027091EB
:100600002D0280912E0290912F020E9464E6609349
:100610003C0C70933D0C80933E0C90933F0CB8E0E3
:100620003B1231C080914002882379F088E292E049
:100630000E9458529C0181E0C83009F080E000E03F
:1006400045E754E26D2F0E9464E080919D06882367
:1006500009F4BEC0C83009F0BBC0E12C18E1F12E8E
:100660000CE116E420E030E040E85FE368E272E08D
:100670008FE694E20E9419DF86E69BEA90930E02D1
:1006800080930D02A1C029E0321233C08091400254
:10069000882379F080E49CE00E9458529C0181E01C
:1006A000C93009F080E000E049E654E26D2F0E9475
:1006B00064E080919D06882309F48AC0C93009F05E
:1006C00087C0E12C18E1F12E0CE116E42AE037EDA9
:1006D00043E25CE360E47CE083E694E20E9419DF9D
:1006E000D0920E02C0920D029092870680928606EA
:1006F0006BC08AE0381233C080914002882379F0C1
:100700008CE39CE00E9458529C0181E0CA3009F0C1
:1007100080E000E04DE554E26D2F0E9464E080919E
:100720009D06882309F454C0CA3009F051C0E12C59
:1007300018E1F12E0CE116E420E030E040E85FE340
:100740006CE37CE087E594E20E9419DFD0920E0210
:10075000C0920D02B0928706A092860635C09BE03B
:10076000391217C080914002882351F081E0CB30CC
:1007700009F080E023E046E454E26D2F0E94AE557C
:1007800080919D06882321F1CB3011F582E89CEB06
:1007900019C0ACE03A121CC080914002882351F08D
:1007A00081E0CC3009F080E023E045E354E26D2F96
:1007B0000E94AE5580919D06882351F0CC3041F4C3
:1007C0008FE79CEB0E9442598091BA12811108C0B8
:1007D000DF5F3394D53009F03BCD8DE08093440C3E
:1007E000DF91CF911F910F91FF90EF90DF90CF900D
:1007F000BF90AF909F908F907F906F905F904F9041
:100800003F9008958F929F92AF92BF92CF92DF92C6
:10081000FF920F931F93CF93DF9300D000D0CDB7FB
:10082000DEB710929B068091760690917706A09194
:100830007806B091790681309048A105B10540F065
:10084000109276061092770610927806109279062A
:100850001091760680913B0C1816DCF4282F082E98
:10086000000C330B21503109412F012E000C550B88
:100870004217530774F01FEF180F812F90E0A0E08C
:10088000B0E08093760690937706A0937806B093B5
:1008900079061092BA128091B912181714F41093B5
:1008A000B9128091B912082E000C990B0496212FD1
:1008B000012E000C330B8217930724F48CEF810F69
:1008C0008093B912F090B91200E083E9A82E82E07B
:1008D000B82E94E6C92ED12C2AEB822E22E0922E3D
:1008E000F11017C080914002882349F081E0111176
:1008F00080E024E040E354E2602F0E94AE558091F6
:100900009D06882309F48AC0111188C00E942B4CCF
:1009100081C081E0F81219C080914002882351F013
:1009200081E0113009F080E023E044E254E2602FDE
:100930000E94AE5580919D06882309F46FC0113046
:1009400009F06CC082EB90E81BC022E0F2121BC0E1
:1009500080914002882351F081E0123009F080E05C
:1009600023E04DE154E2602F0E94AE5580919D0638
:10097000882309F453C0123009F050C088E397EB84
:100980000E94425947C083E0F81217C0809140028C
:10099000882351F081E0133009F080E023E044E146
:1009A00054E2602F0E94AE5580919D068823B1F1DC
:1009B0001330A1F584E690EBE3CF24E0F2122EC0D1
:1009C00080914002882351F081E0143009F080E0EA
:1009D00020E243E054E2602F0E94AE5580919D06D4
:1009E0008823E1F01430D1F40E9442B2BE82AD827D
:1009F000DA82C982BE016B5F7F4FCE0101963DD680
:100A00009C828B82DA82C982BE016D5F7F4FCE01EC
:100A1000019633D68091BA12811107C00F5FF3940B
:100A2000053009F05DCF00933B0C26960FB6F89485
:100A3000DEBF0FBECDBFDF91CF911F910F91FF9011
:100A4000DF90CF90BF90AF909F908F9008956EEB06
:100A500076E680E090E00C94786B69EB76E681E0D6
:100A600090E00C94786B64EB76E682E090E00C9476
:100A7000786B6AE475E683E090E00C94786BAF9253
:100A8000BF92CF92DF92EF92FF920F931F93CF937B
:100A9000DF9310929B064091760650917706609105
:100AA000780670917906413050486105710540F033
:100AB00010927606109277061092780610927906B8
:100AC000C09176069091450C1916DCF4292F092E59
:100AD000000C330B215031094C2F0C2E000C550B00
:100AE0004217530774F0CFEFC90F4C2F50E060E06E
:100AF00070E0409376065093770660937806709383
:100B000079061092BA129091B912C91714F4C093D1
:100B1000B9122091B912022E000C330B2C5F3F4FFB
:100B20004C2F0C2E000C550B2417350724F49CEF8A
:100B30009C0F9093B9121091B912D0E0282F30E099
:100B4000220F331FC901825D934F6C01C9018E5C76
:100B5000934F5C01C9018A5C934F7C01111117C04E
:100B600080914002882349F081E0C11180E024E0B7
:100B700042E255E26D2F0E94AE5580919D0688237A
:100B800009F472C0C11170C00E942B4C69C01130B1
:100B900011F580914002882371F0C7010E945555DC
:100BA0009C0181E0C13009F080E000E048E155E2BD
:100BB0006D2F0E9464E080919D06882309F454C043
:100BC000C13009F051C02FEF30E040E050E0B701F4
:100BD0008EE095E243C0123001F5809140028823F7
:100BE00071F0C5010E9455559C0181E0C23009F0A9
:100BF00080E000E047E055E26D2F0E9464E08091C4
:100C00009D06882389F1C23079F524E031E045E082
:100C100050E0B50180E095E221C0133029F58091C4
:100C20004002882371F0C6010E9455559C0181E065
:100C3000C33009F080E000E04CEF54E26D2F0E94D9
:100C400064E080919D06882379F0C33069F427E839
:100C500030E045E050E0B60188EF94E20E940EE0FB
:100C60008091BA12811108C0DF5F1F5FD53009F093
:100C700075CF84E08093450CDF91CF911F910F9148
:100C8000FF90EF90DF90CF90BF90AF900895EF92DC
:100C9000FF920F931F93CF93DF93CDB7DEB76F977C
:100CA0000FB6F894DEBF0FBECDBF7B0109E710E1A0
:100CB0002BE730E1F8013183208322E030E03093EC
:100CC000B3122093B2129093B5128093B41240E005
:100CD00050E0BA018FE790E10E948E78F8018081A0
:100CE00091812BE1FC013496DE01159601900D9265
:100CF0002A95E1F7FC01828193819C838B838EE2AC
:100D000093E09A838983A701BE016F5F7F4F8FEEC7
:100D100093E00E94E0A8CE0101960E94E3B36F9693
:100D20000FB6F894DEBF0FBECDBFDF91CF911F91FC
:100D30000F91FF90EF90089510922D108091FB116C
:100D4000882319F088EF91E100C80895E0919B0F86
:100D5000F0919C0F0190F081E02D682F8BE99FE0CE
:100D60001994CF93DF938091D80F811107C081E050
:100D70008093D80F8FE99FE00E9432B5C091A10FF8
:100D8000D091A20FE091D00FF091D10F82E0199590
:100D9000E091D00FF091D10F81E0199520E030E083
:100DA00044E1BE018FE99FE00E94B0B422ED3FE034
:100DB00047E1BE018FE99FE00E94B0B4E091D00FFF
:100DC000F091D10F80E0DF91CF9119946F927F92D3
:100DD0008F929F92BF92CF92DF92EF92FF920F93EA
:100DE0001F93CF93DF93CDB7DEB7AD970FB6F894CF
:100DF000DEBF0FBECDBF20912E10222309F4D2C139
:100E0000B62E7C018091FB11882309F49AC04423FB
:100E100009F4A0C180911312882311F1E7E7F6E2EB
:100E200084918F010F5F1F4F882319F0A9D7F80114
:100E3000F7CFE4E3F6E284918F010F5F1F4F882321
:100E400019F09ED7F801F7CF61E070E080E090E004
:100E50000E942D8F8AE094D78BE296E20E94159231
:100E60008FE280931812D12C21E009E112E19FE179
:100E7000C92E8091D011D816B8F4CD9CC001112490
:100E8000B80182569F4E2DA70E94717EC8012DA5E4
:100E90008C010196F8013081332321F02D3811F0B7
:100EA0002F5FF6CFD394E5CF27FD08C0B80188EFB8
:100EB00091E10E94717EEEE7FBE203C0F80110822F
:100EC000FACF84918F010F5F1F4F882319F058D7F5
:100ED000F801F7CFB70182E196E20E944476609173
:100EE0001312FDE86F9FB0011124685E7D4E87E00C
:100EF00096E20E9444764091A9125091AA12609104
:100F0000AB127091AC1281E096E20E947E648AE09E
:100F100037D78091131294E0899FF0011124EC5E81
:100F2000FD4E4091A9125091AA126091AB1270919E
:100F3000AC1240835183628373838F5F809313125B
:100F40000CC01092131282E0D82E06C1B70184EFB4
:100F500095E20E9444768AE013D7EEDECE01019638
:100F60006C010E94D3B38AE590E190937A1080934C
:100F70007910F70180818F3209F05CC087010F5F23
:100F80001F4F09F45DC06FE270E0C8010E945BED85
:100F90003C01009709F455C00817190708F051C023
:100FA0004C01801A910AA401B801CE0180960E94DA
:100FB00084EDE0E2F0E0EC0FFD1FE80DF91D10827A
:100FC000CE0180964C018C01F80181918F0188231C
:100FD00011F0D6D6F9CF8AE0D3D66091791070910E
:100FE0007A106115710511F06C5F7F4F21E0AE0141
:100FF000405E5F4FCE0105960E94AD7E811114C008
:10100000E0EEF5E284918F010F5F1F4F882319F006
:10101000B7D6F801F7CFF40181914F01882311F081
:10102000AFD6F9CF8EE282C0D0927A10C0927910FA
:101030008301A5CF8BE790E190937A10809379108C
:1010400087019091791080917A10692F782FBB20B9
:1010500009F457C06115710511F06C5F7F4F21E0F5
:10106000A80188EF91E10E94AD7E882309F445C074
:101070008091091290910A12A0910B12B0910C125A
:101080008093A5129093A612A093A712B093A812D2
:10109000B80182ED95E20E9444764091A5125091EC
:1010A000A6126091A7127091A8128AEC95E20E9494
:1010B0007E648AE065D61092A9121092AA1210924C
:1010C000AB121092AC12EBEBF5E284917F019FEF33
:1010D000E91AF90A882319F053D6F701F6CFB801B7
:1010E00080E090E0D4DD80913D10882319F08DE3FD
:1010F00090E101C0C80160E027C0B80187EA95E22D
:1011000010C06115710511F06C5F7F4F26E5A801D5
:1011100088EF91E10E94AD7E81110AC0B80183E998
:1011200095E20E9444768EE22BD68AE029D60EC044
:1011300081E080932B10B70181E895E20E9444760C
:101140008AE01ED660E0C8010E945D56C6010E947A
:10115000E3B328C0DD24D394EEE7FBE284918F0152
:101160000F5F1F4F882319F00BD6F801F7CFECEF74
:10117000F5E284918F010F5F1F4F882319F000D68D
:10118000F801F7CFE1E0DE1619F00FEF13E002C02F
:1011900005E014E0F80181918F01882309F4D6CE8F
:1011A000EFD5F8CFAD960FB6F894DEBF0FBECDBF2A
:1011B000DF91CF911F910F91FF90EF90DF90CF9033
:1011C000BF909F908F907F906F900895CF92DF9205
:1011D000EF92FF920F931F93CF93DF93CDB7DEB7BC
:1011E000EDB6FEB6DC010D900020E9F79D01281B4D
:1011F000390B2C5F3F4F4DB75EB7421B530B0FB6F9
:10120000F8945EBF0FBE4DBF0DB71EB70F5F1F4FE7
:101210009F938F938AE795E29F938F931F930F93EA
:101220000E9498E5680154E0C50ED11C0F900F9004
:101230000F900F900F900F90F6018081882349F056
:10124000082E000C990B0E941FEDF60181936F018F
:10125000F3CF60E0C8010E94E070882319F0C80154
:101260000E94E69186E795E29093520C8093510C90
:101270000E94FC700FB6F894FEBE0FBEEDBEDF916B
:10128000CF911F910F91FF90EF90DF90CF90089535
:10129000AF92BF92CF92DF92EF92FF920F931F9384
:1012A000CF93DF93CDB7DEB7AA970FB6F894DEBF22
:1012B0000FBECDBF809159108F93809158108F939E
:1012C0008DE695E29F938F937E0181E2E80EF11CFB
:1012D000FF92EF920E9498E50F900F900F900F9061
:1012E0000F900F9010E0F70101900020E9F731977F
:1012F000EE19FF091E1784F46701C10ED11C17FDFA
:10130000DA94F6018081082E000C990B0E941FEDE3
:10131000F60180831F5FE7CF40E050E0BA018EE521
:1013200090E10E948E7800E0CE0101966C018091E0
:101330006110823028F4011114C08FEF9FEF16C0A6
:101340008091661090916710A0916810B09169101B
:101350008F719927AA27BB27892B8A2B8B2B59F7AB
:101360001AC080915810909159100196909359107D
:1013700080935810AA960FB6F894DEBF0FBECDBF6B
:10138000DF91CF911F910F91FF90EF90DF90CF9061
:10139000BF90AF90089540E050E0B6018EE590E137
:1013A0000E94D67B18163CF6F60101900020E9F762
:1013B00031971E2F1C19115068F05601A10EB11C57
:1013C00017FDBA94F501808190E00E941FEDF501B0
:1013D0008083F1CF8A858E3709F4A9CF45E050E0AC
:1013E000B701C6010E9476ED892B09F0A0CFC70195
:1013F000EDDE01E09CCFCF92DF92EF92FF921F9340
:10140000CF93DF9310922E1080916110882321F0EA
:101410008EE590E10E94A57E1092D5111092D21116
:1014200085E38093D1110E94A750EB01A89561E05C
:101430008091D1110E946C4F81ED91E10E9496D272
:101440002398229A219A209A289A85E08093D31192
:1014500082E58CBD1DBC1AE08FEF0E949BD211501B
:10146000D9F720E030E0A90160E081ED91E10E9430
:10147000C1D2182F8093D411813049F00E94A75017
:101480006C1B7D0B613D774060F381E054C02AEA1C
:1014900031E040E050E068E081ED91E10E94C1D28E
:1014A00082FF03C01093D5110EC014E00E94A0D299
:1014B0008093D4111150D1F78A3A11F082E03BC0E9
:1014C00082E08093D5118091D511823021F0C12C1A
:1014D000D12C760105C0C12CD12CE12C80E4F82E52
:1014E00020E030E0A90167E381ED91E10E94C1D2E3
:1014F000A701960169E281ED91E10E94C1D280933A
:10150000D411882349F00E94A7506C1B7D0B613DCC
:10151000774030F38AE00FC08091D511823011F509
:1015200020E030E0A9016AE381ED91E10E94C1D29F
:10153000882351F088E08093D21181ED91E10E94DF
:1015400096D2EEE7FBE21AC00E94A0D2807C803CDB
:1015500019F483E08093D5110E94A0D20E94A0D2FA
:101560000E94A0D281ED91E10E9496D21092D311F7
:1015700081E00E9480A681112EC013C08491EF01EA
:101580002196882319F0FCD3FE01F8CFEFE5F5E2B0
:101590008491EF012196882309F450C0F1D3FE0114
:1015A000F7CF80E00E9480A6811115C0E7E7F6E240
:1015B0008491EF012196882319F0E2D3FE01F8CF40
:1015C000EBE4F5E28491EF012196882309F436C01B
:1015D000D7D3FE01F7CF66ED71E18EE590E10E9471
:1015E0001F7E811114C0E7E7F6E28491EF01219696
:1015F000882319F0C5D3FE01F8CFEAE3F5E2849120
:10160000EF0121968823D1F0BBD3FE01F8CF81E012
:1016100080932E10EEE7FBE28491EF012196882360
:1016200019F0AED3FE01F8CFEEE2F5E28491EF01BE
:101630002196882319F0A4D3FE01F8CF8BE1EEE5C3
:10164000F0E1AFE7B0E101900D928A95E1F780916A
:101650005C1090915D1090937E1080937D108AE5D0
:1016600090E190937A1080937910DF91CF911F9140
:10167000FF90EF90DF90CF9008950F931F93CF933B
:10168000DF938C01EB0190910B1020910C109213C1
:1016900007C08FEF9FE00E94E96C0E94C65BF3CF0A
:1016A000F801A081B1814881598180910A1034E00C
:1016B000839FF0011124ED5FFF4EB387A28755870A
:1016C00044879F5F90930B108F5F821719F0809370
:1016D0000A1002C010920A10DF91CF911F910F9152
:1016E0000895CF93DF93CDB7DEB78091500C811171
:1016F00010C09E01275F3F4F4F81588562E470E024
:1017000086E492E00E94C7E50E942FA883E08093C0
:101710004002DF91CF91089580911D1090911E108D
:1017200081309105B9F1029759F40E94F9A76093AD
:101730001F1070932010809321109093221018C0D6
:10174000109223101092241010922510109226103F
:1017500010922710109228101092291010922A101F
:1017600010921F101092201010922110109222102F
:1017700081E090E090931E1080931D100E94A7506E
:10178000609323107093241080932510909326105B
:1017900081E0089580E0089580911D1090911E10C1
:1017A000019791F482E090E090931E1080931D10B9
:1017B0000E94A750609327107093281080932910DF
:1017C00090932A1081E0089580E00895BC0180E0A4
:1017D00090E04AE0DCD28DE0D3D28AE0D1C28F9291
:1017E0009F92AF92BF92CF92DF92EF92FF92CF93F0
:1017F00020E030E04AE754E4FC016081718182819D
:1018000093810E9464E60E9466EB6B017C01611586
:1018100071058105910561F097FF0AC0F094E0948D
:10182000D094C094C11CD11CE11CF11C8DE201C0FC
:1018300080E28093490CC701B60128EE33E040E016
:1018400050E00E94E6E98AE0882E912CA12CB12C70
:10185000CA01B901A50194010E94E6E9605D6093A7
:101860004A0C8EE280934B0CC701B60124E630E0AF
:1018700040E050E00E94E6E9CA01B901A5019401E7
:101880000E94E6E9605D60934C0CC701B601A501BA
:1018900094010E94E6E9C62FCA01B901A50194018D
:1018A0000E94E6E9605D60934D0CC05DC0934E0CF4
:1018B00089E49CE0CF91FF90EF90DF90CF90BF90B4
:1018C000AF909F908F900895FF920F931F93CF93A7
:1018D000DF931F92CDB7DEB7982F862F692F4983EC
:1018E0000E94ADCF9091D30F8091470C4981891709
:1018F00038F19091D50F8091460C981708F180919E
:101900003D108823D1F0109252100DE310E14423D2
:1019100019F082E00E94A6D085E1F82EF8018191AD
:101920008F01882321F00E948FD0F81AF7CFFF2073
:1019300039F080E20BDAFA94FACF00E310E1E7CF56
:101940000F90DF91CF911F910F91FF900895CF924B
:10195000DF92EF92FF92C0908902D0908A02E090CD
:101960008B02F0908C028091B812882321F120E044
:1019700030E0A901C701B6010E94FFE58823D9F034
:1019800020E030E040E05FE3C701B6010E9464E67A
:101990009B01AC010E9464E62BED3FE049E450E47A
:1019A0000E9464E69B01AC0160E070E080E89FE388
:1019B0000E94FEEA04C060E070E080E89FE360936C
:1019C0009502709396028093970290939802FF90ED
:1019D000EF90DF90CF9008952F923F924F925F92B9
:1019E0006F927F928F929F92AF92BF92CF92DF922F
:1019F000EF92FF920F931F93CF93DF93CDB7DEB794
:101A000068970FB6F894DEBF0FBECDBF1C015B0117
:101A10008A01DC01D7966D917D918D919C91DA9729
:101A20000E9403E66B017C01F50120813181428136
:101A300053810E9464E60E94E8EA0E946BEB69878A
:101A40007A878B879C87D8012D913D914D915C9130
:101A5000C701B6010E9464E60E94E8EA0E946BEBAF
:101A60006D877E878F87988B29853A854B855C8526
:101A7000283731054105510540F488E790E0A0E0A2
:101A8000B0E089879A87AB87BC872D853E854F85D7
:101A90005889283731054105510540F488E790E021
:101AA000A0E0B0E08D879E87AF87B88B91012D5B5A
:101AB0003F4FD9018D919D910D90BC91A02D8D83AB
:101AC0009E83AF83B887BC01CD010E9405E6698380
:101AD0007A838B839C8369857A858B859C850E941C
:101AE00003E6698B7A8B8B8B9C8B20E030E0A9011D
:101AF00069817A818B819C810E94FFE5882339F17D
:101B0000A7019601C701B6010E9464E64B015C0182
:101B100029893A894B895C89CA01B9010E9464E626
:101B20009B01AC01C501B4010E9421EA4B015C019B
:101B300029813A814B815C81CA01B9010E9422EA64
:101B40009B01AC01C501B4010E94FEEA03C060E044
:101B500070E0CB010E94E8EA0E9466EB2B013C0199
:101B60006D817E818F819885909580957095619526
:101B70007F4F8F4F9F4F0E9405E64B015C016D85A3
:101B80007E858F8598890E9403E66D837E838F838F
:101B9000988720E030E0A901C501B4010E94FFE56B
:101BA000882349F12D813E814F815885CA01B901B1
:101BB0000E9464E66D8B7E8B8F8B988FA7019601B8
:101BC000C701B6010E9464E69B01AC016D897E8964
:101BD0008F89988D0E9421EA6B017C01A5019401F7
:101BE000C501B4010E9422EA9B01AC01C701B60104
:101BF0000E94FEEA03C060E070E0CB010E9497EB18
:101C0000F10182889388A488B58875016401C4189D
:101C1000D508E608F7080E9466EBC61AD70AE80A54
:101C2000F90AF7FE6BC020E030E0A90169817A81F2
:101C30008B819C810E94FFE5882309F447C029819C
:101C40003A814B815C81CA01B9010E9422EA6B0191
:101C50007C01C501B4010E9403E69B01AC01C701F0
:101C6000B6010E9464E66B017C0129893A894B899F
:101C70005C89CA01B9010E9464E69B01AC01C701FD
:101C8000B6010E9421EA6B017C012D813E814F81CA
:101C90005885CA01B9010E9464E69B01AC01C701E5
:101CA000B6010E9422EA6B017C0120E030E040E8AE
:101CB00050E469817A818B819C810E9464E69B015A
:101CC000AC01C701B6010E94FEEA03C060E070E00B
:101CD000CB010E94E8EA0E9466EB2B013C0197FFD2
:101CE00003C0412C512C3201481459046A047B046E
:101CF00010F024013501C12CD12C76018FB7F89456
:101D0000D1019C9193FD22C0F101468A578A608ED1
:101D1000718EC40CD51CE61CF71C5A96CD92DD9230
:101D2000ED92FC925D9729853A854B855C85DB9623
:101D30002D933D934D935C93DE97FF962D853E85C5
:101D40004F85588920833183428353838FBF6896A0
:101D50000FB6F894DEBF0FBECDBFDF91CF911F91BC
:101D60000F91FF90EF90DF90CF90BF90AF909F903A
:101D70008F907F906F905F904F903F902F9008953D
:101D80009091C00095FFFCCF8093C60008958F927C
:101D90009F92AF92BF92EF92FF921F93CF93DF93E8
:101DA000CDB7DEB7A0970FB6F894DEBF0FBECDBF9C
:101DB000611571058105910579F110E0842E912C52
:101DC000A12CB12CEE24E394F12CEC0EFD1EE10EBF
:101DD000F11C17FDFA94A50194010E94C4E9F701D2
:101DE0006083B901CA011F5F611571058105910505
:101DF00049F7115010F1E1E0F0E0EC0FFD1FE10FA9
:101E0000F11D17FDFA9580818A3010F097E301C02B
:101E100090E3890FB5DFEDCF80E3A0960FB6F8947D
:101E2000DEBF0FBECDBFDF91CF911F91FF90EF902E
:101E3000BF90AF909F908F90A3CFA0960FB6F894CD
:101E4000DEBF0FBECDBFDF91CF911F91FF90EF900E
:101E5000BF90AF909F908F900895CF92DF92EF92B6
:101E6000FF926B017C0197FF0AC08DE289DFF0943D
:101E7000E094D094C094C11CD11CE11CF11C4AE038
:101E8000C701B601FF90EF90DF90CF9080CF8F9287
:101E90009F92AF92BF92CF92DF92EF92FF92CF9339
:101EA0006B017C01B42E20E030E0A9010E94FFE527
:101EB00087FF06C08DE264DFF7FAF094F7F8F0943C
:101EC000C0E060E070E080E09FE3CB1541F02DECD6
:101ED0003CEC4CEC5DE30E9464E6CF5FF6CF9B01E7
:101EE000AC01C701B6010E9422EA6B017C010E948D
:101EF0006BEB4B015C014AE04ADFCC2379F1C50171
:101F0000B4010E9403E69B01AC01C701B6010E9427
:101F100021EA6B017C018EE233DF20E030E040E219
:101F200051E4C701B6010E9464E64B015C010E94C6
:101F300066EB6B01770FEE08FF08C701B6018DDF76
:101F4000C701B6010E9405E69B01AC01C501B401C1
:101F50000E9421EA6B017C01C150F9F6CF91FF90FC
:101F6000EF90DF90CF90BF90AF909F908F900895AB
:101F70008FB7F8949091140D2091130D291759F0F3
:101F8000E92FF0E0ED56F34F208130E09F5F9F771F
:101F90009093140D02C02FEF3FEF8FBFC90108953A
:101FA0001F920F920FB60F9211240BB60F922F9320
:101FB0003F938F939F93EF93FF932091C6009FB71A
:101FC000F894E091130D81E08E0F8F773091140D0E
:101FD000831731F0F0E0ED56F34F20838093130D1B
:101FE0009FBFFF91EF919F918F913F912F910F9004
:101FF0000BBE0F900FBE0F901F901895CF92DF92DF
:10200000EF92FF92CF93DF93EC01C090F10BD09051
:10201000F20BE090F30BF090F40BA70196016881AE
:1020200079818A819B810E94FFE587FF04C0C88275
:10203000D982EA82FB82C090F50BD090F60BE0903B
:10204000F70BF090F80BA70196016C817D818E81D2
:102050009F810E94FFE587FF04C0CC82DD82EE8273
:10206000FF82C090F90BD090FA0BE090FB0BF09040
:10207000FC0BA7019601688579858A859B850E945E
:10208000FFE587FF04C0C886D986EA86FB86C09034
:102090001B02D0901C02E0901D02F0901E02A701CE
:1020A0009601688179818A819B810E9448EC18168B
:1020B00024F4C882D982EA82FB82C0901F02D090A9
:1020C0002002E0902102F0902202A70196016C818B
:1020D0007D818E819F810E9448EC181624F4CC8269
:1020E000DD82EE82FF82C0902302D0902402E09035
:1020F0002502F0902602A7019601688579858A85D8
:102100009B850E9448EC181624F4C886D986EA8676
:10211000FB86DF91CF91FF90EF90DF90CF900895F5
:102120004F925F926F927F928F929F92AF92BF92E7
:10213000CF92DF92EF92FF920F931F93CF93DF9393
:1021400000D000D0CDB7DEB77C01FC01E354F84DE0
:10215000149182E0E816F10421F481E07CD681112B
:102160001EC16701CC0CDD1CCC0CDD1CC6018F54DC
:10217000984D0E9465714B015C01612F110F770B27
:10218000880B990B0E9405E62B013C0120E030E012
:1021900040EC5FE3C501B4010E9464E6A301920133
:1021A0000E9464E6AB01BC0100E010E09801C701A9
:1021B00064D492E0E916F10479F48DEA97E20E9482
:1021C000657120E030E040EA50E40E94FFE587FDC1
:1021D00009C08DEA97E203C0C6018B55984D0E9455
:1021E000657104C060E070E080EA90E49B01AC019E
:1021F000C301B2010E9464E64B015C0120E030E0C3
:10220000A9010E94FFE5882309F456C000E010E010
:102210009801B501A4017058C7012FD486E0E4E10C
:10222000F3E0DE01119601900D928A95E1F7F70136
:10223000EE0FFF1F81E090E08C0F9D1FE80FF91F4C
:102240008081918118161906C4F0EEE7FBE28491B3
:102250008F010F5F1F4F882319F092DDF801F7CF30
:10226000E3E8F7E284918F010F5F1F4F882319F095
:1022700087DDF801F7CF8AE090E0BC01990F880B69
:10228000990B0E9405E69B01AC01F601E65EFC4F4E
:1022900060817181828193810E94FEEA2B013C0161
:1022A000A5019401C501B4010E9422EAAB01BC0161
:1022B00093018201C701E1D381E0F701E959FB4FA6
:1022C0008083F701E455FB4F8083F601E958F34F13
:1022D0001082118212821382C701A4D7C6018958C5
:1022E000984D0E946571860104541B4FF601E55913
:1022F000F34F20813181428153810E9422EAF8010B
:102300006083718382839383F2E0EF16F104D1F44A
:102310002091111330911213409113135091141303
:102320006091C4047091C5048091C6049091C70463
:102330000E9421EA6093C4047093C5048093C6048C
:102340009093C7040E945B71F601ED57F34FD601DD
:10235000A454BB4F8D919D910D90BC91A02D808375
:102360009183A283B38382E0E816F104C1F480E094
:1023700026960FB6F894DEBF0FBECDBFDF91CF918A
:102380001F910F91FF90EF90DF90CF90BF90AF9093
:102390009F908F907F906F905F904F905CC5269636
:1023A0000FB6F894DEBF0FBECDBFDF91CF911F9166
:1023B0000F91FF90EF90DF90CF90BF90AF909F90E4
:1023C0008F907F906F905F904F9008950F931F9321
:1023D000CF93DF938C01EEE7FBE28491EF0121962E
:1023E000882319F0CDDCFE01F8CFB8018AE697E228
:1023F0000E94447682E2C4DC8AE0C2DC81E0DF91A4
:10240000CF911F910F9108955F9AECEAF4E010824A
:102410008A9A11829FB7F894A8E0B1E08C9181600C
:102420008C939FBF1282129A08958C01E7E7F6E21F
:102430008491EF012196882319F0A2DCFE01F8CFE8
:10244000EAE4F7E28491EF012196882319F098DC01
:10245000FE01F8CF0E9446CED7DF0E94265961E0E8
:10246000C8010E9448560E94244C0E94B18684E014
:102470000E94DCCF8091A00F869586951092D60F92
:102480008093D70F86E492E00E94C7D08091A00F7E
:1024900086958695880F1092D60F8093D70F8BE381
:1024A00097E20E94BAD08091A00F86958695982FCA
:1024B000990F890F1092D60F8093D70F8EE297E273
:1024C0000E94BAD00E94F5A58111D1CF2FEF8BE4E5
:1024D0009DE1215080409040E1F700C00000F89459
:1024E0002FEF84E39CE0215080409040E1F700C052
:1024F00000000E9446CEA895FECF4F925F926F9249
:102500007F928F929F92AF92BF92CF92DF92EF9283
:10251000FF920F931F93CF93DF930E946E560E94FA
:10252000A7506B017C0110914102112309F45FC097
:1025300080915F0C9091600C009709F458C0409115
:10254000150D5091160D6091170D7091180D4601E3
:102550005701841A950AA60AB70AB7FC5AC08330F5
:102560009105F9F034F401970CF441C0EEE7FBE279
:1025700006C0049709F03BC0EEE7FBE226C0849159
:10258000EF012196882319F0FBDBFE01F8CFE0EB89
:10259000F6E28491EF012196882349F1F1DBFE01F7
:1025A000F8CFEEE7FBE28491EF012196882319F042
:1025B000E7DBFE01F8CFE9E9F6E28491EF0121962D
:1025C0008823A9F0DDDBFE01F8CF8491EF0121968D
:1025D000882319F0D5DBFE01F8CFE1E8F6E284911B
:1025E000EF012196882319F0CBDBFE01F8CF212FD4
:1025F00030E0A8EEB3E00E9412EAC60ED71EE81E35
:10260000F91EC092150DD092160DE092170DF092A2
:10261000180D80916E06843008F4BBD70E94A75035
:10262000C090670CD090680CE090690CF0906A0C38
:10263000C114D104E104F10459F10091630C10912B
:10264000640C2091650C3091660C0C0D1D1D2E1D27
:102650003F1D5B016C01A01AB10AC20AD30AD7FC64
:1026600017C0E7E7F6E28491EF012196882319F07D
:1026700087DBFE01F8CF6091610C7091620C84EFF2
:1026800096E20E9444768AE07BDB8BEE96E255C0B0
:10269000C0904202D0904302E0904402F090450284
:1026A000C114D104E104F104D9F00091630C10913C
:1026B000640C2091650C3091660C0C0D1D1D2E1DB7
:1026C0003F1DDC01CB01801B910BA20BB30BB7FDAF
:1026D00007C09091FD0F8091FE0F981709F460C11B
:1026E00080911D0D90911E0D909902C0019604C01D
:1026F000181619062CF4019790931E0D80931D0D4A
:1027000080911D0D90911E0D8E3E9240BCF0E7E72A
:10271000F6E28491EF012196882319F031DBFE0166
:10272000F8CFEBECF6E28491EF012196882319F0C3
:1027300027DBFE01F8CF82EC96E277DE60918A0615
:102740009091FD0F8091FE0F981791F0E091FE0F90
:102750008DE4E89FF0011124ED5FF84F60818091D6
:10276000FE0F9091FD0F891719F08F5F8F70F9CFD1
:1027700070E089E00E94A84F80912D0C882309F415
:10278000F9C000913C0210913D02D0913E02C091EF
:102790003F0260918806709189066E5F7F4F072E19
:1027A000000C880B990B0E9405E698014D2F5C2FB9
:1027B0000E94FFE587FDDEC0F090FE0F912CA12C5A
:1027C000B12CE12C8DE4882E8091FD0FF81609F4D0
:1027D0005BC08F2D90E0889EF001899EF00D112442
:1027E000E454F94F4281538164817581452B462B16
:1027F000472B81F44681578160857185452B462B97
:10280000472B41F44285538564857585452B462BBE
:10281000472BA9F1889E9001899E300D1124F90162
:10282000E454F94F6F0166857785808991890E940C
:1028300005E62B013C01F60162897389848995893B
:102840000E9403E69B01AC01C301B2010E94FEEAB3
:10285000F60123A134A145A156A10E9464E63B01E3
:102860006C019B01AC01692D7A2D8B2D9E2D0E9450
:10287000FFE587FF04C0962CA72CBC2CED2C81E033
:102880008F0D8F70F82EA0CF209134023091350239
:102890004091360250913702692D7A2D8B2D9E2D55
:1028A0000E9464E69B01AC01B8018D2F9C2F0E9411
:1028B00022EA6B017C0198014D2F5C2F0E94FFE5FD
:1028C00087FD14C00091380210913902D0913A026C
:1028D000C0913B0298014D2F5C2FB601C7010E94A9
:1028E00048EC18161CF08601DE2DCF2DC090190D76
:1028F000D0901A0DE0901B0DF0901C0DA7019601D1
:10290000B8018D2F9C2F0E94FFE587FF1CC020E09F
:1029100037ED43EA5CE3B8018D2F9C2F0E9464E6FB
:102920004B015C0128E431EE4AE75FE3C701B601E1
:102930000E9464E69B01AC01C501B4010E9422EA39
:102940008B01D82FC92FC801AD2FBC2F8093190D33
:1029500090931A0DA0931B0DB0931C0DB8018D2FF1
:102960009C2F0E9466EB709389066093880680E036
:102970000E9413CE0E94C65B8FEF9FE0DF91CF9144
:102980001F910F91FF90EF90DF90CF90BF90AF908D
:102990009F908F907F906F905F904F900C94E96C18
:1029A0005F9A1092AC048A9A1092AD049FB7F89483
:1029B000809108018160809308019FBF1092AE044E
:1029C000129A8ECECF93DF9380E090E00E943D5D1F
:1029D000C3E5DCE0688379838A839B8381E090E0B0
:1029E0000E943D5D6C837D838E839F8382E090E0B7
:1029F0000E943D5D688779878A879B87DF91CF91A9
:102A00000895CF93DF930E946B71E0916D06F0E023
:102A1000E453FB4F8081882371F0EEE7F6E2849166
:102A2000EF012196882319F0ABD9FE01F8CF8AE097
:102A3000DF91CF91A5C9DF91CF910895CF92EF9209
:102A4000FF920F931F93E0900002F090010200911B
:102A5000020210910302C090560428EC34E044ECCA
:102A600054E060EC74E08CEB94E00E94FBBC1F919E
:102A70000F91FF90EF90CF900895AF92BF92CF92B9
:102A8000DF92EF92FF920F931F93CF93DF9300D0CB
:102A90001F92CDB7DEB779015C01AA0CBB1CAA0C52
:102AA000BB1CC50184549B4F6C01FC011082118238
:102AB0001282138249835A836B837C830E945B71E9
:102AC00049815A816B817C81F60140835183628305
:102AD0007383C090560420E030E0A901B801C7011B
:102AE0000E94FFE5811108C0F501E65EFC4F3081D0
:102AF00021819281838104C0302F212F9E2D8F2D23
:102B0000E32EF22E092F182F28EC34E044EC54E089
:102B100060EC74E08CEB94E00E94FBBC0E945B5D77
:102B20001092EC040F900F900F900F90DF91CF91C7
:102B30001F910F91FF90EF90DF90CF90BF90AF90DB
:102B4000089580918A0D90918B0DA0918C0DB0917C
:102B50008D0D8093000290930102A0930202B09326
:102B600003028091880D9091890D90931A028093B1
:102B700019020C946B718091000290910102A09156
:102B80000202B091030280938A0D90938B0DA09363
:102B90008C0DB0938D0D8091190290911A02909333
:102BA000890D8093880D84E690E090931A028093BB
:102BB00019020C946B714F925F926F927F928F9279
:102BC0009F92AF92BF92CF92DF92EF92FF920F93BC
:102BD0001F93CF93DF935C014B01EA018901409081
:102BE000000250900102609002027090030228815E
:102BF00039814A815B816091C4047091C5048091E0
:102C0000C6049091C7040E94FFE587FF29C0F80120
:102C1000C080D180E280F38020E030E0A901C701CC
:102C2000B6010E94FFE5811106C0C12CD12C20E81D
:102C3000E22E20E4F22EC0920002D0920102E09235
:102C40000202F092030288819981AA81BB8180935C
:102C5000C4049093C504A093C604B093C704EEDEE9
:102C6000F801C080D180E280F38020E030E0A9014B
:102C7000C701B6010E94FFE5811107C095E5C92E85
:102C8000DC2C95E0E92E93E4F92EC0920002D0925C
:102C90000102E0920202F0920302F501808191812B
:102CA000A281B3818093BC049093BD04A093BE0421
:102CB000B093BF04F40180819181A281B38180939C
:102CC000C0049093C104A093C204B093C304B6DEC1
:102CD000288139814A815B816091C4047091C50467
:102CE0008091C6049091C7040E9448EC18164CF5D8
:102CF000F801C080D180E280F38020E030E0A901BB
:102D0000C701B6010E94FFE5811106C0C12CD12C7C
:102D100080E8E82E80E4F82EC0920002D0920102F2
:102D2000E0920202F092030288819981AA81BB811C
:102D30008093C4049093C504A093C604B093C704C1
:102D40007DDE0E945B5D4092000250920102609223
:102D5000020270920302DF91CF911F910F91FF90B9
:102D6000EF90DF90CF90BF90AF909F908F907F902B
:102D70006F905F904F9008959B01AC0160EC74E000
:102D80008CEB94E018CF8F929F92AF92BF92CF922C
:102D9000DF92EF92FF92CF93DF93CDB7DEB7289704
:102DA0000FB6F894DEBF0FBECDBF2091730C3091EB
:102DB000740C4091750C5091760C0E9422EA6B01C4
:102DC0007C0169837A838B839C838090111390901C
:102DD0001213A0901313B090141320E030E0A90157
:102DE000C501B4010E94FFE587FF0AC0A501940157
:102DF000C701B6010E9421EA69837A838B839C8391
:102E00002091C4043091C5044091C6045091C70478
:102E100069817A818B819C810E9448EC181654F458
:102E20001D821E821F821886BE016B5F7F4FCE01FE
:102E30000196A2DF28960FB6F894DEBF0FBECDBF75
:102E4000DF91CF91FF90EF90DF90CF90BF90AF9048
:102E50009F908F9008951F93CF93DF93CDB7DEB7E8
:102E60002C970FB6F894DEBF0FBECDBF9091AF0484
:102E7000981779F1182F60E070E080E291E483DF29
:102E80008091BC049091BD04A091BE04B091BF0498
:102E900089879A87AB87BC878091C0049091C104D1
:102EA000A091C204B091C3048D839E83AF83B88781
:102EB00019821A821B821C829E012F5F3F4F44ECB5
:102EC00054E0BE016B5F7F4FCE01099674DE109314
:102ED000AF0480E02C960FB6F894DEBF0FBECDBFD6
:102EE000DF91CF911F9108952F923F924F925F9261
:102EF0006F927F928F929F92AF92BF92CF92DF920A
:102F0000EF92FF920F93CF93DF93CDB7DEB7649725
:102F10000FB6F894DEBF0FBECDBF2B013C014901B7
:102F20005A0117018091000290910102A0910202C2
:102F3000B0910302898B9A8BAB8BBC8B60E070E005
:102F400080EA90E420DF85E595E5A5E0B3E4809391
:102F5000000290930102A0930202B093030219862B
:102F60001A861B861C8620E030E040E251E4C50151
:102F7000B4010E9421EA6D837E838F83988720E0CD
:102F800030E040E251E4C301B2010E9421EA6983CA
:102F90007A838B839C839E01275F3F4F44EC54E0F0
:102FA000BE016B5F7F4FCE01019605DE81E053DFEE
:102FB000882339F0C12CD12C80ECE82E8FE7F82E35
:102FC000F4C00E946B7120E030E040EA50E4609170
:102FD000730C7091740C8091750C9091760C0E941A
:102FE00022EA6B017C0169877A878B879C878091B5
:102FF000111390911213A0911313B09114138D8794
:103000009E87AF87B88B20E030E0A901BC01CD01DD
:103010000E94FFE587FF0CC02D853E854F855889AE
:10302000C701B6010E9421EA69877A878B879C874E
:103030002091C4043091C5044091C6045091C70446
:1030400069857A858B859C850E94FFE587FF0EC088
:1030500080E090E0A0E8B0E489839A83AB83BC83EE
:10306000BE016F5F7F4FCE01099686DE80E090E063
:10307000A0E0B0E48D839E83AF83B88720E030E08A
:103080004BE953E46091730C7091740C8091750C52
:103090009091760C0E9421EA69837A838B839C83CA
:1030A000BE016B5F7F4FCE01019666DE1092EC048D
:1030B00089DC80915B0C90915C0CA0915D0CB091CF
:1030C0005E0C8093C4049093C504A093C604B0938F
:1030D000C7040E945B71209111133091121340912B
:1030E0001313509114136091C4047091C50480911E
:1030F000C6049091C7040E9422EA6B017C01011171
:1031000006C060E070E080EA90E43DDE04C080E04C
:10311000A2DE81114FCF93E0291631040CF439C09F
:10312000EDE5F9E284911F01AFEF2A1A3A0A8823EC
:1031300021F00E94C08EF101F5CF43E0C301B2013E
:103140000E94478FE8E5F9E284913F01BFEF6B1AD7
:103150007B0A882321F00E94C08EF301F5CF43E063
:10316000C501B4010E94478FE3E5F9E284915F0154
:103170009FEFA91AB90A882321F00E94C08EF50199
:10318000F5CF43E0C701B6010E94478F8AE00E9455
:10319000C08E89899A89AB89BC89809300029093FB
:1031A0000102A0930202B0930302C701B601649624
:1031B0000FB6F894DEBF0FBECDBFDF91CF910F9158
:1031C000FF90EF90DF90CF90BF90AF909F908F9047
:1031D0007F906F905F904F903F902F90089580E187
:1031E000E3E8FCE0ACEBB4E001900D928A95E1F7E6
:1031F0000895CF92EF92FF920F931F93C0905604C1
:103200007B018C012FE83CE04BE85CE067E87CE068
:1032100083E89CE00E94FBBC1F910F91FF90EF9010
:10322000CF900895CF92DF92EF92FF920F931F936A
:10323000CF93DF93EC01CC0FDD1FCC0FDD1FFE0120
:10324000E055FB4F20E030E0A9016081718182816F
:1032500093810E9422EAFE01E958F34F20813181D7
:10326000428153810E9422EA6B017C01FE01E559F3
:10327000F34F6083718382839383CE01895B964D84
:103280000E9465718E010F50144FA70196010E9494
:1032900022EAF8016083718382839383CE01855C87
:1032A000964D0E946571C55EDD4FA70196010E9493
:1032B00022EA688379838A839B83DF91CF911F9170
:1032C0000F91FF90EF90DF90CF900895682F880FB7
:1032D000770B80915C0490915D040E945BED9C01F2
:1032E000909353048093520481E0232B09F480E0EF
:1032F000089580915204909153044AE050E060E0B8
:1033000070E001960E94F3E297FD1EC08091520486
:10331000909153044AE050E060E070E001960E9412
:10332000F3E26F3F71058105910509F07CF480910E
:103330005204909153044AE050E060E070E001963E
:103340000E94F3E2862F089580E008958FEF08959C
:10335000EF92FF921F93CF93DF937C0184E5B6DF5A
:10336000182F882339F1C5DF8823F9F0EEE7FBE257
:103370008491EF012196882321F00E94C08EFE01E6
:10338000F7CF8DE40E94C08EB701FF0C880B990B1C
:103390000E942D8FAEDF682F70E088E299E20E94D4
:1033A0002B768AE00E94C08E09C0A3DF809355046B
:1033B00010E004C08091560480935504812FDF9162
:1033C000CF911F91FF90EF900895E0915204F091FA
:1033D0005304818121E030E0803239F42F5F3F4F88
:1033E000DF01A20FB31F8C91F7CF8D3211F08B321A
:1033F00031F42F5F3F4FDF01A20FB31F8C918E324C
:1034000019F4E20FF31F818180538A3030F471DFA9
:1034100091E0811103C090E001C091E0892F0895EF
:1034200080915204909153044AE050E060E070E0D3
:1034300001960E94F3E2CB0108958091520490918D
:1034400053044AE050E060E070E001960C941BE405
:103450000F931F93CF93DF93C0915204D0915304E5
:1034600065E470E0CE010E945BED8C01CE01019617
:103470000115110541F460E070E0DF91CF911F91DB
:103480000F910C948DE1F801108260E070E00E94D1
:103490008DE125E4F8012083DF91CF911F910F91F9
:1034A0000895BF92CF92DF92EF92FF920F931F93F6
:1034B000CF93DF9383E8E82E8CE0F82E0CEB14E03A
:1034C00097E5C92E94E0D92EC0EBD2E0BC2E84E063
:1034D000B80E8991FBDE8823D1F0BADFF601208196
:1034E000211104C020915B04222331F0F8012081D6
:1034F00031814281538103C020E030E0A9010E9464
:1035000022EAF70160837183828393830AC0F80102
:1035100080819181A281B381F70180839183A2830D
:10352000B383F4E0EF0EF11C0C5F1F4F8FEFC81A4E
:10353000D80ABC12CECF86E4C9DE8823B9F088DF72
:1035400020E030E0A9010E9448EC18167CF480DFEE
:1035500020E030E040E752E40E94FEEA609300027F
:10356000709301028093020290930302DF91CF9146
:103570001F910F91FF90EF90DF90CF90BF90089533
:1035800067DF20E030E04AE754E40E9464E60C94F0
:103590006BEB2F923F924F925F926F927F928F923E
:1035A0009F92AF92BF92CF92DF92EF92FF920F93D2
:1035B0001F93CF93DF931F92CDB7DEB70E94FC70AD
:1035C000811180C280916E06843058F42FB7F89430
:1035D0008091130D9091140D2FBF891B8F7709F0E7
:1035E00047C180912D10882309F46CC280916E062A
:1035F000811102C01092870DEE24E3944091A9122C
:103600005091AA126091AB127091AC128091A512E8
:103610009091A612A091A712B091A812481759072D
:103620006A077B0708F4E12C00E010E099249394EA
:1036300080E6882E99EFC92E98E2D92E25EFA22E8A
:1036400028E2B22E3DE8732E80916E06843008F099
:1036500039C2E11037C28091870D811133C2809148
:10366000001290910112A0910212B0910312809366
:10367000A9129093AA12A093AB12B093AC1241E09E
:1036800050E0BE016F5F7F4F88EF91E10E94B47AF6
:10369000019719F4898190E002C08FEF9FEFF82E17
:1036A000EE24E3942090A9123090AA124090AB121D
:1036B0005090AC124091A5125091A6126091A712A1
:1036C0007091A8122416350646065706C8F4E12C58
:1036D0008F3FEFEF9E0709F47CC0FAE08F1709F4E3
:1036E00097C02DE0821709F493C083E2F81619F011
:1036F0009AE3F912A3C08091860D81119FC083C007
:10370000E4E1F9E284912F012FEF421A520A882353
:1037100021F00E94C08EF201F5CF0E945B5D88EF20
:1037200091E10E94A57E80911312882359F1815066
:1037300080931312789EC001112441E061E0885EFD
:103740009D4E0E94E686E091131284E0E89FF0010E
:103750001124EC5EFD4E4081518162817381409362
:10376000A9125093AA126093AB127093AC1288EF17
:1037700091E10E948E7880912E108823D1F0909252
:103780002D1017C010922D10D092520CC092510CD7
:103790000E94FC700E94E0A70E94F9A76D3371059A
:1037A0008105910530F0B092520CA092510C0E940C
:1037B000FC701092B11280912E10882319F00E9493
:1037C000488921C00E94FB8980912E108111F7CF7A
:1037D0001AC0E7E7F6E284912F019FEF491A590AD0
:1037E000882321F00E94C08EF201F5CFE5E0F9E2D6
:1037F00084912F012FEF421A520A882321F00E9450
:10380000C08EF201F5CF83E2F81202C09092870DCC
:103810001092860D0115110509F416CF80916A04E6
:10382000889E000D111D1124F801E351FB4F1082F9
:1038300080E00E94CD7000E010E006CF0F3511054A
:1038400008F002CF9BE3F91202C09092860D80919E
:10385000860D8111F9CE80916A04F801889EE00DF1
:10386000F11D1124E351FB4FF0820F5F1F4FECCE8F
:103870000E94B88F20911F0D3091200D8A3019F0D1
:103880008D3009F0EEC01092850D2115310509F437
:1038900099CEF901EB5DF24F10821092200D10923B
:1038A0001F0D25E23DE06901F90180812F5F3F4F47
:1038B0008032C9F386018E3411F0C12CD12C6AE21A
:1038C00070E0C8010E945BED5C01C114D10409F4F1
:1038D00076C060EF78E2C8010E947EE5FF24F39491
:1038E000892B11F4F12C09C06EE470E0C801049634
